:20000000003A0120D924020039FB021039FB021039FB021039FB021039FB021039FB0210E2
:1C00200039FB021039FB021039FB021039FB021039FB021039FB021011FB021002
:200040002DE9F04FAB4EC34C05460121ADF1540DAF78327894F842000E91297845293FDC6F
:20006000452900F0078728291EDC282901F03980002901F0F982891E01F0E382491E01F064
:200080005583491E01F04E83C91E01F0CF82491E01F07882491E01F06B82DFF8C0C2C91F5E
:2000A000122952D901F0F0BA2A3901F00980491E00F0FF87DFF8A0C2491E00F098870E398F
:2000C00000F03887491E01F01883491E01F01183491F00F00287891E00F0EE8601F0D4BA27
:2000E000D8291CDCD82900F007814A3900F0A886491E00F08F86491E00F08286491E00F0CB
:2001000074865339242935D92D3901F0C982491E00F0B283093900F01F8201F0B5BAE13983
:2001200001F0B882C91E01F0B182891E00F0C680491F00F09880BC4A0E397CD0491E46D026
:20014000491E3ED0491E01F09FBADFE811F0070AC709A9099D0AE60A910982099D0A600952
:200160003F099D0A0A09DB089D0AE20ADF0ADA0AAE08DB07DFE811F0B90AB50AB10A320665
:20018000AD0AA90AA50A2D069E0A1006D305A20577056605560546053A0530052705990A06
:2001A0001E050405DC04A2047E047104FE03F203E703880A880A880ABC039C03880A880A7E
:2001C0008A036868002801F0998000F00BBE6868002801F093801146097831F0010140F0B0
:2001E00001860488466802208DF820003146ADF8224009A829F0E4FD08A815F0EDFB012888
:2002000015D14FF6FE70A0420BD0304628F00CFC28B9002120460A4626F074F808E00020B0
:2002200006E0002130460A4621F084FA00E00E980F95139055E1696891B11046007830F05E
:20024000010040F0CF85084600218DF820100990022108A88DF821101DF080FE01F01EB980
:200260000F9501F04BB86868007878B9002027F0D1FE26F0F1FF0E980DA98DF834005220DA
:2002800025F0CAF928F0A0FA01F054BA4FF6FF7027F0C0FE30784FF4807122F041F830787D
:2002A0004FF4807120F03AFE00200DF135018DF83500522025F0B0F901F03CBA68680028A5
:2002C00001F03882A34C01886180807A60B929F0D8FE40F28A21B0FBF1F220780821521D7D
:2002E00029F039FF01F026BA708F0E9928F0EEFE01F020BAE4FA002068680F95002800F0DD
:20030000FD8700681090807E27F06EFF061C00F0B0821098C76900252C464FF00309387821
:20032000A04200F3FF800F2410FB04F0401CC0B240191CF08FFC5FEA000800F0988224F00A
:20034000B7F9002840F0EC800025139588F800504CE0C0464CFF002098FD00201C030120FA
:200360001099032315FB03F6BA1991F81AA0B1F80C9052880F2015FB00845046494625F073
:20038000EDFBBA195288834608AB504623F0E4FB641CBBF1FF0F1AD0C8B1A6489DF827304D
:2003A0000168D80838BF8C2012D39DF826001623207103FB0B10C18800F10E02A4F80510D3
:2003C0000189C4F80B201398A4F8071000E086202070B8194078BB1960705888608098F8BB
:2003E00000006D1CEDB2401C88F800003878A842B6DC1098817E474600F10E064FF00F093D
:2004000085893A78109190F80AA01196139912950C468A4267DC204629F03EFF061C5BD0E5
:20042000139D024641E0C046ADFE002015FB09F0391838184078491C02F8010B487802F84B
:20044000010B887802F8010B4888001202F8010B0B7843BB4B78F3B9087902F8010B48796A
:2004600002F8010BB1F80500001202F8010BC87902F8010BB1F80700001202F8010B087920
:20048000834628F09AFE70B1D1F80B10584617F0EFFA024607E0487A02F8010BB1F80900A7
:2004A000001202F8010B6D1CEDB23878A842BDDC139900910E98019002900391CDF810A0BA
:2004C0000594129A069610980791119909230FF0EFFE304629F020FE384624F05DFB28F08A
:2004E000C3FC1398C6E111FB09F3F818FB185E78241DA4B2401C86B9467866B90079834699
:2005000028F05BFE641DA4B238B158461CF018FE001984B201E0A41CA4B2491CC9B278E765
:200520004046A2E114FB0972109930785288898908AB23F011FB50B19DF82600014628F0FE
:200540003CFE20B108461CF0FBFD2D18EDB2641CE4B2E4E69C03012068680F95002800F02E
:20056000CD8600681090807E27F03EFE002800F080811098D0F81C8098F80000002800F002
:2005800078818000401C1CF065FB0028119000F06E8129F08FFB24F08BF8002840F06481FB
:2005A00000261396129698F80000B04200F3E4801398012840F08C80CC4DA878EA68162119
:2005C00011FB00F081B2562029F018FD05F10C0640B9A8783268162111FB00F081B25620B1
:2005E00029F012FD6078802121F09AFE2F78B8001CF030FBB8465FEA000B69D02E78B8F141
:20060000000F0CD005F11800594642784A70428810F8144B4A807F1E01F8044BF5D1002EFA
:200620003CD037464FF000094FF0140AA6B305F1180411E0FC0C0120002808BF4E4607D0AD
:2006400041680668216124F0A7FA207B401E2073304624F0A1FA2E7820690028ECD1761EF3
:20066000F6B216FB0AF2A0184188618041786170C188E1808188A18001890C30218109C8CC
:2006800004F10C0181E80900105D2070A318C3F8109083F80C902E707F1EC7D10FF06AFC84
:2006A000B8F1000F11D018355C4647466078618825F042FEFF2804D02678810001EB0011F8
:2006C0006E547F1E04F10404F0D1584624F064FA12981199087018B9002048700E9F0F704C
:2006E000109890F81AA00C4600F10E098689857A2078042110FB01F0804629F0CDFD071C23
:200700001ED0014600202278824222DC012A03D164780CB9DDF83880002000900E99019112
:200720000291039004953246CDF81480072306974946079050460FF0BBFD384629F0ECFC70
:20074000119824F029FA28F08FFB26F0BFFA002090E08200A3185B780B70A3189B784B70A4
:20076000A318DB78A2188B70B2F80320401CC0B21212CA70091DC6E7109B9F890E2016FBD8
:2007800000856D1C93F81AA0B5F80190394650464A4625F0E3F9834608AB504623F0DCF938
:2007A000BBF1FF0F48D0002846D02F78002F58D19DF82600E97888423CD19DF82700C008B3
:2007C00036D3BD480168A8884FF6FF72824201D1EF88B7B1162202FB0B17F880E88838814F
:2007E000E87828F0EAFC00B30E370021042238461EF0ACF8E8781CF0A3FCD5F80A100246F2
:2008000010E0162000FB0B156889E880A889042205F10E070021288138461EF097F80422D1
:2008200005F11201384628F035FD0E98139018E08C2002E08D2000E08720129BDDF844C05E
:2008400099000CEB0102507028780CEB01075B1CB8700CEB0102DFB21297B5F80110A2F87B
:200860000310761CF6B29EE6119824F095F9102000E002200F9DB6E26868002800F03E853B
:200880006868006825F072FD00F008BEAF68002F00F0348500246C7040B12046014604F065
:2008A00019FB002808BF201C00F0B8810E98B5E16868002800F022850020696868700978BB
:2008C00061B984F8460094F82100401E84F821000E98014625F07AF900F02CBF29F058FBD8
:2008E0000E98014607F08EFE00F024BFF00C01206868002800F002850678476800210822B1
:2009000008A81EF023F8E7B1CD4800210170AEB1761E0ED0761E0AD0761E03D0761E10D1A4
:200920000E990170384608A918F0F8FEC2E20E990170384608A924F04FFABBE222F09EFDE0
:20094000B8E20220B6E26868002800F0D784686800F1120124F040FA00F0A0BD6868002899
:2009600000F0CC846A6810785188928817F05AF900F094BD6868002800F0C08490F800900B
:2009800046888188B0F806B0B0F808A00A301090C94807790F91002F00F03D81C5490F6865
:2009A000002F00F0AB8480467868007881454FD128F048FB00284BD0037C002B48D04469D8
:2009C000002C45D000200C22834240F3978410FB02F1615A8E4238D10E201CF03BF9071C52
:2009E00000F01981002407F10A0004235B1E00F8014BFBD1BC80FF2038704FF6FF737B80E2
:200A00003C81FC8087F800900F9A7E801099BA8007F10A00A7F806B00422A7F808A028F028
:200A200039FC08201CF016F9D8F8141018B9384624F0B2F8EFE007604160C8F8140098F802
:200A40001000401C88F8100067E1401CC0B2BBE73F68002FA8D100F051BC6868002800F0AE
:200A60004D840020687068681FF000F9A968088000F060BEA868002800F040840021697048
:200A8000AD68267860786F1C002E08BF29700ED0402124F061F84FF47A710F2300F2E7309D
:200AA000B0FBF1F116FB03100F3828702678002F00F040863046B2E0FC0C0120AF68A18FAB
:200AC00094F83F2094F83E3094F84060D4F838C094F841E094F8438094F8449094F845A074
:200AE00094F846B0002F00F0098400276F70AF683981A968CA72A9688B72A9680E73A968F3
:200B00008873A868C0F804C0A86880F80DE0606BA9680860A86880F80F80A86880F8109056
:200B2000A86880F811A0A86880F812B000F002BE6F68002F00F0E283002068706868077DDB
:200B400017B1C07C84F845006868877D17B1417D84F84610077C17B1C089A0876868077B97
:200B600017B18068A0636868877C1FB1407C84F84100686807790FB10068606300F0DABDE4
:200B80000021697070B194F83F0080090AD208A808221DF0DBFE28F0C3FF08A81AF084FD35
:200BA00000F0C8BD28F0BCFF4FF4FA7027F0FCFD00F0C0BDA868002800F0A0830020687080
:200BC00029F040FA2AE0D948A9680078002900F095830021697021E06868002800F08E83E9
:200BE0006868007822F088FE00F058BC6868002800F08483002068706868007806F0E8F90B
:200C000000F098BDA868002800F078830020687023F09CF908B90E98E5E00078AF68387069
:200C200000F088BD6868002800F068830020687069680888897822F057F800F07BBDC046C3
:200C400054FE00206868002800F05883B84C6968082204F10C0028F01DFB686801896180F4
:200C6000807A2070B3E06868002800F047830188ADF830104088ADF832000CA9532024F05C
:200C8000CBFC50200DF1320124F0C6FCE1200DF1360127F021F868689DF8361000798842C2
:200CA00000F095808DF836000DF13601E12024F0B3FC8CE024050120F00C012068680028B0
:200CC00000F01C83007825F033FA686896F83C104078884213D086F83C000DF13701E120CB
:200CE00026F0FAFF68689DF837104078884206D08DF837000DF13701E12024F08DFC686881
:200D00000E9F407807FA00F0F06428F04BF80024A6F89440384621F063FC204663E06F68CA
:200D2000002F00F0EB82387886F84A007C887487387A86F83C007B89F3877A68F264B9894C
:200D4000A6F84810B87B86F85C00F87B86F82900387C86F827007C697465B86996F896100A
:200D6000B065387F884201D025F0E2F9696806F15D001D3129F010FA96F84A0006F124048F
:200D8000082824D121207421224629F03DF90020022125F0F7F81AE06968002900F0AE8246
:200DA0000888498825F034FC70B9696808880E9A498823F049FD69680888498825F028FCC6
:200DC000002808BFC8200ED0696809794170002009E06868002800F0918203E0686800287B
:200DE00000F08C8212202C465BE26868002800F049846A6810889178D27825F083FA4DE3E0
:200E00006868002800F03E846868017A427A20F091FC43E36868002800F0348441788DF880
:200E2000201081788DF82110007828F001F8002800F064820C3008A9022228F02BFAC6E751
:200E40006968002900F01E84A868002800F01A84087808A927F063FB6868A96800780870C9
:200E60009DF82000A96848709DF82100A968887000F025BC6868002800F004840A3007783B
:200E8000002F0CBF00220E9A47780FB142F0020287780FB142F00402C7780FB142F00802A7
:200EA000007908B142F04002696808880023891C24F000FE044630E76868002800F0E283A3
:200EC00002206F688DF828003988ADF82010FA78B97808A821F0D4FAE0E26868002800F0FA
:200EE000D18302218DF8281001884FF6FF70884205D0821E8A4202D0C01E88420BD128F008
:200F0000D5FFADF820006868C27A837A811C08A823F08AFB687068680188ADF82010C27A08
:200F2000837A811C08A823F07FFBB7E2DC02012094FF00206C68002C00F0A48302208DF8D1
:200F400028002188ADF8201063462279B4F80680267AD4F80CB0277CD4F814A061880F92A0
:200F60001A1D14680346F21912FB03F00F305FFA80F9B9F1500F00F3198128F097FF88424B
:200F800033D121700812607028F054F9A41C0146204629F001F904460F98207084F801806F
:200FA0004FEA2823A370E670241D66B15846A41E017804F8021F30F8021B761E4FEA2121A2
:200FC0006170F5D1A41C27705FB1641E5046017804F8021F30F8021B7F1E4FEA2121617037
:200FE000F5D1C74820224B465EE01846FBE66C68002C00F0478302218DF828102088E14663
:20100000ADF820006288A388A679D4F80880277BD4F810E0D9F80400F41914FB01F1891D9C
:201020005FFA81FCBCF1500F42DC9DF828100F2918BF022908D1BDF820404FF6FF71A14223
:2010400004BF891EADF820104FF6FF71914208BF8A1E00F8012B111200F8011B00F8013BCB
:201060001C1200F8014B00F8016B66B14146801E0A7800F8022F31F8022B761E4FEA22224C
:201080004270F5D1801C07705FB1401E71460A7800F8022F31F8022B7F1E4FEA22224270D3
:2010A000F5D148460622634608A91FF037FD9AE67CE06868002800F0E5820220052216E0AD
:2010C0006868002800F0DE8202206F688DF828003988ADF820103A79798808A827F094FB82
:2010E00081E66868002800F0CD82022002468DF8280068680188ADF82010418808A827F07D
:201100007BFECBE12C466368002B00F0CC80187D27F0E2FE002800F0C6809D691C331F7830
:20112000002F0CBF002002205F780FB140F010009F780FB140F00800DF780FB140F0200026
:201140001F790FB140F040005F790FB140F0800083466068007D28F0A5FD5FEA000800F076
:20116000A2806168887A8DF829008889ADF82A00087802288DF828000CD001280AD00F2887
:2011800008D0032809D1891C08A8082228F082F8616802E04888ADF820008F7B002F72D0A6
:2011A00078001BF057FD061C02D1254610201AE600216068877B8F425FDCC18A838CCDF8B2
:2011C0003C80826A13950C2F109190F822901193BDF8208012924ADA404620F03FFD0C28E2
:2011E00014D14FF6FE7020F039FD0C280ED1BA4A0E9992F8D4500020DC3212F8083B9D424B
:20120000C4BF1D1C081C491C0C29F6DBC24D4FF6FE7305EBC00568686B8018B123F0BCFCBA
:201220000020686077B14FEA470A50461BF012FD6860002808BF10201AD0686831465246B4
:2012400028F028F8A5F80280C3486F70129B0078139F28700F990093109A019708A8CDF8EC
:2012600008B0119BCDF80C900DF06AFA00E002206070304623F090FC5CE200694A00105A06
:20128000491CB05295E7886A00900195CDF808B091F822000390CA8A8B8C08A841460DF0F9
:2012A0004FFA2546FAE0254628E0686830B3007827F012FE071C21D0387B22F0F7FA0028E9
:2012C000687040F03782AE4845683E46002D00F031822F46002117B9BE4202D02AE2BE4212
:2012E00009D1B54219BF3068086031684160304628F00AFF1EE239463F68ECE7022072E502
:2013000098FD00206868002800F0BC81A868002800F0B881002108221DF018FB69680878D6
:20132000498826F0CDF8071C19D00020A968687038880880A968B8788870AC68A078002817
:2013400000F0F8811BF086FC6060AA685068002800F0F0819278F91C27F09CFFEAE1B12017
:201360009CE06F68002F00F08D81AF68002F00F089810024664668686C70376801782046B3
:201380003FB13A79914204BF401CC0B23F68002FF7D1A9680870A868007840001BF05AFCF6
:2013A000A968376848606868A96800784968002F00F0C0813A79904204D1FA88661C21F8F4
:2013C0001420F4B23F68002FF4D1B3E16F68002F00F058816868002764466F7006782068AF
:2013E00090B101798E420BD1002F04BF0568256002D001683960056823F0CEFB284601E036
:20140000074600680028ECD123F0C6FC92E102206F686870002F00F08D81644639787A888F
:201420002068002800F0868100270379994202D1C3889A4204D0074600680028F5D179E1BC
:2014400007B967460168396023F0A6FB23F0A4FC35E16868002800F01581807800280CBF37
:2014600000220E9A68680E9900881FF0E5F815E06968002900F00681887828B1C878002810
:201480000CBF0E99032100E000216A68107908B141F040011088527913F01AFC687049E1B1
:2014A0006868002800F0EE80696808A80822091D27F0F0FE032027F071FF6868C07B24F037
:2014C00007FF6868817B009102788389418808A815F076FEE2E7C046200100206868002829
:2014E00000F0D080384627F0E9FC041C16D11C201BF0B0FB041C00F01D8100211C221DF01F
:2015000025FA2771204624F07DFB38B9204623F043FBD120C2E7C046F4010020E08887498D
:2015200040F00800E08040F00400E080022028F017FD8349032028F013FD68680168089148
:2015400000798DF824000E9F8DF825708DF8267008A820F05FF8A1E7C6FE0020686800280C
:2015600000F0908068680088002103F0B3FCE1E06868002800F086806868007870709EE0FB
:20158000281A00206F486F680478002F7AD0686800212A2269701DF0D9F9708F6968088019
:2015A0006868B6F84870847269688F81F08F6968C8826868082206F1240707F139010E30F8
:2015C00027F068FE27F036FE014668680822801C27F060FE6868082207F11C01183027F083
:2015E00059FE96F83C10686880F823100E986968554C81F8210021784A0824BF6A6882F873
:2016000024008A0824BF6A6882F82500CA0824BF6A6882F826000A0924BF6A6882F8270030
:20162000C90924BF696881F8280083E0686848B390F90000044627F0EDFBA86800B104704E
:201640003DE06868F0B100200E9F687069680F7069684F7068680226867068680624C4705B
:20166000696803230B7165E0686858B1407818B1FF20032124F086FC28F024FC0E98334925
:201680000860FEE7022009E7122007E729461DF0EFFB4EE000202E496870EF780F7049E0B9
:2016A000002068701CF0CEFA44E00020687025F01DFF3FE010464FF4807120F073FA0020CB
:2016C000ECE629461FF02EFB33E0294613F0B0FC2FE0294618F034FF2BE0294628F002FB18
:2016E00027E0294621F018FF23E0294621F0CDFB1FE029461EF0D0FB1BE0294619F096FEB3
:2017000017E0384629460EF08FFA12E027F06AFEC4E6294620F040FC0BE03846294607F0B9
:20172000E5FB06E0294607F0EDF802E0294607F065FA0E900E9815B0BDE8F08FD1480200A9
:20174000519A020034FD0020E61201207C052043481900202DE9F04704464FF6FE70ADF1E5
:20176000600D217AADF85400606808AA13F0A4FF002800F072849DF822000228B4BF0127BE
:2017800000279DF824000228A8BF0027BDF82A104FF000084FF6F87088420ED04FF6FE7073
:2017A000401F884209D04FF6FE70001F884204D04FF6FE70C01E884200D1474628F070FB7B
:2017C0009DF82310884240F04884002F00F04584208D9DF82660678EDFF80093ADF84C007B
:2017E000ADF82E70D6B161689DF821209DF83C30012027F0A3FD002840F02F844846001DF1
:20180000007801280AD1208D28F066FC30B1417901F0EF01417141F0080141719DF82570E1
:201820004546002F4BD19DF83D00474658BBBDF82A00034623F050F94646022808BF012638
:20184000002E9DF8226018BF0127B9F83A10994208BF47F0020727B1002E14BF40202020EE
:201860000743184623F038F9012808BF47F00107002E3DD01298007828F01CF9012818BFC3
:2018800027F0010734E09DF8411041B1FF2906D09DF84000119A24F001FD50B128E0B9F8F3
:2018A0003A00BDF82A10884205D099F84A0004281ED101251CE09DF82660222721E0BDF82E
:2018C0002A10FF2025F0FCFD002804BF3E1C082708D09DF8250047F001062C2740F00100D9
:2018E0008DF8250006F00306012E08BF47F011079DF8266007F002012846084308BF47F02E
:20190000800796B999F82F0078B107F0220022280BD007F04200422840F09F8312980078B3
:20192000062818BF072840F09883B8111690F80956D399F832001299BDF82A2080080AD2BE
:201940000878C01E01282CD9001F2AD0C01E28D0801E26D003E00878401E0A2821D9B8F1E2
:20196000000F1ED1B9F83A00904240F076830D780520BDF82C408DF8110004A826F044FE1E
:20198000002800F06A830269032313271370511C0F704C7022128A70CD7044800AF06CF9BE
:2019A0005BE3169840081BD30878032802D148780D2815D09DF8280038B1BDF82C000E997F
:2019C00011F0CCF9012800F044839DF8270038B1BDF82A000D9911F0C1F9012800F03683AA
:2019E000B9F84800B4F84410884209D1CDF80080208DB4F8421094F84620434613F0E2FEFC
:201A00009DF82600002846D0208DB4F8421024F0FFFD9DF85150061C25D19DB999F890004D
:201A200001283AD112980078062802D11698400833D2BDF82E104FF6FE70401C884240F058
:201A4000B6800AE3042026F048FD011C00F005836420087001274F70208D488099F8000066
:201A600021F01AFEF9E29DF82130606819184A7BF1788A4203D0F270404670606068C0185E
:201A80000421401C26F0DFFF7168814200F2E582401C706001E09DF8515099F8320080084E
:201AA000C0F0DB820DB3BDF82C0027F09FFBB8B9BB49BC4CBDF82C000B6822699901A1EB45
:201AC00083019047012840F0C8826169BDF82C008847A168BDF82C008847BEE2E4FA002037
:201AE0006168487800F0DF0048709DF8320038B161688879401E8871C0B28DF8320008B91B
:201B000007F07F07380924D39DF82500F9084FF4805814D279091AD3811011F0070F01F04C
:201B2000070604D0072E1CBF761EF6B20EB907F07F0700F0E30040EA8600C0B205E020F04A
:201B40001C00C11021F0030108438DF825006168087299F84A00042800F00082092800F0B1
:201B6000FD8117F0610F40F0E6809DF82200012811D112980078052800F0D68003280AD17D
:201B8000BDF82A0027F032FB28B1218D08A815AA002300F0FBFE9DF8320068B99DF8220081
:201BA000012804D112980078032800F0568208A8214620F041FD50E226F0AEFF002840F060
:201BC0004C829DF83D0000286DD19DF82400BDF82A10FD100028ADF854102ED13A0930D2D5
:201BE0009DF82220012A28D0084600211DF000FC002620B14079012816D0022814D0BDF8F1
:201C00005400B4F8441024F003FD28B1807826F097FC08B1082807DBBDF82C0027F0E6FA3F
:201C200018B104208DF824000126BDF82A10301C08BF022272D09DF824006A0838BF00233A
:201C400000D340230DF13D021DF00CFC30B16168087848F0200800F03F0008709DF83D00F9
:201C600040B1BDF82A1010A822F016FF48F04008ADF854009DF82200012806D0BDF82A0097
:201C8000BDF82C1000221AF01BF868082CBF40220022BDF82C10BDF82A0016F0EDFB08B1BE
:201CA00048F0200833E09DF840009DF84110119A24F0F4FA00282ED09DF8410038B9BDF8A7
:201CC0002A00ADF8540028F007FA00BB1DE011999DF8286001EB400030F8020C002EADF814
:201CE00054000CBF082010209DF827600EB10830C0B29DF82560002106B1012140186168B3
:201D0000401CC2B2505C401E505448F0400826F0C9F91690A3E0BDF82A100B22BDF82C00C7
:201D200000231DF01DF998E1218D08A815AA002300F02CFE91E10020169078086AD3B4F8E9
:201D400028A09DF833C0B74D1E211698EA79944506D1BDF82C302A88934201D1AE782EB9B8
:201D6000491E05F1080500F10100EFD11E2826D0AE790EB3B9F84810504625F0A9FC08B111
:201D8000761EAE71B64833210279FF2A02D00288924509D0491E00F12400F5D107E0C0465F
:201DA0006CBC0200ECFB0020A879401EA871A8796628A4BF1698A87127F060072AE026F0E3
:201DC00071F916909DF8320028B9BDF82C00218D814202D11EE0BDF82C00B9F83A10884282
:201DE00002D199F80600A8B1218D169A08A812F06DF858B1380932BFBDF82A004FF6F870E4
:201E0000C01D48F00408ADF8540003E0002027F020071690B8094FEAA71510D394F8460056
:201E200094F8476094F948308DF81000E26B8DF8116004A98DF8123008A804F0DBFC680833
:201E40000DD3218D169B08A815AA00F09FFD169028B112980078012808BF48F01008BDF8B2
:201E600054104FF6FE70884204BF002016907E481B30007801282BD1618E4FF6F870C01DD1
:201E8000884225D0218D884222D0BDF82A204FF6F870401C90421BDDBDF82C00884217D0B5
:201EA00028F01AF9A0B10179012918BF02290FD101218DF810104088ADF81C0004A821F013
:201EC0000DF828B105A820F095FD08B125F0C8FE37F07F0000F0C1801698002800F0BD8067
:201EE00020891AF0B7FE071C00F0B7806168228927F0D0F9002605969DF822008DF81000CF
:201F00001699009104ADCDF80480B046CDF80880BDF854100395228D237A384617F05CFC6A
:201F2000C0B999F80100002800F09780BDF82A00ADF81A0045468DF81E508DF81D50BDF8A4
:201F40002C70ADF81870169E8DF81C6006A827F0F1FA82E0384622F01FFE7EE04149BDF8A7
:201F60002A000988814209D022F0B6FD022805D09DF8250000F0030001286ED19DF822007A
:201F8000002851D012980178042903D19DF83C10022942D00178072905D19DF83C2099F8B5
:201FA0000000042A06D0032957D108A8002115F0E7F952E04FF4806120F0B2F9092089F858
:201FC0004A0029484178022904BF0021817727F031F901460D9827F00BF801283DD11020D8
:201FE00026F07BFA07460E991298002F00F1010033D002223A704378027802EB03227A8085
:20200000807878704A2023F007FB9DF8260010B9164905200870394620E5002008A90DF08F
:2020200017F81AE0CC02002094F8460094F8477094F948608DF81000E26B8DF8117004A9CA
:202040008DF8126008A804F0D5FB06E0BDF82A0001E0BDF82C0021F021F918B0BDE8F0877F
:20206000E40D00201EFB0020ACFE002034FD0020C64A2DE9F04FADF14C0D10780F91090C62
:2020800080F058840F99890B80F025840F99890980F054830F99490980F0D6820F98DFF8DE
:2020A0000093C00980F060820F98000A06D321F09DFD0F9880F0800000F05BBC0F98DFF821
:2020C000D8B2DFF8D882DFF8DCA2400A80F0DC800F98000B80F0C28010460F99C078490BEC
:2020E00080F0B2805C460F99606AC90B80F096800F992078890863D20F98E188800A40D21E
:202100000F98000907D3114601200F9F887187F0080000F02EBC0F98C00A0AD31046B0F871
:202120004800012122F05EFA0F9880F4806000F020BC0F98400C38BF0020C0F01A84544612
:20214000332501262434207980B105280EDA607900090BD28DF804606088ADF8100001A8DB
:2021600020F0BCFE10B102A820F044FC6D1E04F12404E8D1854900200F9F087187F4803039
:20218000F7E310461746B0F84850A7F848105020A11D23F041FAE6883227444660898542FE
:2021A00005D0864204D0204626F0EBFF00E066817F1E04F11C04F1D10F9880F40070D8E3C7
:2021C00040B301A827F08CFF27F05EFE49460546032091F8228091F823608DF80D0003A8DD
:2021E00026F012FA071C15D038690B2100F8011B00F8018B06700126BE7727F01BF878627A
:202200007D807E7701A838620023BE763846237009F032FD0F9880F00200AAE380B1494693
:202220001431097801290BD18047A06A00B18047564800784FF480414FF47A7227F088FFA2
:202240000F9880F4804094E320B100201146C87022F062F90F9880F480508AE322F05CF980
:202260004946087A01280BD1497A49B1474800784FF47A7212FB01F24FF4006127F068FF33
:202280000F9880F4006074E327F010FE4FF6FE71814200F06581104690F832008008C0F0B2
:2022A0005F8100252C46284625F03AFC071C1AD03879012817D0022815D0F879334E411CC2
:2022C000F97196F88B1081420DDABC727C72388824F03CFC388801A925F03DFE01A820F026
:2022E00089FB25F0BDFC6D1C332DDCDBA8F11C0632274FF6FE75119436F81C0F85420DD07E
:20230000307B224C411C317394F88B10814205DA1198B0747074308824F018FC7F1EEBD1F0
:202320005C46032104F1380010F8047F0FB17F1E0770491EF8D15446332605F1010934F8FC
:20234000240F81451FD001208DF804006788ADF8107001A820F0C2FDA8B1A8F11C053227F3
:2023600035F81C0F2188814208D0BDF80610814204D002A8A91C26F03BFE10B1284626F05C
:2023800000FF7F1EECD1761ED9D101E0E4FA0020119D2C4608E0C046ECFB00206C0800201E
:2023A000ACFE0020C00D0020284625F0B9FB48B1017931F0040105D1807A26F0C1F808B13E
:2023C000641CE4B26D1C332DEEDB25F0D3FF119E5FEA00080ED03546284625F08FF928B111
:2023E000807C26F0ADF808B1761CF6B26D1CEDB2A845F1DCA019C7B2002F41D0B8001AF01D
:2024000029FC1090002808BF119F3BD0BA00FF211CF09CFA119E3546B44218DD284625F039
:202420007FFB031C10D0187930F004000CD1987A26F086F8011C07D0009718885A7A109B41
:202440001BF06BF9761CF6B26D1C332DE4DBB8F1000F17D0119C204625F050F9061C0AD01F
:20246000B07C26F06DF8011C05D00097109B3088727C1BF052F9641CE4B2A045EBDC01E0E2
:2024800011981090BB4890F83000002808BF4FF0620805D026F046FFC0F154005FFA80F89A
:2024A0000320B8F1600F98FBF0FAA8BF4FF01F0ADDF840904FF6FE7BABF1020BB8F1000FD1
:2024C0000EBF119D2025DDF84480BA45A6BF3C1C45F040055446032014FB00F0801C8DF890
:2024E000050001A826F090F84E46031C26D01869082104F01F02017045EA02014170801C38
:20250000A4B12246C01E361F16F8041F00F8031F318809124170B17801F0070CF178521EF5
:2025200001F0070141EA0C118170EDD1A3F802B001209876184609F09FFB00E00120E9094B
:2025400006D2641EE4B20CB109EB84093F1BFFB205F040052843B1D0109808B122F01CFB92
:202560000F9880F4807004E2B64C1E25002106264FF00408A078002840D0401EC3B2607991
:20258000A37026F0FDFC071C37D05BB9787B022808BF7E7331D07E733868407BF02121F097
:2025A000D1FD2AE0A3791BB9787B032813D024E0237913B3E078401EC3B2E370EBB96D4815
:2025C00090F82500E0702079401EC3B22371787B032812D123B92046394622F03DFB0CE006
:2025E00087F80D8027F04DFD624B00F00F00401C3881187820211FF0D5FA01216D1E04F15C
:202600000804B7D15B48007801290FD040211FF087FE494691F82900012811D1002081F828
:20262000290018F0C3FD25F01BFB09E0402122F093FA28B94F4800784021642227F088FD22
:202640000F9880F0400094E1102122F085FA30B94848007810214FF47A7227F079FDB34813
:20266000DFF8CC82417808F52774491ECFB217BB012141700020052126F076F9071C1BD07E
:2026800006253846052126F06FF90646388978B1401E80B2388158B97889C00802D3387B0C
:2026A00024F03CFA7D733868407BF02121F04AFD371CE6D100E0477096274FF6FE760025E0
:2026C0002079A0B1FF2812D0401E2071C0B270B96079032805D16088218802221EF082FC62
:2026E0006079012803D0268066806571A5717F1E04F10804E4D108F184040827207A401E92
:202700002072C0B230B99C48214624F06FFB90B9668025707F1E04F10A04EFD1974A0C21D1
:2027200012F8080F08B1401E1070491EF8D10F9880F010001DE121F09DF9E4E7202122F0C7
:202740000BFA28B90B480069002808BF01261BD027F0CAFE044627F08BFB8B4F4FF47A7108
:202760006043B0FBF1F13869002808BF002008D002E0C046E4FA002088428CBF4FF0FF3038
:20278000081A460869D0FFE70020042126F0ECF8071C62D04FF00009FF254FF0FF3B062407
:2027A0004FF0010A3846042126F0DEF810903889864204D8801B83B23B8113B14AE0A7F822
:2027C0000890BB7B012B02D17889C0083CD3ABB38DF804508DF805508DF806B03968086AF5
:2027E000C97F02AA12F068FFC846012808BFD0465FEA08001DD0788A40F08000ADF836009D
:20280000B87B8DF838007889000908D3BDF8360040F48070ADF83600387B8DF83A007B69A3
:2028200013B1187BADF8180001A94A4602A803F0E1FF7C73387B1BF0D5FD0BE087F80DA037
:2028400008E0C046CC0200207C733868407BB72121F078FC109F002FA4D10FF0FFF84A481A
:2028600003780121002026F07FF818B1184620211FF098F90020042126F076F8B3B278B1AF
:20288000414A0789147826F06FF8F8B9BB42AEBF0027FF1ABFB2204627B920211FF082F937
:2028A00000200DE07A00202127F055FC27F01CFE044627F0DDFA4FF47A716043B0FBF1F022
:2028C000314908610F9880F0200052E00289BA42D8BF171CD7E727F079FC294C0546201D14
:2028E0000068074698B1284857F80C1C007821B94FF400511EF012FB03E04FF400511FF06C
:2029000051F9204639460022001D23F04FFF284627F0E6FD2FB13846FEF71CFF384625F07F
:20292000C3FE0F9880F4005023E0C046D4130120200100201FF008F9071C17D01149203154
:202940000A78FF2A0FD03C780B460020944207D0401CC0B2C200D1189A5CFF2AF6D102E0DA
:20296000496838468847384625F09EFE0F9880F4004013B0BDE8F08F39430200EC0100205D
:2029800038050120E0B80200E4FA00202DE9F04F064693460020ADF13C0DABF80000B06A03
:2029A000099303460078884627F084F848B17089044622F091F8022804BFABF80040B36A95
:2029C00001D0002009901878C84DDFF82493401E0A2800F20984DFE810F02D03B1020A0473
:2029E0009E028D0151010704BE00880066000B00BD4C207D012840F0F7835B1CB06913F881
:202A0000015B1F7827F098FB002800F0F5830379002B00F0F183032B80F2EE830E2D1CDC3A
:202A2000DFB9D04907752DB901EB85010A6BC261096B0AE001EB85010B6B9A01A2EB830286
:202A4000C2610A6B9101A1EB82018161012180F8201025F005F9002500E001250320B689F1
:202A6000A47F8DF8190006A825F0CEFD071C00F0C38338690C2100F8011B00F8015B047004
:202A80000124BC7726F0D6FB786204A9304625F062FA10B17C7704A838627E80BC763846E1
:202AA00009F0EAF8A8E35C1C207820F01F0700F01F00012840F09883641C04A8214627F03D
:202AC0006BFB284604A95D3026F092FA002800F08B83002F40F088830834A27861782078EF
:202AE00001EB022123F06EF986E3688F7189884240F07A835C1C14F8016B04A8214627F0E2
:202B00004BFB284604A95D3026F072FA06F01F0726F01F06002800F06F83002E40F06C8397
:202B200078001AF097F8011C00F0668367B184460834384663782278401E04F1020402EB37
:202B400003222CF8022BF5D100910AF03AFD084622F022F850E35C789A1C34F07F0704F0A2
:202B60001F0E40F04983377F03201EFB00F0801CC1B2B94240F04083002714F01F0F04BF31
:202B80004FF6FE7C614618D0D9789B7870464D4603EB012C5378117812F802EF01EB0321C0
:202BA0003EF0770340F028832B888B4208BF0EF00707521C401EEDD1BFB960464FF6FE72E2
:202BC000824212D004F06002602A0ED04D462A88A30907D2E30902D2904203DD0CE3904294
:202BE00003DD09E39142C0F20783B08927F074FA002836D1B0894FF6FF7124F069FD041C85
:202C000014D123F0EBFC041C00F0F68200211C221BF09CFEB0894D460E3520802888608109
:202C2000AA23A3740622227401216174207C0C2805DB0620072F2074BCBF7F1CFFB26774B9
:202C400000202073A01C25F0EFFE002840F0D482307A002800F0D082B169A01C27F09CFABE
:202C6000CAE20021C171017A0C2905DB0621072F0172BCBF7F1CFFB24772BDE2484671894E
:202C80000088884240F0B082307F022840F0AC82A94C201D00884FF6FE71814240F0AC82BA
:202CA000162025F01AFC071C00F0A68201213970B07900280CBF081C02207870B06A407891
:202CC000B872000902D2B08922F096FDB169B81C27F062FA0020F8742878394620F0DCFC1B
:202CE000B089A08088E2C046ACFE0020E4FA00201EFB0020708921F0EFFE002840F07482C5
:202D00005F78B84987B10C2F03F1020380F274828C463D465A7818786D1E03F1020300EBE1
:202D200002202CF8020BF5D1484675890488DFF8D492AC4200F0B180B37C002B00F05C82EE
:202D40003B1C0A974FF0000811D0A64A38464146921E32F8023F9C4206D0401E01F101013D
:202D6000F7D104E018BC02000A914FF00108284600211CF03DFB00280B907DD04079012829
:202D80007AD10B98807910F0180F75D00B984188384626F003F910B9B8F1010F6CD109F22A
:202DA0004C704FF6FE754FF000080C97B6F80CB008904FF0010A0D95C14611E0B8F1010F16
:202DC00008BF4FF0010908D027F05BF9C0B290FBF8F101FB08F1A0EB01094FF00008C246E1
:202DE000089D32271C3D35F81C4F4FF6FE70A04213D0A34511D00C98214626F0CFF860B9A2
:202E00006B7C53B1072B08DA08F10100BAF1000F5FFA80F801D1C14521DD7F1EE3D1B34D07
:202E2000332735F8244F0D98A0421AD0A34518D00C98214626F0B2F898B96B7A8BB1072BE8
:202E40000FDA287901280CD002280AD008F10100BAF1000F5FFA80F803D1C14501DC0D9402
:202E600007E07F1EDDD1B8F1000F02D0B9F1000FA4D00D980B994880B37C5A4C581EB074E9
:202E8000F77C00970A9D0195029401220392B189B269708918F098F8AEE1B4890C2F80F23E
:202EA000AB818846ADF81040BC488DF812700168CDF8148009B104A8884720461EF0CEFEE1
:202EC0000C2803D14FF6FE701EF0C8FE0C2880F2938109EBC005D435686808B121F05CFEF3
:202EE0002FB1780019F0B6FE686010B984E1002068606C80C2486F700078287068780028F2
:202F000000F07A816868002800F076817A00414626F0C0F970E1307F022840F06581099836
:202F200028B94D4671892888884240F06581099831460CF08DF85EE1ECFB0020B5F84810AF
:202F4000404623F065FBA846074608202FB17D781DB90621397007257D70B16A0A79CC789F
:202F60008B794D7891F802A0CF7904EB02244A7902EB03296A0928BF1020AA0924BF0830CC
:202F8000C0B235F0700340F03781327F904240F0338105F07005680938BF002006D306A85F
:202FA000083127F0F9F825F010050820A90907D3B16A091804A8083127F0EEF825F020059A
:202FC0002046514624F0A0F908280DDA8D4B410001EBC001C9188879B84240F30D818F71CD
:202FE000002002E0360100200420B8F83A10A14219D048B9B189484601222B4610F0CCFE67
:2030000028B1F9E020010020042840F0F58006A804AE009049463A465346019620460295C0
:2030200013F090FEE8E0B189484601222B4610F0B3FEE1E0B5F84810404623F0E9FA4FF0A9
:203040000609041C03D06078002800F0CD80B06A817847780891C378017900F1050A03EB23
:2030600001200990404620F063FB9AF8001009185FFA81FAB80928BF4FF00E0937F078006E
:2030800040F0B28007F01800182800F0AD80307F814540F0A9804FF00009CDF80090089956
:2030A000B089524643461CF017FA032800F09C80002807F078074DD117F0180F18D195F802
:2030C000310028B1B089414601223B4610F064FE09984FF6FE714A463B4610F05DFE002837
:2030E00038D14FF6FF70ABF8000039E0C00D002047F00107780928BF47F00207B0893946CB
:203100001CF076F990B1817911F0180F0ED0417901290BD154B14088B5F8481023F078FADC
:2031200020B1437813B1607898425DDCB089414601223B4610F030FE60B94FF6FF70347A47
:20314000ABF80000002C0CBF4946B169B089524625F044FEBBF800104FF6FF70884243D1AF
:20316000012000900899B089524643461CF0B4F90998394622F0D8F9698F81422ED109988C
:2031800026F0AAFF60B10079012818BF022807D1099804A924F0DFFE08E0C04674FD002026
:2031A00026F048F8014604A826F0F6FF307A012803D1B16906A826F0EFFF06A8009004AF57
:2031C0000197B06A407840F0300002900999089BB0894A4613F0B6FD48460CE0B06A80F8C3
:2031E00005A024F05FFF06E04FF00009F4E70999304614F0C5F8099009980FB0BDE8F08FB9
:20320000C6FE0020A40100202DE9F04FC24C04F128000768ADF14C0D17B1002087F8450073
:20322000DFF8F082002517F148030BD0BF6DB84E73612FB940460068D0F84C05804773695A
:203240005868706026F0C2FF1190082016F03CFC1CF09CFC464610B1B2A027F03DF91FF061
:20326000E3F8684626F040FB042069468DF80000284626F007FDE06326F08CFA09A826F0EE
:2032800061FC042009A98DF82400284626F062FC606326F089FA0DA826F064FC04200DA90F
:2032A0008DF83400284626F065FC616BA06319B9A4A027F011F9A06B10B9A7A027F00CF933
:2032C000E06B10B9A9A027F007F93068D0F8E00380473068D0F8180280473068D0F8F002DD
:2032E0008047404600682F460726A03001687B5823B11846804740460068A030761E07F128
:203300000407F3D1D0F8B8028047EB2026F0D4FDA06A2F4670B105A8FF2108221BF016FBF0
:20332000A06A05A9082225F0AFF904F12806012818BF3768924A0CCA05A8391C80E80C0004
:2033400021D1082019F086FC5FEA000856D0A8F10206032726F095FE06F8020F7F1E4FEAF8
:2033600020207070F6D12020F82706F8020F4146082204F1440088F8077025F08BFF4046F2
:2033800021F00AFC04E004F14400082225F082FF0120082105AA26F031FE04F14406002894
:2033A00018BF092826D124F022FE80081DD205A8FF2108221BF0CAFA07AFFF21082238461F
:2033C0001BF0C4FA0120294608223B4626F004FB80B9384605A9082225F056F928B930468A
:2033E0003946082225F056FF04E001200821324626F00AFEE220314622F00EF924F0F7FD5C
:20340000400834BF2E1C0126CA4F5520012107F1420226F0F3FD18B916B1284624F07CF880
:20342000C54FE22007F1440124F056FC30461FF0D9FC05A8294610221BF088FA3846407868
:2034400030F001000FD1BD4F05A91022384625F01BF928B905A83946102225F01BFF02E088
:2034600005A823F003FC6220102105AA26F0C6FD28B926B16220102105AA26F0C5FD05A8B3
:20348000294610221BF062FA304614F04DFE304622F086F8304615F0BFF81EB128460121C8
:2034A00022F070FD242019F0D5FB0028206400F0A481E06A216B221D1DF0F8F915490968CD
:2034C000D1F84C138847216C201D0860E06A216B04F108021DF0EAF910F05EFF216C04F11F
:2034E00008004860E06A216B04F10C021DF0DEF904F1300904F12C08D24ED34F3070D9F855
:203500000010D8F800C0266C2B4607F1100005E0DCFF002014010020D4DB002006F1080E0F
:2035200034E0C04652616E646F6D5F736565644175746F6D617469632829206661696C65F7
:203540006400C04641455343434D206F70656E206661696C656400C0414553454342206F0C
:2035600070656E206661696C656400C054524E47206F70656E206661696C656400C046C06B
:2035800004BF020040F823505B1CDBB2002BF9D07D61CEF80020604604F110021DF086F9C6
:2035A000C54F654EB870308EB880C24831463D703C3126F0F1FD04F110033046216C90F8F4
:2035C0002500CB60D9F80010787006F14C00F860D8F8000004F114021DF068F904F1180AD7
:2035E000B649B84AB64E0870B74BBE60206C7A6204F11406D9F800100661D8F80000BB6282
:2036000052461DF053F9B14EF071022286F824204FF6FE70B08325F00DFEAD48A54906F193
:20362000140B0560584626F0B7FDAA48FF2138221BF08CF9A848AA4B8360AA4AC260A749D4
:2036400041600570A84B0361A84A4261AA493961A74B8361A74AC261A84B7B61A84ABA6115
:20366000AA48A84BA84AFB61AA491061A84FD16006F13000976015F067F909270BF12C00B0
:203680007F1E40F8045BFBD1F07948F2010120F0CDFBF0794FF4004120F0C8FBF079212142
:2036A00020F0C4FBF079222120F0C0FB206CD9F80010C0F814A0D8F8000004F11C021DF0FB
:2036C000F5F8954E48F21501307020F0AFFB3078382120F0ABFB924F0222F760914B86F803
:2036E00028208E483361216C70614FF6FE7704F11C0304F12002D8F800008B61D9F8001038
:2037000037841DF0D3F8884AD580D5609570556101271574064615700648177148F202016A
:203720004670304620F082FB48F20101304620F07DFB05E04CFF0020ACFE002028BC020096
:20374000304648F2040120F071FB784E78483D49784B3061784A4B60084604F12003826023
:20376000D9F80010226CD8F80000D36104F124021DF09CF8714B207071499870284626F088
:20378000EFFB7049384626F0EBFB6F49042026F0E7FB6E49062026F0E3FB6D49072026F074
:2037A000DFFB6C49082026F0DBFB98784FF6FE71491C20F03BFB68487949684B8862684A36
:2037C0005A606848684A98600B46DA621846674A83F84670664F0263674BB760654A674FC0
:2037E0001848674E1360674AC76003461F461E61206C7A6104F12406066213F080FF14F0C8
:2038000067FD119826F06CFE11F0BCFD24F046FD64480068D0F8D40090F8430024F050FD2E
:2038200060480068D0F8582429460120904726F0A1F855485B4F05707868C068007860B9C9
:2038400004E0C0469C0301204819002038460068D0F8582428460146904719F093FE4C4F52
:203860003D704A48058145818581C581058245828582C58205832B464583464E8583072150
:203880000360464A43604448357024F0ADF919F055F921F0A3FE22F062F8434840780228C5
:2038A00004D14FF40040012117F0EAFA13B0BDE8F08FC046E0000120AC000120DC040120E7
:2038C00065490100F1AB0100859B020034FD00209CFF00206C010020FC0201207DA40000A1
:2038E000A98802004D0A02007B67020081800200C9600200A9850200058E010001770100ED
:203900003980020009C3000034040120D5650100D9DE0100E95B0100E80001207D5A0200AD
:20392000E5730200897C0200F00C012020040120619902005B9F0000DD390200281A002054
:20394000A19A0200659A0200799A02008D9A0200B5960200CD960200B5350200DC0201204E
:20396000D94902002D2F020085530200C543020057490200F0FA0020D5410200FD8101009E
:20398000311A0200AD420200061401208C110120FF130120FE130120EC0000205DA202007E
:2039A0004CFF002014010020ACFE00202DE9F04FCA4CCB4DDFF838B3DFF838930F46380C1D
:2039C000ADF11C0D80F05782DFF81883780880F0FD81C64EB80880F0C181B80980F0AA8115
:2039E000DFF804A3F80B80F04E81BB480668780980F02981380928BF87F0080080F05A8307
:203A0000780A80F0BA80F80880F0AD802069F90980F09080380A63D2B80A5CD2C44C380B18
:203A20002BD2F80A27D3142019F014F9061C1FD00025A846207A012813D10096042029464F
:203A40004246142321F0F6FE58B92068306060682946142233467060042022F0F3FD84F821
:203A600008806D1C0C34032DE4DB304621F094F887F480601EE300201CE3182019F0EAF855
:203A8000061C25D000252434A846207A012813D10096062029464246182321F0CBFE58B924
:203AA0002068306160682946182233467061062022F0C8FD84F808806D1C0C34032DE4DB79
:203AC0003046414618221AF041FF304621F064F887F40060EEE219F0ADFF87F40070E9E26C
:203AE0001CF04CFF2078052818D1E07904211EF017FCE07904211DF011FA062025F04EFC07
:203B0000287800F00700022801D026F083F824F0A7F819F08FFF23F04FFC01E024F0A0F84D
:203B2000012023F0F9FC0320012104F06BFD87F08000BFE2A0B117F089FB206906682069C7
:203B400021F02AF826615EB1F28802E0F088801AF0803668002EF9D1E079402126F0FBFA63
:203B600087F04000A6E2FF20032122F00BFA26F0A9F9C34901200860FEE7424692F84A001E
:203B8000082818BF04285BD124322120742126F03BFABC4D6868298800241BE0A30003EB15
:203BA000C403C65C36F07F0212D016F07F06C654034405D101A8FF210C221AF0C7FE01AB5F
:203BC000012021460C2222F03DFD284629884068641CA4B2A142E1DCB94C4FF0FF085546C0
:203BE0000026E06995F8211080291FD169798DF809102A798DF808206B88ADF806302888B1
:203C0000ADF8040085F82180297D8DF80C10EA798DF80B20AB798DF80A30A8690490314684
:203C2000102201AB032022F00DFDE069761C2435332ED7DB00B180470020022122F0A2F9B8
:203C400087F4807036E24EB17168087818B1486800781BF0D7FD3668002EF5D126F026F9F2
:203C60001C34208025F0E6FA484608300078012806D1444620784FF40061642226F06BFA5A
:203C800087F0100016E20120022123F035FFC4B294B3E00018F0DEFF5FEA00082ED0834680
:203CA0004FF00109554633262879012818BF02280DD18DF804906888ADF8100001A81FF0A8
:203CC0000DF920B102A9584626F066FA8346761E05F12405E8D111E02405012034FD00208D
:203CE000E4120120E4FA0020E40D0020C0FE0020E0120120ACFE00204FF00008B8F1000FE4
:203D000012D074B10F204FF6FC768DF80C001F25ADF8046001A922464346B148009516F0A9
:203D200043F8404620F038FF87F48040C2E1C04664FE0020207A50B92078062802D10720B2
:203D400025F02CFB3078012801D124F03DFDE07910211DF027FF87F02000ABE1207A00BB01
:203D60002178E07908291AD124F004FF092025F015FBB9480078052806D0072809D1072024
:203D8000012104F03FFC04E0012023F0F5FF1CF0F5FD3078012816D124F016FD13E01021C5
:203DA0000FE026F077F8EF2803DB002023F0E4FF09E026F06FF81030C0B226F07DF8E07988
:203DC00001211DF0EFFE87F0020073E1012025F0E5FA5D466678287900F00701122001296F
:203DE00018BF02293DD1E6B1032E1AD0012E38D1012936D10A2025F0D1FA444620784FF429
:203E000080611EF08DFA502005A923F065FFBDF81400A4F84800BDF81400002120F0E2FB13
:203E200026E025F0B7FE002818BF032E15D1022025F0B4FAA149E06809781FF0C7F8A97914
:203E400009090ED270B99E4A5178491CC9B20429517004BF9B49E16003E026F012F913F0D9
:203E60001FFA28B1E07901214FF47A7226F073F987F001001EE1DFF854924FF0000A10E1B6
:203E80007C052043300501204146934823780E784278701E00F0E280401E13D0183800F04A
:203EA000FA80B93800F0F3802A3840F0EC8086480168002900F0F28040468847EEE0C0464B
:203EC000FC020120012A18BF022A40F0E78099F820004E46072818BF082805D1227A1AB93E
:203EE000012104F08FFB2378032B7BD00A2B11D0042B14D00D2B12D00E2B10D00C2B0ED09D
:203F0000002B00F0CB8023F057FAE07910211DF049FEC3E0287800F00700012862D0237AC7
:203F200060785BBB84F80BA05046307120F038FBE0B120780D2819D00E2817D0062025F053
:203F40002DFA9BF806000BF10406000904D34FF40040012116F094FF307800F007000228B4
:203F600001D025F057FE23F027FA97E0052025F015FA42F2107024F017FC8FE0012819D1B5
:203F8000E07A401CC0B20428E07204DB5048007801280DD00EE04F4800884FF6FF71814201
:203FA00006D003206070012666710423A37201E084F801A022F032FF22F0A0F80BF1060011
:203FC0000078000903D34448007D012866D16078032863D10820012116F052FF5EE0C04605
:203FE00098FD0020237A002B33D1E07910211DF0D9FD20F0D5FA28B320780A2808D12978D5
:2040000001F00701022903D032490822891C0A7003280CD123F0D0F996F82000022806D152
:20402000012023F079FA0220012104F0EBFA062025F0B4F9287800F0070002282ED025F000
:20404000E9FD2BE0052025F0A9F9012020F0E4FE24E05046FAE7C0466CFF0020022B1DD159
:20406000012A18BF022A19D125F08CFF10B116F0AFF898B125F0BCFF00280CBF5046012057
:2040800021F006FB0AE040461CF026F906E0404616F05AFD02E0404610F0A8FA404624F006
:2040A00003FBE0791DF050FD5FEA00087FF4ECAE87F4004007B0BDE8F08FC0468DFF0020A9
:2040C00094FF002000F8FF07F40001204CFF0020AD0001202CFB0020ACFE00202DE9F04F7B
:2040E000B54CDFF8D8C294F8207088465FEAD800ADF1140D80F092825FEA184006D3DFF8AF
:2041000004B34FF6FF7AAAF1010A59E1604600785FEA5831A0F1020080F03181B84DA91DDA
:2041200009885FEA182280F0EA805FEA980180F0D1805FEA183028BF88F4006080F0558352
:204140005FEAD81080F0A280E7685FEA98305DD2A0695FEAD83138BF0020C0F04683A74932
:2041600028C96A4628C209881180676938B9384625F0E4FAA061C0B997B90B2011E0017BFE
:20418000FF2906D031F07F000FD101F07C0104290BDBE06940B9384625F0D0FAA06120B9A7
:2041A000002025F08FFD2EE0A06160784FF4804143F2C82225F0CFFF94F82010A06908295B
:2041C00019D00188ADF80010017A8DF80810017B491CC9B231F07F07017306D10188427A0D
:2041E000684624F011FBA06909E0008800210A4622F088F8F7E7017B41F04001017340698B
:2042000025F09CFAE06188F48040EEE2DFF8C0B200264FF0030AB14687B96078012E04D0D9
:204220004FF400511EF07CF805E04FF400514FF47A7225F090FF88F40050D6E27D68287813
:2042400010B3F02820DC51464A466B461FF084FCD0B1029803889BB984F83E908DF80DA0AA
:204260008DF80C9003AB0A204946524620F042FADBF8001084F83E9031B12878884703E071
:2042800001880126491E01803F68C5E71FF05EFE07462078BFB1401EC0B22070A0B16078EA
:2042A0004FF4804120F058FC30B9606925F046FA10B938781DF06EFA6078402143F6982275
:2042C00025F049FF207810B90B2025F0FBFC88F040008AE2B0F1FF3F18BF00280CD168465C
:2042E000002108221AF032FB684617F0DDF918B1607802211DF056FC88F0020075E208466F
:2043000000211FF0DBFD28460678FF24C6B14FF6FF75001D00212B4610F8142F52080BD324
:20432000C7884FB1BB4207D055B10289BF1ABAB29542C4BF0C1C151C761E01F10101EBD18D
:20434000FF2C19D02E49A00000EB0410401818300189C088401A80B250B929484470FF20E8
:2043600009F030FCFF2120460A4620F0E5F900202349C88024F078FA88F0800035E2B0F14A
:20438000FF3F18BF002814D13846401E0CD0801E0FD194F8220002280BD1012084F8220052
:2043A000002020F039FD04E094F82110002021F00DFC88F4805018E24CFF0020ADFE002040
:2043C00060781DF0C1FB051C08BF88F4004000F00C822F78D32F00F0098194F82000B84251
:2043E00012D00A2F40F0168194F83F002871A16A002900F00F81A81C88470BE1A8B60200E4
:20440000F00C0120E4FA0020B94840787F1E00F09680BF1E40F0FE80012818BF022840F040
:20442000F980AF787FB37F1E40F0F4806F7860781FB325F03BFD4FF6FE720021824218BF1A
:204440000121081C04D15846408F1146814209D010465F46ADF8100004A9A7F83AA0532098
:2044600021F0DAF822F0DAFC21F048FE5946002081F84A0019F0E6FBCCE0022140F6B832BF
:2044800084F82210A7E06878002854D125F0B0FD00210E4603460BF1080063621F460160AB
:2044A000002F44D1002B38D0002E1F4635D0B146C64824F056F801280CD08D48408E4FF699
:2044C000FF7181420CD03988884209D01BE0C046E0020120BD4807F10C0124F089FD90B180
:2044E000BBF83E003989884201D1824501D1FB784BB19BF836007979884209D17C48B97910
:20450000807B884204D0384621F030FF761EF6B2BF69B9F10109CBD1636A226B002AA9D093
:20452000184631469047206B002873D1A2E7BF69761CF6B2B4E7002021F0AAF86AE001280C
:2045400018BF022866D16F7894F845003FB194F84410491CC9B2884284F8441043DB94F877
:204560002100401E04D0401E3AD0401E1ED051E025F010FB98B994F8460020B1E06A00287D
:2045800048D0804746E0002102200F468DF808000246ADF80070684624F02EFC13E0012094
:2045A00025F0F6FC014604F02DF833E0AB2000216A461EF0D9FFCDF808D004208DF80C00AD
:2045C00002A812F0E9F960784FF480511DF0A8FE607841F288324FF4805125F0BCFD19E00E
:2045E00021F0D8FA16E001200021DCE7E88948F20101401A0BD0401E05D0801E0AD12846E1
:2046000019F0DEFA06E0284616F09EF802E0284618F0BCF9284624F047F8D1E66178381C17
:2046200009D0401E00F0DB80C01E00F0D180801E00F0C080D7E094F83F00C10880F09F8031
:2046400081087AD20009C0F0CE80062084F8200025F098FC00286CD01FF078FC2569071C7B
:2046600067D068684078800837D33878032100226B461FF071FA28B968684078410831D213
:204680000E201BE002980188B52912DAB421018060784FF47A724FF4005125F05CFD544809
:2046A000416829B10078FF2814BF3878FF208847256968684078400803D2092025F002FBF9
:2046C0000AE0092003228DF80C0003AB00218DF80D200A2020F00EF82569686840784108F1
:2046E000C0F0818043490E6826B9800821D37AE0ACFE002038781DF04DF8002600B1012688
:204700000325301C02D00E2025F0DCFA0C2020706078402143F6982225F01DFD0A208DF874
:204720000D5003AB00212A468DF80C001FF0E2FF59E00E2025F0C6FA55E0042294F84000F9
:2047400084F8202040084ED394F84270002F3FD160460078012818BF022844D1012504F13F
:2047600020000021E5701AF0F1F8032084F8200028461FF0C7FB284624F0CFFC33E004F15D
:204780002000052594F84010057089080FD394F8421061B90121E170042200211AF0D6F881
:2047A00084F8205000201FF0ADFB0220E4E72846002111E0002084F83E0084F820003222FF
:2047C0000846042125F0C7FC0DE0C04648FD002024F03CFB0420012103F014FF03E001209B
:2047E000014621F0F3F988F0040005B0BDE8F08FDC020120000301202DE9F04FBE48C84C8E
:20480000ADF1340D06902569406801214FF0E047C06809934FF000080170C24808921F40E6
:2048200080F800804FF0020000EA020008BF002840F0E682DFF8F092DFF8F0A21E4611464F
:204840004FF4803018EA060700EA010008BF002833D141464FF4003011EA060700EA02008A
:2048600008BF00280ED137464FF48000394000EA020008BF002800F0B78285F804801CF0A0
:20488000B5F9B1E285F80480EB2021F00BFE4A46514682F800800878862801D121F084FEFD
:2048A00025F094FCE1690A6882F804800968E16125F016FE24F08EFB96E285F8048021F096
:2048C00059FE81262778A4F80C809949A770994D0860994B2E70FF221A702169069E087AEF
:2048E000801E81B230684A46D0F8000182F80080C0890B918842C0F26B82E16908310968BA
:2049000004F1180001600426A6810B98657EA17E04F11902C01E80B2069EE37E0B9005EB83
:2049200001205178C1F301193168608101F1B80CDCF80010237109780792002908BFB9F163
:20494000020F00F04582B9F1020F00F3418219B110F0070F00F03C82667800F00705AD1EEB
:20496000022D08BF002E00F0338231B151460978862902D1002D40F02B82001300F00200E3
:20498000022864DA35435AD1DCF81C0090F88300022851D0E1690C31097805A80170052774
:2049A000A78125F013FC554606462878862840D106980068403001680F6837B9D0F80C0546
:2049C000804706980068006C07689DF9140025F041FC787706980068016C096881F81E8049
:2049E000006C9DF914100068C177304625F078FD2679678925F0EAFB51460A7807F0100741
:204A0000862A15D1BA4D05F11E031A88521C1A8087220A7025F064FDE879B04206D11FB99D
:204A2000404618F001FB07E01B20FAE7E920F8E70646304625F054FD24F0CCFACAE15146BD
:204A40000878862803D121F0AFFDA77866788FB186B9012F00F0BC816089022F03D110F0D0
:204A6000070F40F0B581032F05D100F00701032901D0ADE16089010980F0AA81011301F09C
:204A80000201022902DA810A80F0A28107994978C1F3810BBBF1010F4FEAA1110A9100F01B
:204AA0009781012900F09481B9F1020F14DA00F00701012918BF03290ED1BBF1000F0BD16B
:204AC0000A9F002F00F0848106990968AC3109680F78002F00F07C81BC49B9F1020F0DD06B
:204AE0000A9E11F80B708A5DB918CFB25EB3C10929D3BF1E12E0C046140100200A460A997D
:204B00000BEB0207891809793A795218C109D7B214D20A995BEA010615D0BF1CFFB212E0CB
:204B20006811012010050120071401200A140120E813012005140120250001200A995BEAA6
:204B4000010608BF02270B9AC0F30021781A61718242C0F23D81069E1046C01B4018316887
:204B600080B2D1F850122081743080B2884700286678606100F02C814146742219F0E6FE24
:204B800084F8038062891EB9C14902F020000870BF4861790678C446002E30D000292ED101
:204BA00002F00700032808D0012828D106980068D0F8D40090F882600EB30698406840691B
:204BC00006781EB124F022FEFE2815D006980068D0F84C02804750B906980068D0F8440249
:204BE000804720B96289617994F803C007E00420E0706289617901E00420E07084466569F4
:204C0000268905F1740305F17400AB65079B686093F801A02E812089CAF301190029A5F873
:204C20005C001878AA8100F0780049EA00004CEA000028744FF0FF06AE730CBF20794046A1
:204C400085F83AB085F849000A9885F83000A089002FA0EB010086B2A68100F0B480E16927
:204C6000E78068463A468919083116F03FFFBF19B8B2A0812846017C4FEAAA0212F0030F39
:204C800002F003076D4601F0400B42D0B9F1020F434601D1C9090BD29DF801209DF80010F7
:204CA00001EB0221A0F844100DF10205A0F84210814EB0F84410B6F846208A4203D04FF647
:204CC000FF728A4223D1032F14D06A78297801EB022189B24186B6F84420AD1C01208A4231
:204CE00014D04FF6FF728A4218BF181C0EE0C0464C02012060692946323025F04DFA606921
:204D00003B363146323024F073F908350346002B56D00798407886111ED06169B9F1020F91
:204D200003D0087CC00903D309E05BEA070306D16A782878AD1C00EB0220A1F84200032E0A
:204D400005D068782A7802EB00220A8504E060692946283025F020FA06990968AC310A685C
:204D60006089167886B1B9F1020F0DDA00F00702012A18BF032A0BD162692FB94F4BB2F8E8
:204D800042201B8893421BD100F00702032A05D0012A18D1886A90F88200A0B1D1F89C117B
:204DA0006069884778B9079881786769407884F80380C1F3011100F078000843387402E004
:204DC0001BF014FF06E00DF077FE03E0A8C3020024F0F2F825F0FAF9E1690A6882F804804D
:204DE0000968E16125F07CFB0899099E202047460840374008BF002830D024F0A5F82DE0F3
:204E00002F4991F90000002803DD91F90000401E08702C4991F90000002803DD91F9000097
:204E2000401E0870114640461E464FF080770840374008BF00280DD0234991F9000000287C
:204E400003DD91F90000401E087020480121017024F004FB85F804801BF0C8FEDFF864C037
:204E60009CF90070B7B108994FF0E0470220374000EA010008BF002816D09CF900000028A8
:204E800012DC06980068D0F84C0580470CE0C046071401200E48069F80F800803868D0F8B5
:204EA000582441460846904706984068C06880F800800DB0BDE8F08FDCFF00202200012045
:204EC000130501201205012014050120110501200E050120964A2DE9F04FADF13C0D00247C
:204EE0000A918E2309900121101D01708046D47240215171502593712046D0730021D17159
:204F0000DFF830B21172A02191729089917340F430509081204611681074C44CC24855726B
:204F2000084084F832304CF21011014300200C909BF80000116058B90C981DF053FF94F848
:204F40003200000910D30C9808A98DF8200008E094F83200000907D301200DF121018DF8EA
:204F60002100522020F058FB12F0C9FB24F022FADFF8E4A20B90002840F0C78011F082FD2E
:204F800000280B9040F0B6800C9804F1240674210D903246212025F031F8002857D10D9906
:204FA00021207422334624F017FD00284FD1608F4FF6FE7181424AD001200D9094F84A001D
:204FC000082806D0042804D011F07EFB0C980D903DE0DDF8349042200DF122018DF82290A0
:204FE00020F01AFB06F12F01432020F015FB06F12C01472020F010FB06F11C014A2020F0AE
:205000000BFB06F11A014B2020F006FB06F12401284620F001FB06F11601532020F0FCFADF
:2050200006F12D01542020F0F7FA06F11801E12020F0F2FA94F83200000938BFDDF8309076
:2050400052200DF122018DF8229020F0E5FA0C9D18E00B9151E00C9AA80000EBC5002946BC
:205060000C23814609EB07000090012020F0E2FB30B917F80900FF2804BF002007F809008E
:205080006D1CADB2BAF80000DAF80470A842E2DC10F034FF8A48001D006800B1804720F076
:2050A000C3FF0D98F0B124F001FFABF81C0028B998F8000000F0F80088F80000C548401CD3
:2050C0000078022818BF012003D1002184F84A1003208BF8010039360BF11400314625F0B9
:2050E0005BF801E009200B900B9F74480021002F4180AED0012771480B9794F83C108146A1
:2051000001208840CBF80C0079E011F0BBFC11F0DBFA04F124022120742124F075FF02A8CD
:20512000FF210C2219F012FC0C9D56460CE0C046E012012034FD0020294601200C2202AB04
:2051400021F080FA6D1CADB23088A842F4DC02A8FF21102219F0FAFB0C9D03202946102203
:2051600002AB21F06FFA6D1C332DF6DB5448006800B1804722F0C4FD002006220C99ADF86D
:20518000100002A819F0E2FB142017F063FD061C1BD0B1480C300768A7B103270225A8B220
:2051A00002A90622801924F075F8AD1D7F1EF6D104A93046022224F06DF84C2014213246FB
:2051C00024F022FF30461FF0E7FC182017F042FD071C10D00C9D1822294619F0B7FB06207E
:2051E000294618223B4621F02DFA6D1C032DF6DB38461FF0D1FC19F0D3FC304881460B98AF
:20520000954D01286AD1734E737804F124072BB3012B0DD0022B13D198F8000000F0F8000C
:2052200040F002000AE0C0460000FFFFE4FA002098F8000000F0F80040F0010088F8000027
:20524000864823F08EF9002808BF00200DD0042103208BF80A1008E03005012098F8001037
:2052600001F0F80188F8001002208BF8010024F008FF0999B36B00F07F000818CBF80C30A5
:205280006430022180B20C90FF2020F07BFE01201AF024FD4FF6FE706087461CE087002012
:2052A000A4F8486020F044FF0A9801280AD002A80021082219F04AFB02A804E04804012074
:2052C0001003012000201FF047FD212074213A4624F09AFE0020022120F054FEE8680B9C89
:2052E00080B9122017F0B6FC0646002EEE606DD04FF6FE70B61F0327411C26F8060F7F1EA6
:205300007180FAD1002C61D106AB4C200021022224F062FB002852D1BDF8180000284ED042
:2053200004284CDA182017F095FC03274FF0020800244FF6FE7A0646EB681FFA88F14C205A
:2053400006221B1924F048FB78BBE868015B8A452BD056B3009620184188002218230620CE
:2053600020F068FA3069EA6800F2E93333611019418805F13402880000EBC100E968135028
:20538000081973694188880000EBC1008018E96843600819418818223346062021F052F968
:2053A00030460021182219F0D1FA7F1E04F1060408F10608C0D116B130461FF0EDFB054B90
:2053C0007120002108224C3324F006FB24F0E2FB30B101E0ACFE00200120A8700027EF7021
:2053E0001F48C9F80C001F48C9F8100022F048FB1E481D490860DBF8100050B10BF11004C4
:20540000076820681FF0C8FB38460028CBF81000F6D109984FF6FF71814217D0012000273B
:205420008BF800000BF1090201468BF80970852024F0E4FD0BF1090428B9852039460122D4
:20544000234624F0C9FA0C9823F09EFC22F03CFE0B980FB0BDE8F08F54FE0020E000012076
:2054600095170100659C020084020120C19F01002DE9F04F0746C44C97F824000026ADF14B
:20548000840D0128ADF83C6006D197F828102078012902D148B9B2E2207830B9387D0228E9
:2054A00000F0AD82032800F0AA826078CB4D01280ED1C94821790078884209D097F8380001
:2054C000E32840F09C8223F05DFF012800F08D824FF4FA60F860E86924F0A3FC40B9E86999
:2054E000F96824F009FE05F1980024F091FE02E0F9680818F86097F8250002288DF83000B1
:2055000003D008B9F86A0D9005E00DA807F11801082224F0C3F80CA80DF13E010FAA1AF0A0
:2055200015FC58B913A807F13401042224F0B6F8BDF83C000DF13E011DF078FF2078012806
:2055400000F0BB80002840F05A82397D31F0010018BF042940F0538268463146242224F08C
:205560009DFE384669460BF0CBF997F81780BDF8000010F0070F06D000F0070002280CBFF1
:2055800014270B2700E00F279DF81900C01987B2384624F081FE5FEA000900F03082044679
:2055A0006946022224F07AF8BDF80000A41C10F0070F18D000F00700022823D102200DF1EA
:2055C000080A8DF82400082251460AA824F066F820460822514624F061F89DF810000834B6
:2055E00004F8010B0EE00DF1040A8DF824600AA80422514624F052F820460422514624F09C
:205600004DF8241D05A92046042224F047F89DF81800241D04F8010B9DF8190004F8010BCB
:205620009DF8190068B10799002900F0E8810246204624F033F89DF819002418079824F0F7
:205640006BFD08A92046022224F028F89DF8220004F8020FB14CE068FFB248B90C2024F078
:205660001BFEE06000B186604770C0F8049015E0E4680834206820B100F1080420680028B4
:20568000FAD10C2024F008FE206038B183680BB1866020684770C0F804902068011C00F0E3
:2056A000AE8181F8008009A808F078FDA869322124F022FD05F174009FE197F83800E32851
:2056C00005D1206918B18047002800F0988197F83800E2280DD0E3280BD0E02809D0E1282C
:2056E00007D097F82800012803D0387D032840F08681BDF83C0000280CBFB0460DF13E08EB
:2057000031462822684624F0C9FD0AA83146032224F0C4FD97F838C0DFF8E8B2BCF1E30F86
:2057200023D097F8250010F0070F16D000F0070002281AD102A807F11801082223F0AEFF15
:2057400097F830009DF8283097F838C08DF8100003F0F80040F0020005E0F86A9DF8283030
:20576000019003F0F8008DF82800BCF1E30F0DD097F829109DF82800C90000F0F70001F05E
:205780000801014306E0C046200401209DF8281041F008018DF8281097F826309DF8292004
:2057A0009DF82800190102F0EF0200F0CF0001F03001022B42F0200241EA00018DF82920D3
:2057C0009DF82A208DF8281002F0F8008DF82A0006DA8BB116E0C04620FB002048190020C0
:2057E00097F8273043B1012B0CD19DF8290000F0FC0040F0040003E09DF8290000F0F8005F
:205800008DF82900387D032807D1FB6B9DF82900099340F008008DF829009DF829009DF829
:20582000282097F84030800100F4006100F4F860084302F030019DF82820014302F0080076
:205840009DF82820084302F007017A6B8DF818C0084305923043ADF8000023B18DF8193048
:2058600007F141000790BBF83A00ADF8200097F91500082805DC10F16D0FB8BF6FF06C0031
:2058800000E00820BB7D6E3040B2002B4FEA60000CBF311C022197F8179040EA81108DF8C3
:2058A0002200BDF8000010F0070F06D000F0070102290CBF14270B2700E00F27800A06D252
:2058C0009DF81800E22808BF8DF8196001E03F1DBFB29DF819003F18BFB2384624F0DCFCBE
:2058E0005FEA000A00F08B8006466946022223F0D5FEBDF80000B61C10F0070F10D000F0E8
:205900000700022812D102A93046082223F0C6FE9DF81000083606F8010B07E070040120E8
:2059200001A93046042223F0B9FE361D05A93046042223F0B3FE9DF81800361D06F8010BEC
:205940009DF8190006F8010B9DF8190060B10799002954D00246304623F0A0FE9DF81900C6
:205960003618079824F0D8FB08A93046022223F095FE9DF8220006F8020FBDF80000800A5D
:2059800004D3701C09A9042223F088FE85F85B70F220BBF84870E378C5F85CA0A9F10C06AE
:2059A00085F85500E188A5F85670002B85F85A6006BF0F204FF6FD71022085F85400B8F1A4
:2059C000000FA5F84C100AD098F80100800906D305F1580008F10B0123F08CFA66E60CA806
:2059E00019F062FEA5F8580060E624F0B3FA286AC82124F081FB05F1BC0024F009FC21B09B
:205A0000BDE8F08FE4FA00202DE9F04FC748C84A0178CD481170CD4D4170CD495C306861A9
:205A2000ADF12C0D086005F0E9FECE49C948CB4EDFF82CB3091D0A91C74982468946E7E025
:205A4000480AC0F09980C8489BF800400078012868D024F0A9FA011C00F08A808A7B96F80E
:205A6000248086F82420778F8A7B08698BF800208A898B7B72870122009200220192012202
:205A8000029200220392049342780592406800232122069001200790F2200AF009FC8BF8E3
:205AA0000040C84986F824800F200870DAF80800778750B3AB490C681434276857B102693F
:205AC0003969914205D007F114042768002FF7D100E097B9DAF80C707FB1786824F01CFB2D
:205AE0000021DAF80C000A9F4160386824F014FB0020CAF80C00DAF8080024F00DFB002096
:205B0000CAF808002068CAF80800D9F8181024F04BFA68B30846322124F0EEFAC34824F040
:205B200077FB25E0B9F85810778F7187C24999F85A008BF8000096F8248086F82400012366
:205B400000930022019202930392049099F85B000590D9F85C0004232122069001200790D9
:205B6000F2200AF0A5FB8BF8004086F824807787296921F480712961D9F80C008A0A3AD3F6
:205B8000071C34D0C468F968A1421FD839468F6800B3D0F80880814210D00246434601E0A9
:205BA0001A469368B3B1AAB19942F9D198689060184624F0B1FAD9F80C000BE0B4480068ED
:205BC00024F0AAFA4046C9F80C0003E0F968091BF960BF68002FD5D14CB1D9F81C1030B122
:205BE0000846214624F088FAAA4824F011FB296921F400712961C80A05D31DF0C9FE296996
:205C000021F480612961080924BF21F008012961E8684FF0FF3124F05BFC0028F8D02878B2
:205C20001BF092FF041C00F0418121782878923900F09C80333961D0491F7BD0491E70D0EF
:205C4000173904D0491E68D0891E61D091E094F84000443080B224F01FFB071C00F089807C
:205C600004F10408381D0C22414623F017FD20693861207D387594F915007875A07DB875AD
:205C8000E07D0A2208F11401F87507F1180023F005FD608C788494F8240087F8250094F813
:205CA000250087F8260094F8260087F8270094F8270087F8280094F8280087F82900E06AC2
:205CC000F86294F8300087F83000606B786394F8380087F83800E06BF86394F8402004F157
:205CE000410107F1410087F8402023F0D7FC3846FFF7BEFB384624F00FFA3AE020790028C1
:205D000037D10A208DF8200008A823F00BFE30E0A188A01D12F07EFE2BE0201D20F08EFB8B
:205D200027E0CD21002203230AE0C046D4DB00200D140120002108AA08238DF82010C12190
:205D40001BF07CFA15E0C046C8E800207CFB0020F8FD00207004012048190020E4FA002037
:205D6000AC0001207804012020040120201D15F0D9F820784FF00108712825DC712851D02D
:205D8000652810DC652868D0801F77D0423800F0838018386FD0401E6AD0401E01287BD970
:205DA000801E5DD070E0663854D0801E4ED0801E032871D9001F45D0401E3FD0401E37D031
:205DC00062E0C0468003012091280FDC912863D07238022860D9C01E20D0401E1AD0401EC6
:205DE0005AD0C01E58D0801E56D04DE092380DD0C01E012850D9303806284DD91B384BD081
:205E0000801E012848D9093846D03DE0E76A002F42D035E0A768002F3ED031E06769002F23
:205E20003AD02DE0E768002F36D029E0BC190020E768002F30D023E094190020E768002FFD
:205E40002AD01DE0E768002F26D019E0E768002F22D015E0E768FFB112E0E768E7B10FE0B2
:205E60002746786908B11EF097FEFF69A7B107E067698FB104E0676977B101E0A7685FB1E5
:205E800038461EF089FE07E04FF0000807E0C04654190020E0190020204622F005FCB8F10C
:205EA000010F03D014B1204622F0FEFB29698808FFF4C6AD08A80021082218F047FD08A84A
:205EC00015F0F2FB23F0D4FF4FF4FA674FF47A71B1FBF0F081B207FB01F024F0F5FAFF2044
:205EE000032120F04FF823F0EDFF024901200860FEE7C0467C0520432DE9FC47D44C0F46B7
:205F00000646F80B80F00C826078B90F80F0AC81B90880F09F81DFF84C83F90A80F002810A
:205F2000390B80F0CC80380907D2F80FC0F02E8227F080471AF09AF928E224F047F9814640
:205F400022F0F2FB002800F0B480082023F0F6FF002840F0AE80802023F0F0FF002840F046
:205F6000A880684615F0DEFF012803D10098002800F09F8094F84102002840F09A80002537
:205F80000126E8B223F092FC48B1837A3BB1867290F9090006FA00F0C0B220F04BF96D1CF4
:205FA000032DEED3032084F8240004F5CE7024F005F9484624F094FAC34800252A460168AB
:205FC000056050F8081CD44940F8085C04F1600022F0FAFA40460068006B8047A168401A59
:205FE000010BE06AC1F1FF3282422CBF08444FF0FF30E06294F8300020B12069E16AB1EBC0
:20600000C02F25D922F0A0FB294600B13146081C1BD0C24840F6090101804580417B06F0FE
:206020000F0221F00F010A434273017B05F00F0321F00F0143EA010202732946416023F0C0
:20604000F9FD418811F4406FFBD084F83060E5621DF0F0FDD14829460560022022F08EF80E
:20606000022020F02BFD112013F038FA207818B96068503024F0C0F8C948007810B90E2063
:2060800013F02CFA94F8310020B184F83150052020F014FDC348A06284F82450B4F9B400A8
:2060A000B4F9B610884214BF0220072017F03EFC02E0484624F014FA27F008073AE720B19C
:2060C000042020F0FBFC0020607065681FF0BAFC38B128462D6A6FF4807100224FF00073FD
:2060E000A847E06858B140460068006B8047E2686168801AC860000BC8600026E660AA49D9
:2061000004F16000002222F05FFA0221D4F8A00084F8241018B104F1E00024F075F827F424
:20612000006707E724F052F8064622F0FDFAD4F898100028894600F08480002900F08180DE
:206140009A49042504F16000002284F8245022F03BFA304624F0C4F904F5CE7024F02EF8CD
:2061600040460068006B8047E0604FF0010884F80180284620F0BAFCD9F810006060D9F8D4
:206180001000816AC90803D3436A29460022984740461BF06FFA606880F81980606813F0A2
:2061A00079FB6568D5F808A040F60A02D01F564600F1010C00E01E46736833B119888A42EE
:2061C00003D0884218BF8C45F5D100217160727B08F00F0322F00F0213437373D9F80C206F
:2061E0001288904224D06046904221D02B8F03B3E96305F13802518095F8440001F00F0345
:2062000020F00F00034385F8443095F8450008F00F0320F00F00034385F845307260707B38
:2062200001F00F0520F00F0045EA0001717300E0E160504623F0FEFC5146404621F09EFF97
:2062400002E0304624F04CF927F480679EE0C04630F500200CF086FBD4F8A00008B927F001
:20626000020793E08C010010514A116841F08001116020B1042020F021FC0020607023F0A9
:20628000A5FF80464B480068016804208847216A81421BD1357ECDB1A568BDB1D4F8A85093
:2062A0006DB1E968098840F60300884204D0E9680988401C884202D106F1140001E006F149
:2062C00010001EF0A9FC06E01410044040F6C411316171612062404624F002F91FF0B2FB6B
:2062E00080B1356A30466FF4807100224FF00073A847D4F89800002808BF47F0020701D0DD
:2063000019F0B4FFF569002130464FF080630A46A84727F0005739E0011C0200F41201209E
:2063200023F054FFD4F8B06066B306F1280106C90A234FF0E0450B40154008BF002B21D1FE
:2063400006F1280191E8000306F1280595E8060006F1280322EA090221EA080183E806003C
:2063600024F0BEF8B16879B1B9F1000F08BFB8F1000F09D03069B6F93010B5684B46424641
:20638000A84701E024F0ACF827F4804727B104F1E000394623F038FFBDE8FC870000046091
:2063A00052C30200B9670100F95D010009870200CC210840E00100102DE9F04F4FF0FF08FB
:2063C0004146ADF14C0D0E910F914FF0000910914E46089609960A96AD4C0B9604F1300BDC
:2063E0000C96E0680D96494611919EE0E068710306AA042323F040FE119903AA304622F09E
:20640000FFFB02AA3046012122F0FAFB3046022101AA22F0F5FB069800F0FF0028709DF837
:206420001900069F6870C7F30140E8709DF80E30AB702878FF2834D0BDF80C70FE2830D063
:206440004FF6FF70B8422AD107A81EF0F5FFE06871034FF088524FF4005323F00DFEBA4857
:206460004FF4005750F8041D3F1FBFB2B1F1FF3F07F1885201D1032FF4D810684FF0010A06
:20648000514600F0FF03FF2B18BF8A46491C000A0529F6DB1060079822F0E4FE5744EF8027
:2064A00001E01020E8809DF80A00BDF8087028719DF806302F81BDF804206B7129786A8142
:2064C000E068FF292AD0FE2922D07E291AD07C2912D078290BD0702904D00D99491CC9B2B2
:2064E0000D9120E00C99491CC9B20C911BE00B99491CC9B20B9116E00A990F96491CC9B2A3
:206500000A9110E009990E96491CC9B209910AE00899B046491CC9B2089104E009F1010750
:2065200010965FFA87F9761CF6B2E578B54200F323810D9F002F38D10898022835DA0C9856
:20654000022832DA099802282FDA4D452BD00C98C0B90898A0B90B980A99084325D021F0F7
:206560001BFB854219DCB9F1000F14D094F83200FE2120F043FAE5780120DDF8408015E07A
:20658000012013E0089860B9B9F1000F07D121F003FB854201DC062008E0032006E00220B1
:2065A000EBE7022002E0119800E004200028A07000F0CC80401E49D0401E00F0AA80401E97
:2065C00006D0401E00F09880801E00F094800EE121F0E2FA05460C2084F83C5015FB00B0C2
:2065E000817E84F83D10C07E84F83E0010F0C0FAE2782D1895FBF2F050432D1AE8B284F820
:206600003200401C90FBF2F15143401A84F831007C201FF0FBF9FF2810D17E201FF0F6F9A0
:20662000FF280BD1FF201FF0F1F9FF2806D178201FF0ECF9FF2808BF94F8310084F833005B
:206640000C2110FB01B0808BE0868FE00F9F08F1010090FBF5F184F832806943FF2FA0EBC5
:206660000100C1B284F8311014D10E98FF2804D10C200E9111FB00B004E00146880000EB3D
:20668000C100584484F83310808BE086AFE0C0465CFC00203A46D0B2910084F8330001EB32
:2066A000C2015944898B1729E18640F2A080C91F01AA89B215F046F89DF80F00C0083FD3DE
:2066C000119F0097BDF81220E18E94F833000323891AC91F01AA89B20CF09AF8002840F0E1
:2066E0008680BDF81010002900F081809DF814001CF0ACFF7BE0FEE7119EB54226DD3046E6
:2067000012F08CFE6178E578761CF6B201436170F3E708F1010084F8328090FBF5F1694349
:20672000401A84F831005FFA88F012F077FE6070FE215FFA88F020F061F9012084F835000E
:20674000119802F041FD52E00020001111986D1E84F831000C2184F8325010FB01B184F8B8
:206760003300898BE1867E2120F048F994F83200FE2120F043F93AE00C2116FB01B506AA94
:206780000423710323F078FC1199304603AA22F037FA304602AA012122F032FA30460221AC
:2067A00001AA22F02DFA0699163501F0FF0201F0FF00FF2A09D0FE2A07D07E2A05D07C2A05
:2067C00003D0782A18BF702A0AD1119F47B9C1F38542032A04D19622B2EB116F3FF41EAEF7
:2067E000304612F01BFE002860703FF4FFAD13B0BDE8F08F2DE9F04FADF1840D1B91CB4906
:206800001C923CC9064610A83CC00EC980E80E0000248DF84240317F8DF84340B28D8DF8D1
:206820004D40D6F828C0ADF844400F46ADF85A20F2898DF854706046ADF84A20027802F093
:206840000303022B8DF8402000F3C38123461D93401C1F9353083CD202F00C0EBEF10C0F83
:206860000CD053093CBF10F8013B8DF84230BEF1080F04BF01238DF84C3001D08DF84C401A
:20688000BEF10C0F0AD0737903F00303012B0CD142F00C0273898DF8402004E04578037829
:2068A000801C03EB0523ADF84430530911D245780378801C03EB0523ADF846300378457891
:2068C000801C03EB0523ADF8483010F8013B8DF8433010F8013B32F07F058DF855301ED0CB
:2068E000037833F003058DF8413040F06E8103F0030EBEF1030F00F0688113F0030F00F139
:2069000001000ED010F8013B02F00305022D8DF8573004BF10F8013B8DF8583001E08DF8A5
:2069200041401490A0EB0C003F1AFFB2B942C0F24C81C91B8DF85470C8B28DF84D00074354
:2069400000F04781D00907D370891EF0C5F8002840F03F819DF8402002F00C002146001F77
:2069600008BF01211E91910933D301211F9180B3B28923F09BFA904202D1F08D000A0ED2EB
:2069800023F094FA904222D0F08D01460B0A38BF101C07D39DF8402002F0030C2EE07089BF
:2069A000ADF85A20804623F081FABDF85A10884205D040461BF072FF002800F00A81864833
:2069C000026810A940469047002840F002819DF84020F08D02F0030C01460B0A0ED2D309D1
:2069E0000CD39DF8413013F0030F07D102F00C030C2B03D0082B1CBF01231D93DFF8E081A0
:206A0000BCF1020F00F0C280BCF1010F00F0908012F0030F40F0DD80704A92F82F20012A6A
:206A200003D1B779002F00F0D4809DF8542002231A92040A9DF84250BDF846B0BDF848A088
:206A40009DF855E09DF857C0DDF850908DF86430B2899DF84370ADF85C2034D21E9F404605
:206A60001A30046897B91D9F1FB1104610A915F0DCFD1F9800901C9F0197B07C1B9A02908A
:206A8000F37C17A910A813F043FAA2E0307C002C8DF8560000F09D8023F008FABDF85C2047
:206AA000904240F0968030791F9F00901C9D01971B9A02951D9B039196F8300010A90490D3
:206AC00017A8A04785E0ADF830008DF820308DF8227034798DF833407189ADF818108DF8F9
:206AE00035E08DF82350ADF826B0ADF828A0CDF82C90307C8DF836C0B27C8DF8320096F886
:206B000030308DF83420354C8DF83730B4F8481096F83270ADF824101A998DF8387006A834
:206B2000ADF82A1006F052FE53E0C04620C102001D9FB58937B1000A04D2284610A915F026
:206B400074FDB5899DF85400B6791030C0B221F0C4FC071C3DD07D81022038703E737C7056
:206B60009DF854203A7207F110057D609DF84000800928BF01247C721499786822F08AFBFA
:206B80004046007839461CF087FD22E09DF8417040462230B189036817F0030F10D110A871
:206BA00007901048ADF8181006A920F01FF980B1062141730068407B21461DF0C3FA08E0FA
:206BC0003BB110A82246984703E08DF84D408DF8544021B0BDE8F08F80020120E4FA002026
:206BE000AE000120CB3402002DE9F04FD24CDFF84C93DFF84C83080CADF1140D019180F021
:206C0000D4810846400838BF0020C0F0D881676823F06AFC054623F02BF94FF47A764FF627
:206C2000FF726843B0FBF6F081B267B13B887888CB1A9BB2984210DDC01A8242C8BF82B247
:206C4000FF68002FF2D14FF6FF70904200F095802078012123F07FFA8FE0B87902287FD0F1
:206C600023F042FC054623F003F997F838204946684301F10A03B0FBF6F03880187890429E
:206C800066DD97F83600FF2808D197F83800401C87F8380097F8370087F8360097F8356073
:206CA00097F839300020012101E0401CC0B283420FDD97F8365001FA00F285F0FF052A4253
:206CC000F3D03618814097F83600F6B2014387F8361097F83400B98F10FB06F2891A89B280
:206CE0008842C7BFFF2087F83600011C97F8360099F82420FF2818BF97F83A0006D1404695
:206D00000078642510FB02F212FB05F0788046B9388D3E7A40F020003885386C87F82E603F
:206D20000BE03A8D4FF6DF70104038853D6C87F82E6097F8342012FB06507862F879CEB239
:206D400087F82D0007F110007E8406F03FFD10E0B87E97F82A10FA8BE9231EF0C7FE05E013
:206D6000387CFF2802D0B86921F09EFC38461FF0E5FD207801211AF015FF019880F0010049
:206D80001DE12878012840F00D8195F8338095F813A06F6995F831006988022220F01AFA1F
:206DA00005F11C0405F1020B06460020002E02907BD1687F400876D3A87FCDF80CA022F020
:206DC00071FFBA4605F11009071C60D01C2015F041FF061C59D000211C2217F0B7FDA87FD4
:206DE000694621F09CFB9DF8010002213075304620F01EFE6888317DB08095F83100FF228F
:206E0000F07102FA01F0707478680078307495F83000B07495F8331011FB00F0303080B205
:206E200021F05BFB0746B76127B930461FF086FD00262AE01A20387000237B701A467A8024
:206E4000E0885946B880B81D21F0FEFCE0783C4BF87303F1200000883882608BB885608962
:206E60007882A0783875207B787599F80000B87599F80100F87599F902003876039A7A763F
:206E8000C7F81CA007F13001B962304600E000200028064600F08680274886F80880007866
:206EA00001211AF07FFE002E7CD0307AA8EB0000B0F1FF3F04BF01200290307CFF285CD01E
:206EC0006078400828BF4FF00008317DF07C4018404503DCF074FF2088407074B069B17C19
:206EE000227D806A08FB0100216922F0D3F9029F317D727C012398FBF1F04843A8EB0000AA
:206F000003FA00F11143C9B27174DFB1401CFF2202FA00F001437174B769B17C207D08FBC0
:206F20000100B884707CFF280CD1307CB1691CF0B3FBFF20307420E0DC040120ACFE002016
:206F40000CFB002023F0D0FA074622F091FF1D4B1D4A4FF47A717843B0FBF1F0308093F8BF
:206F6000241010781F4610FB01F1B87A6423401C10FB01F010FB03F07080F17C327DA8EB45
:206F80000100801AB0F1FF3F04D0707CFF2801D0029F3FB1E175707C2076BBF8000021463C
:206FA00015F043FB284621F07FFB084800781AF0CBFD051C7FF4E5AE019880F4004005B0D2
:206FC000BDE8F08FACFE00200CFB0020DC0401202DE9F04FB74D20F03100ADF1340D0B9087
:206FE00095F83F00002840F06781687804211DF0B3FD002840F060810B99AF7895F83F00F3
:2070000001F03F01012F40EA010085F83F00014600F03B810120A87022F0CCF9012805D126
:20702000562020F081FB08B123F049F8B34C00202071E06808B121F017FFB148476800239E
:20704000A24680467FB10C247868007821F0FAFF061C05D0327C1AB10020824200F31E81DA
:207060003F68002FF0D1184620F09AFE002859D1D8F80470002F55D07868007821F0E2FF3F
:20708000061C4CD0337C002B49D04FF0000844E074690C2018FB00F94C44E079C00838D383
:2070A000786800788DF814002088ADF81600A088ADF81800079A089B069905981DF0CCFE40
:2070C000B0B90DF1240B00210422584617F03EFC74694FF6FF700090CDF804B00A23029398
:2070E00002460392CDF810B034F809104C440AE002681189D388009102F10A00019002935C
:207100000391049021887868A288007817F0AAF8337C08F101005FFA80F84345B8DC3F6836
:20712000002FA9D19AF80200DAF80C20162410FB04F081B2562022F061FF0AF10C060A2881
:207140002BD0092825D021F08FFE562020F0ECFAB0FBF4F0C7B2384620F022FE01281CD039
:20716000336814FB07F082B20021562022F034FC8AF802700DE041680468CAF814101DF078
:207180000BFD9AF81000401E8AF8100020461DF003FDDAF814000028EDD108F0EBFE21F024
:2071A00063FE05F142035520002101221E4622F013FC3078002866D052480078012818BFDD
:2071C000022843D1504804680021204621F08BFF00283BD122F0DEFC002837D120460AA9E2
:2071E00005AA17F035FB04469DF82400FD282DD002282BD0032C4FF0000715DA05A83946CF
:20720000142217F0A3FBFF202146142205AB8DF8240004201FF016FA3C49A00000EBC40067
:207220000F5009184F604F7285F8427055200121324622F0E9FEFF2003211EF0A3FE687855
:2072400085F8207004211AF0ADFC54E095F83F000B99072440F0100001F03F0185F820402C
:20726000014385F83F1000200146FDF733FE10B912F0F4FD3FE0002020F04EF90021204699
:2072800001F0C0F937E095F83F106878002904BF072485F82040F1D00027D1E7716910FBF8
:2072A0000411C979C90824BF5B1CDBB2401CC0B2D3E6C0464CFF002095F82100D8B995F8FB
:2072C000427095F83F1087B10B9880080DD348090BD221F0BBFD0420012101F093F90B9880
:2072E00095F83F1080F002000B900B9800F03F00084385F83F000DB0BDE8F08FF00C0120CE
:2073000020050120ADFE0020B800012064FE00202DE9F0430D460146ADF19C0D04A822F019
:2073200038FF0026304615A920F04EF937460A2800F08681C44C0D2824D1280922D33046E9
:2073400004A91CF073F820460DF11B01022221F001FC78B90DF147012046022221F0FAFB50
:2073600040B90DF14B012046022221F0F3FB002800F066810C2022F08FFF002800F060817D
:20738000044651E1304604A91AF034FA10B9761C052EC7DBAD4E280980F093800DF14701F1
:2073A00003A8022222F07AF9BDF80C009DF88A50ADF80E00680808D30DF18B000DF10E01B5
:2073C000022221F0C7FB012827D09DF88A0080082FD30DF18F040DF10E010222204621F0B4
:2073E000B9FB01280CD09DF88A00042240F001008DF88A000DF18B00214622F04FF95BE0CA
:207400009DF88A00FF21042200F0FD008DF88A000DF18F0022F042FF4EE09DF88A00FF21BE
:20742000042200F0FE008DF88A000DF18B0022F035FF0A36304601686C460DF132054368A9
:2074400021600DF17606018963600A2221813046294621F07FFBC8B90DF1800829460A2204
:20746000404621F077FB70B9684631460A2221F071FB012820D1684641460A2221F06AFB1B
:20748000012816D018E020A80A22B5E70DF1760620AD0A223046294622F000F969460A2217
:2074A000284622F0FBF868460A22314621F052FB10B115A821F003FB384615A91BF0B6FF21
:2074C000BEE09DF81000C00918D29DF81100400851D304A815A919F079F8002800F0B08078
:2074E000C5F341110020022908BF01209DF8551001F0FE0108438DF855003CE03046016845
:2075000043686E460DF176083160018973600A2231816846414621F01DFBB8B90DF13209BC
:2075200040460A22494621F015FBB0B90DF1800868460A22414621F00DFB28B9404649468A
:207540000A2221F007FB7BE020A801E00DF176000DF132010A2222F0A1F8C5F34110002142
:20756000032808BF01219DF8540000F0BF0040EA81108DF854009DF81100800906D30DF1C5
:207580005F000DF11B01022222F088F89DF81100C00913D39DF855000DF11D01012240F00E
:2075A00040008DF855000DF1610022F077F80DF166000DF12201102222F070F89DF81000FB
:2075C000800904D315A9087840F0200008700DF162000DF11E01042222F060F89DF84F0054
:2075E0009DF850608DF8930015A98DF8946038461BF01CFF20460DF15F01022221F0AAFAB6
:2076000068B90DF18B012046022221F0A3FA30B90DF18F012046022221F09CFA80B10C2082
:2076200022F03AFE041C0BD000210C2222F036FE0120A072204622F07FF9204622F06CFD6C
:2076400027B0BDE8F083C0461EFB002052C002002DE9F04FAF4CDFF8C082DFF8C0B2ADF198
:20766000340DA0780591090C6ED20598400824BF059880F0010080F081810598800805D381
:207680000120059FE07087F0020077E10598000938BF0020C0F0728158463230E76A0078DB
:2076A0000026B146000922D222F01EFF054622F0DFFB236B4FF47A7142466843B0FBF1FCC3
:2076C00092F82610928EACEB0300824238D8B0FBF2F39BB29942ACBFDDB20D1CB0FBF2F1F3
:2076E0005143401A80B2ACEB0000206300E00125EFB1C846F878A8420ADD401BC0B2F87026
:2077000040B109F101061FFA86F93E467F680CE087F803807868002E82460CBFC4F82CA05D
:20772000706038461DF038FA5746002FE2D1A078B9F1000F04D10021216308211AF0F0FDD2
:20774000059880F0080019E11AF0FEF9071C00F01281B87FC0B9788CE56A132815D1B7F8A0
:207760000290281C11D000260188894508D14568002E0CBFE56275601DF00EFA284601E0D6
:20778000064640680028EFD1E56AB87A97F831102E46022855D1788866B1DFF8E8C13288A7
:2077A000904204D1B2789CF80030914247D07668002EF4D181468A464646002D08BF002042
:2077C00004D0012015B16B68002B34D1F18E814237DD082015F03EFA96F82610002830D044
:2077E000A0F8009080F802A0C17000234360E36A83B9E0629BF83200000911D222F074FE50
:20780000054622F035FB4FF47A716843B0FBF1F0206300E06860584690F83200000910D307
:20782000A07808211DF098F958B9A078B28E082122F08EFC05E0401C1D4680B2C2E7F37059
:2078400096E0514805683878012806D0022840F08F80384618F032FC8AE007F11004B81C96
:20786000BE8908943B7E0690FA7C07967969099397F819B00A923C7F0B9107F11C0604F0EC
:207880000C000C280DD0B87F4FF0FE09FF2804D022F008FA041C10D16AE0002D68D06C68BB
:2078A0000FE0B088FE211EF03DF98146B9F1FE0F5ED022F0F7F9041C5AD0207821F0B8FAEB
:2078C00005464FF6FF7A0BE0207821F0B1FA054606E0B078FF284BD12D68002D48D06C6816
:2078E000002C45D0AB68AAF1010823B9A3680BB1B3F8028007E021780220984718B1B0F8CE
:2079000000801DF049F93389227898450AD03AB943B11CE0AC000120ACFE0020E4FA002013
:207920009A4514D196F80280B27008980090099B01930A9902910B9A0392CDF810B0079B52
:20794000069A3046214613F0F7F986F80280307800F00C000C28BCD1B08849461EF0E2F8A3
:207960008146B9F1FE0F03D022F09CF9041CABD1384620F099FE059880F400400DB0BDE89B
:20798000F08FC046D2FE0020240501202DE9F04F0E46074630687C68BD68ADF1140D0028AA
:2079A0003AD022F013FCD4F8E81081460120019008294FF0000088BF0198B168084202D1D9
:2079C0007168084205D0019880F00100C0B201281DD1D4F8C000B8B9C4F8C060C4F8C46063
:2079E0000020C4F8D0000146C4F8D41094F8FC30C4F8D810002BC4F8DC100CBF019805203C
:207A0000D4F8C410087410E094F8F80030B903203074484622F064FD002050E1D4F8C40044
:207A20004661C4F8C46006233374D4F8C4000021416194F8FC00012808D1022194F8FB0068
:207A400084F8FC104FF4E0211FF0F0FB706810F0704F06D128B104201FF048F806201FF071
:207A600045F802201FF042F894F8F800DFF85482002840F0B480E86B3168884240F2AF808A
:207A800094F8FC00002840F0AA8094F8F90028B1D4F8EC00B0F1FF3F40F0A180484622F0F6
:207AA0001FFDB768AA463FB1D4F8E800B94609282CBF0220019802E004F1F409002077684E
:207AC000039037B1D4F8E80009282CBF0220019802E004F1F60700200290DAF80010D6F86A
:207AE00000B048685FEA0B0540F0020048604ED04046A0F11008D4F8E800ABF1010B092819
:207B000020D3019803460DE0D8F800108A68398890470346002003B10198031C02D00298F8
:207B20006D1E3F18DAF800000DB1012BECD0D8F80010C9680A4669469047BDF80000A9F8AE
:207B400000001FE0019803460DE0D8F800108A68397890470346002003B10198031C02D056
:207B600002986D1E3F18DAF800000DB1012BECD0D8F80010C9680A46694690479DF8000095
:207B800089F800000398BBF1000F8144B3D17768DAF80010D4F8F030CA680020134218BF9A
:207BA0000198102B18BF80F001000028F4D117F0704F06D12FB106201EF080FF04201EF05A
:207BC0007DFF02201EF07AFFD4F8C010002008740746C4F8C4703E46C4F8C0606EE0D4F891
:207BE000D800002843D1D4F8DC00002842D1287922F0EEFA4646D4F8CC00326829694068FB
:207C00005268006891FAA1F1B1FA81F1134602229847D4F8CC0032686969406852680068DE
:207C200091FAA1F1B1FA81F1134602229847287922F0C8FA287922F0CDFA204629460CF0EE
:207C400013FB0021D4F8C000C4F8E0100068B0F5806F03D9204629460CF006FB94F8FE0089
:207C600060B92968486840F00200486006E0D4F8DC0018B9204629460CF0F6FA296848696E
:207C800040F001004861484622F02AFC94F8F800A0B9D4F8EC1004F16C05284621F037FF84
:207CA00060B1D4F8C00003210174384609F0E4F92846002121F02BFF00200190019805B071
:207CC000BDE8F08FD40100102DE9F04FC54CDFF80893207888465FEA1841ADF1140D39D2F1
:207CE000BE4D281D00685FEA58011AD25FEA980028BF88F0020080F06B8164885FEA181043
:207D00000DD36846FF21082216F020FE20466946002201231DF0CEFE88F0080058E100205A
:207D200056E10830002113F0E1FA4C46206818B120F0BAFC002020606868806A1CF02CFF9B
:207D4000686800248462686820F0AEFC88F001006C603DE119F0F8FE061C00F03781012072
:207D600037780390F7B996F802A00025AB4617E0A80000EB090759F80000807C82450DD13F
:207D800005208DF803A061688DF8020009B168468847386820F088FCC7F800B06D1CEDB244
:207DA000002DE5D03078012850D17068017801F00202022A4ADAC1F38302032A46D1CF11FC
:207DC00009D0407800F0070101293FD002293DDC30F07F003AD13089273080B220F07DFB29
:207DE0002578071C32D00020787002233B70F06B06F132010A22786007F1120021F04AFA01
:207E000007F1080006F128010A2221F043FAB6F84400F883B6F84200B88396F8460087F8DD
:207E2000210096F9480087F8200096F8490087F822007168328907F1240021F02BFA307AA3
:207E4000394687F8230028461BF026FC3078022803D1304602F050FC307808287ED1F0787D
:207E600021F01EF8071C79D0B078002873D02578401E11D0401E3AD0401E4ED106F11C0107
:207E8000384606F035FE01282AD038461DF004F8002087F8290061E006F11C01384606F000
:207EA00027FE01281CD097F84100F02853DA97F8260000280CBF0398002097F84050387544
:207EC00097F8410007F1420187F83800681EC2B207F1410087F8402021F0DCF9257818E053
:207EE00003203875207839461BF0D6FB36E0042097F8413097F84020387507F1420187F82F
:207F00003830501EC2B207F1410087F8402021F0C1F9284639461BF0BFFB97F82900E8B131
:207F200097F825008DF8000097F82500002804BFF86A019005D001A807F11801082221F0AC
:207F4000A9F926481321016097F830100023684603F0F4F902E038461CF09EFF307805281E
:207F600004D1304608F012FF0390307804281BD1E068A8B196F84000443014F06BFEE568BD
:207F8000071C0DD096F840203146443221F082F900201349B860384621F0CCF83046A8472E
:207FA00030461CF079FF30786168062803D111B1304688473078072803D1216909B13046E8
:207FC0008847039810B1304620F06EFB88F4004005B0BDE8F08FC0465819002048050120ED
:207FE000541900209C0301202DE9F04FBF4CDFF80083207889465FEA1941ADF11C0D3FD298
:208000005FEA590111D32079211D88F83C00E1201DF002FB20F0C6FE0020A8F894000120F2
:208020001AF0DEFA89F001005CE1E7885FEA990116D25FEA191038BF0020C0F0538194F8D4
:20804000310050B1E06A94F8301021F032F820B994F83100401E84F8310089F0080041E159
:20806000002F04BF0020A07007D07F1EB9B24EF66022E180022122F06EF889F0020031E1B0
:2080800019F062FD071C00F02B81C346387894F83120A178313800F00B81401E00F0BC809B
:2080A000A13840F01481FE89383E0FD047F6DD70361A40F00C81B8690678002E40F007812A
:2080C0004078C009C0F0038178885CE089490EC904A880E80E00D7F818A00421504620F092
:2080E000B2FC3D4606460AF1040010F8011B049606298DF8141010DBFE2918BFFF290FD17D
:208100000278FF298DF816200AD1401C4278007800EB0220ADF8180002E000788DF81500DB
:2081200006295ADBFE2931D0FF2912D0287B002840F0CD8068882084002600963346019304
:208140003246029231460391687C802114F046F9BDE09DF816509BF89600A84205DB002D88
:2081600040F0B580FF2840F0B28028461DF0E0FF3EB1DBF84C00864203D0CBF84C6020F08F
:2081800011FEBDF8180020F01BFEA0E09DF8165098F89600A84205DB002D40F09880FF28D3
:2081A00040F0958028461DF0C3FF002001218140314202D1401C1B28F8DB98F83C108842DC
:2081C00000F08580207198F82B00642110FB01F20121207821F0BFFF79E02B7B002B76D1E1
:2081E0009DF815A0BAF1000F71D0BAF1060F6EDA304620F05EFF002869D1AAF10106687C67
:208200008DF815606B88607004A923840EC904F12C0585E80E005AE0FF2A12D000201AF066
:20822000DFF90246002000906078B8F894103B4615F0D5FE94F83100002848D0082132226F
:20824000C7E798F83C007A6801213B46814011420EBF00213844017A5D680020012282405C
:20826000154203D0C218127A8A4204DB401C1B28F4DB002018D0B8F892002084102600969B
:2082800021896289002015F0AAFE0120E070A07840B93C20E080207802214EF6602221F0AC
:2082A0005AFFA078401CA070002084F831000EE004290CDA10480178104820F0FAFE30B9F9
:2082C00078882081FF2684F83160B8886081384620F0EAF9207819F037FC071C7FF4D6AE4B
:2082E00089F4004007B0BDE8F08FC046E8000120E4FA002088C2020036FB002000F8FF073E
:208300002DE9F04FADF1440D0B908069007800210DF12A020F909C2011F020F8B54D681CD8
:20832000007830F0010009D1002004211FF0E4FB5FFA80FA9DF82A00504402E001204FF02F
:20834000000A8DF82A000F989DF82A10884280F2DE809DF82A000F99401AC0B20D9002285A
:20836000C4BF02200D901A2110FB01F000B214F071FC0E90002800F0CD800F980D9F0E9C61
:208380000C90002F08BF002074D04FF00008B946012645460C9882450ADC0F9940468A45A1
:2083A00004DAA1EB0A01C9B20C9163E00C9561E0411CC9B20C911FF0B3FB071C54D08E48BC
:2083C0000146B0F848005D312080A01C21F0E4FE388860820223E375FF222276B87A6076A9
:2083E0008DF81C503888ADF81E0007A816F0E8FAAB46012808BFB34604F10A00BBF1000FDE
:2084000006D104F10A00FF21082216F09FFA02E008A921F0C1FE3B797BB93F88002F04BF99
:208420002575281C04D07448267590F85C00401E207602206075A57515E06F4890F85C00BA
:20844000401C20763879032804DB26753879032805D106E0022020753879012801D06675FF
:2084600000E06575A6751A34B9F1010908F1010890D140460D9981424CDD0D9DDFF878B100
:2084800004F1020804F10A0702264FF0000A4FF001091A3C2D1A0C9987206A4610F05EFF27
:2084A0005749BDF80A0024F81A0F404621F074FE0DF10201384621F06FFEBDF800004D4BC5
:2084C0006082587830F0010003D16675A675FF2006E084F8159084F816A09BF85C00401E5A
:2084E0002076E675638A9DF81200002B60760CBF84F814A084F814900C9808F11A081A37CB
:208500006D1E00F10100C0B20C90C4D102E000200E900D900B98417C0D9F0E9D8DF82B1087
:20852000801C16210B9017FB01F0001DC0B28346401C14F08FFB5FEA000854D008F1010415
:208540000020A2468AF800009DF82A000F9F88F802000D9E88F8037088F8046096B30D9F2B
:208560002E46241D06F102090A362046494621F013FE08343146204621F00EFE0446A87C49
:2085800004F8010B688A001204F8010B287D2070697D40EA8100C0B22070A97D40EA01109E
:2085A00004F8010BE87D04F8010B287E04F8010B687E09F11A091A367F1E05F11A0504F897
:2085C000010BD2D10D4D0B990DF12B0048F231025B462C1DC4F800A018F0A0FA40461CF0DE
:2085E000DBFA09346C600E9808B11CF0D5FA11B0BDE8F08FACFE0020E4FA002098FD002001
:2086000041FB0020FEB5BC4CBC4A0D46014694F83E705078491E00F02C81491E00F00981BC
:20862000491E00F0C980B64B491E00F0A780491E6AD0491E1FD0491E40F03A810026012D7E
:208640008DF8016004D0022084F83E0007460DE016F06AFA0D2084F83E00607884F8206025
:208660000421C82221F077FD94F83E7094F83F0000F0EF0045E003208DF801000FB90120CB
:2086800020722078002840F035816278606921F055F8002840F02E8110464FF480411CF034
:2086A0005BFA002840F026810025A561E5611EF049FF60784FF4804119F032FE267A94F85E
:2086C0003E702EB10B2F03D1284684F83E002F46257294F820106078062906D094F8230083
:2086E000062808BF84F8235007E084F820500421322221F030FD94F83E7094F83F0000F017
:20870000F70084F83F00D3E00221012D8DF8011016D0082130F0010084F83E1021D194F895
:208720004200F0B9002552200DF105018DF805501CF072FF21F0F4F918F08CFB28460EE073
:208740000025184684F83E50008850863232832021F05AFC032128461DF014FC072020F0DA
:208760001DFE002084F8200060780421322221F0F2FC94F83F0000F0FB0077E001208DF81F
:20878000010065B100201F8884F83E00022157863232832021F038FC072020F0FFFD0020A2
:2087A00084F8200060780421322221F0D4FC94F83F0000F0FD0059E0012818BF022877D188
:2087C00060780421322221F0C6FC94F83F10606A012D23D00222002084F83E2005468DF8C1
:2087E000040021F0020184F82050012284F83F1052208DF8012001A91CF00EFF21F090F912
:2088000018F028FB284620F0C9FD606A00284DD01DF0ACFD606A0028FAD147E001210028F6
:2088200084F8201066D01DF0A1FD606A0028FAD1FEBD002021F0C6F8042601208DF8016013
:20884000D0733DB1002084F83E0084F83F00072020F0A4FD002084F820006078314632221B
:2088600021F079FC94F83F0000F0FE0084F83F001CE0012818BF02281AD1012D23D00120AB
:2088800007278DF801004FF48051607884F83E7019F046FD00201EF03FFE002084F83F007C
:2088A0006078022141F2883221F055FC94F83E70A66AFEB18DF800700A20002103226B465F
:2088C0001BF018FFFEBD002003211DF05BFB04213222607884F8201021F03DFC0820002184
:2088E00012F0CEFA002084F8210060784FF4805119F016FDFEBDC0464CFF0020ACFE0020F3
:208900002CFB0020F0B50E467068ADF1140D002800F06381002771687770B24C087858B116
:20892000487800280CBF381C01202246012110730C32632021F068FB71680D7965B1487997
:20894000224600280CBF381C0120012150730D326D2021F059FB71688D79ADB90D7ACDB1E7
:20896000088A10F0070F02D0CA68632A12D9C96820F00AF83846012112F082FA9A4A352039
:20898000282121F041FB04E0C9794FF4005012F077FA71688D7C45B1888A22462E32022140
:2089A0001080442021F030FB71688D7D45B1088B2246303202211080462021F025FB71682E
:2089C0008D7E45B1888B2246323202211080832021F01AFB71688D7F45B1C87F2246921C03
:2089E00001211070292021F00FFB716891F820504DB191F821002246D21C012110702B20B4
:208A000021F002FB716891F822504DB191F8230022460A3201211070432021F0F5FA716848
:208A200091F824504DB191F825002246521D012110702E2021F0E8FA716891F826504DB1FD
:208A400091F827002246921D012110702F2021F0DBFA716891F828504DB191F82900224686
:208A6000D21D01211070302021F0CEFA716891F82A504DB191F82B002246121D0121107075
:208A80002C2021F0C1FA716891F82C50A5B191F82D20102A8DF8002003DD10208DF8000040
:208AA0000246096B0DF1010020F0F4FB812011216A4621F0A9FA716891F8345055B191F850
:208AC00035001028C8BF10208A6B0146622021F09BFA716891F83C5045B1086C22463832E4
:208AE00004211060842021F08FFA716891F844504DB191F8450022460B32012110704B202F
:208B000021F082FA716891F8465065B104F13C0547310822284620F0BDFB472008212A46AC
:208B200021F072FA716891F84F5035B101F150020120082121F068FA716891F858504DB1C8
:208B400091F859008DF811000DF1110152201CF063FD716891F85E5045B191F85F00234A54
:208B600001211070332021F04FFA716891F85C5035B391F85D0004F1080501212A4628709E
:208B8000322021F041FA3220394601222B4620F023FF04F1090333203946012220F01CFF7F
:208BA0001348217A0078012904D04FF4006119F0B7FB04E04FF40061642221F0CCFA71682C
:208BC00091F860705FB191F861000A4977680A4D087097F86100287001E00220707005B021
:208BE0000120F0BDACFE002034FC0020B5FE0020E4FA0020291A002070FB0020F0B50E46D5
:208C00007068ADF1140D002800F06581B068002800F061810025B24C7268757004F10C00CA
:208C2000177803783FB1B06801210170284603B10846B16848707068637B877847B1B06889
:208C400001210171284603B10846B16848717068C7785FB1284620F061FCB2680121800B75
:208C6000917138BF291CB068C171706807794FB1B06801210172B0680C3020F04FFCB1689F
:208C8000088270684779E18D37B1B068012280F82C20B068C18570688779218E37B1B06878
:208CA000012280F83020B06841867068C779618E37B1B068012280F83420B068C1867068BD
:208CC000077AA1783FB1B068012280F83820B06880F839107068477AE1783FB1B068012209
:208CE00080F83A20B06880F83B107068877AA17A3FB1B068012280F83C20B06880F83D10F7
:208D00007068C77A61793FB1B068012280F83E20B06880F83F107068077BA1793FB1B06804
:208D2000012280F84020B06880F841107068477BE1793FB1B068012280F84220B06880F8CE
:208D400043107068877B21793FB1B068012280F84420B06880F845107068C77B37B3B06844
:208D6000012111226B4680F846102946812020F033FE9DF80000B16881F84700B26892F8BC
:208D8000471089B113F066FFB1688864B268906C002808BF82F8475006D09DF800200DF136
:208DA000010120F077FA00E095647068007C80B1102013F04FFFB1680865B168086D40B14C
:208DC000012081F84C000B6D10226220294620F003FE7068A16B477C37B1B068012280F8BF
:208DE0005420B06881657068877CE17A3FB1B068012280F85C20B06880F85D107068C77C94
:208E000057B1B068012180F85E103649B06808225F3020F03FFA7068077D67B1B0680121E3
:208E200080F8671020F006FA0146B0680822683020F030FA7068477D87B152200DF1110182
:208E40001EF04AFF9DF81170B068012180F8701007B92946B06880F871107068877D3FB167
:208E6000B068012180F87210B06880F873507068C77D237A57B1B06801212A4680F8741004
:208E800003B10A46B06880F875207068077E617A3FB1B068012280F87620B06880F8771021
:208EA0007068477E5FB1B06801210F4F80F87810387800B10D46B06880F879507068807E8A
:208EC00058B1B068012180F87A101BF0CFF8B16881F87B0001E00220707005B00120F0BD08
:208EE000ACFE002041FB0020291A0020F8B50D4606466868002800F06281002730466F7056
:208F00001FF0DCFF041C13D11C2013F0A3FE041C00F0578139461C2215F018FD26712046C7
:208F20001CF070FE20B920461BF036FED12047E1686807785FB1407820B9E1884FF6FE7014
:208F4000084002E0E08840F00100E080686887785FB1C07820B9E1884FF6FD70084002E0B9
:208F6000E08840F00200E080686807795FB1407920B9E1884FF6FB70084002E0E08840F02A
:208F80000400E080686887795FB1C07920B9E1884FF6F770084002E0E08840F00800E0803C
:208FA0006868077A5FB1407A20B9E1884FF6EF70084002E0E08840F01000E0806868877AAD
:208FC0005FB1C07A20B9E1884FF6DF70084002E0E08840F02000E0806868077B5FB1407B12
:208FE00020B9E1884FF6BF70084002E0E08840F04000E0806868877B57B1C07B002807BF56
:20900000A06820F00100A06840F00100A0606868077C57B1407C002807BFA06820F00200DF
:20902000A06840F00200A0606868877C57B1C07C002807BFA06820F00400A06840F0040099
:20904000A0606868877D57B1C07D002807BFA06820F01000A06840F01000A0606868077E44
:2090600057B1407E002807BFA06820F02000A06840F02000A0606868877E57B1C07E002869
:2090800007BFA06820F04000A06840F04000A060686890F822705FB190F82300002807BFA7
:2090A000A06820F48060A06840F48060A060686890F826705FB190F82700002807BFA068F5
:2090C00020F40050A06840F40050A060686890F828705FB190F82900002807BFA06820F4E5
:2090E0008040A06840F48040A060686890F82A705FB190F82B00002807BFA06820F40040B5
:20910000A06840F40040A060686890F834705FB190F83500002807BFA06820F48010A06868
:2091200040F48010A060686890F838705FB190F83900002807BFA06820F48000A06840F4D4
:209140008000A060686890F83C705FB190F83D00002807BFA06820F08070A06840F0807098
:20916000A060686890F83E705FB190F83F00002807BFA06820F00070A06840F00070A060F4
:20918000686890F840705FB190F84100002807BFA06820F00060A06840F00060A060686820
:2091A00090F842706FB190F84300002807BFA06820F08050A06840F08050A06001E00220A9
:2091C00068700120F8BD70472DE9F04FB04E4FF0000A8146ADF1140D57467069CDF808A025
:2091E000CDF80CA010B1804700B90B27F078002F40F09B8096F8314096F832700146B9F189
:20920000000FA1F101011FFA81F818BF012155464FF0F80B86F83F1022E0AF421ED0F0683D
:2092200069036A46042320F027FF009911F4403F1CBF0AF101005FFA80FA01F0FF017C2958
:2092400018BF782909D1284606215A461FF0E6FC0C2015FB006080F848B0F0786D1CEDB2FA
:20926000A842DADC401E504503D196F8350000285BD0B8F1000F06F1300500F0CF800398B3
:209280004FF4005B019096F83F30F06813B9012186F83F106A466103042320F0EDFEB9F1AF
:2092A000000F05D00099F07811F4403F40F09B80009800F0FF00702803D0204670211DF004
:2092C0009DFBF06879036A46042320F0D5FE009800F0FF00FE2803D03846FE211DF08EFBB5
:2092E00038460621FE221FF099FCB800FE2300EBC700FF2186F83C70A200A6F840B04019A7
:2093000086F83D4000F1180A8AF80030019B86F83E1002EBC4004019A6F84430808BA6F860
:20932000420001F065FC102801D10020ADE0B9F1000F0CBF10214946B9F1000F07D0B6F860
:209340004000C0F50050814207DC01200390B6F84000C0F50050814201DD782100E07C21C4
:2093600038461DF04BFB0DF003FC96F83F300446A8EB04000621FC221FFA80F8181B86F8BB
:209380003F0038461FF04AFCFC208AF80000029A96F83210F078091996F83E400C27891847
:2093A00091FBF0F24243891AC9B286F83210491C91FBF0F24243891A86F8311014FB0751BB
:2093C000898B102905D1611C91FBF0F24243891ACCB20198B9F1000F96F83270029019D0DC
:2093E0000398B8B11AE096F83F30641C94FBF0F1A8F101024143A6F840B01FFA82F8581ECB
:20940000641A029986F83F00E4B286F83D40481C80B20290B8F1000F7FF435AF7C201CF006
:20942000F5FA00240746FF2F1CD17E201CF0EEFA0746FF2F16D196F831700C2017FB005000
:20944000807DFF280AD0F27896F832008018401E90FBF2F15143401AC7B203E038467E2119
:209460001DF0CCFA0C2086F8337017FB0050808BF08696F83200FE211DF0C0FAB6F8400055
:2094800086F83540C0F5005000B205B0BDE8F08F5CFC00202DE9FE4FA84E00900578775D97
:2094A000002FADF8047000F04681DFF894820D2D4FF0000B4ED0052D15D0072D08D00C2DC2
:2094C0001AD14068C08A400A28BF4FF0010B13E08478002C08BF07F11B000BD0807D242121
:2094E00010FB017006E08178012900F02481007CC0192430ADF80400BDF804001EF0EDFF4D
:20950000041C1FD10C2D40F0168100984068002800F0118120F05AFE444607462068009BEF
:20952000D0F85413181D8847BDF804001EF0D5FF041C04D1384620F0D3FFBDE8FE8F384658
:2095400020F0CEFF072D21D0725D009920461FF0A1FE19E044462068D0F8282401A9532051
:209560009047BDF804104FF6FE70884200F0DE80BDF80410401C884200F0D880009F3889E9
:20958000002800F0D3803C46052D46D0072D55D1009908782070487860708878A070C878B3
:2095A000E0700A7ACF798E79487900EB026000EB074000EB06206060A778E7B18F7D27721B
:2095C00067B1896951B1BA0004F1100002EB47121FF060FE04F11000E06002E00020E06086
:2095E00020720098806948B31BF0D6FA009800218161817522E01B222272896904F1100027
:209600001FF048FE04F11000009FE060B8691BF0C3FA00980021816110E0616804F11806C1
:20962000242230461FF036FE66606169227C06F124001FF02FFE606824306061DFF808A149
:20964000DFF808910D2D0DD00C2D2CD1009840781A2828D0676837B3F88A400823D309F051
:209660007CFB20E000994B681878C0F3830200F0020002284DDA33480078904249D15F7866
:2096800037F03F0745D191F83000022841D109F064FB0098418E4FF6FF728A4203D1406895
:2096A0008079022817DA50460078BBF1010F19BF4846007800212170214619F0EDFF0C2DA7
:2096C00039D100984168002935D044462168D1F85413001D2EE0201C1FD054F80C7CAFB93C
:2096E00010F8021CFF2911D14D46297800F8021C17480A2221461BF0AAFD01280DD12878A5
:209700004FF4005118F04EFABDE8FE8F1EF0CCFF03E050460078032A02D04446206806E072
:2097200001220A7019F0B8FFBDE8FE8F2068D0F8541368468847BDE8FE8FC04638C2020032
:20974000140100201AFB00209C030120E4FA00203C0501202DE9F04F81460D462C20ADF126
:20976000240D13F077FA071C00F0498120F09EFB698B884214BF012002203870697B2869CD
:209780000026401A7860687B87F82660B8707C68B87887F827602418207800F00700787094
:2097A0002078C0F3C100387420780421C0F3401A601C1FF048F94FF00508B861BAF1010F3B
:2097C00087F81C8006D007F108003146082215F0BDF808E0397F07F10800091920F0DCFC93
:2097E000387F08303877387C012805D1387F205CB875387F401C38772878DFF80CA200F0E1
:209800000300012803D0504630300078804687F8018078781FF086FD7877397F28692C7DB2
:2098200040182861397F7B7F601AC01AC0B22875F8704FF6FF74BC82B869B0F1FF3F32D0D2
:20984000387C01281CD038B9062078823946484616F06AFC40B30CE0387C022802D00328FB
:2098600007D01EE0062078823946484616F05CFCD0B104207882394648460BF005F913E0F0
:209880009AF82F507E82B32075B99AF8651001290AD1B87D19F03AFCB882844218BF301C13
:2098A00002D1A12000E0A32004463878022806D11FF0C0FC014607F1080020F06DFC002CBF
:2098C00040F09980514D6878B046012818BF02281CD197F82600012803D097F82700012824
:2098E00014D1B978F8784018397F4018001D13F0B1F95FEA000809D0B878FA783C7F796848
:20990000121840461219121D1FF0C4FC38460BF04BFE04466878012818BF022865D1002CF6
:2099200063D0B8F1000F66D040F203154FF0680A4FF0010900E05C4697F82600012803D08F
:2099400097F82700012850D1B978FA783B7F786852184146D218121D1FF09CFC97F8260064
:20996000A34630B997F8270040B1BD8287F8276003E0A7F814A087F826607E8238460BF075
:2099800013FE041CD8D168463146142214F0DEFF7B8A8DF81190D3B9B88A682803D085428E
:2099A00015D1FF2011E07868C17B0529C3D12A30FF211FF098FB0028BDD005A8082214F027
:2099C000C5FF05A820F0EEF8FC208DF8100002A807A9324614F03CFF01469DF81C0020B195
:2099E000042014226B461CF02DFEB8F1000F02D040461BF0D1F838461BF0CEF800E01024DE
:209A0000204609B0BDE8F08FE4FA0020ACFE00202DE9F04305468078ADF14C0D1FF0B0FAFF
:209A2000071C00F03B816878F873DFF888826878F12809D0CD2807D01A2805D0E92803D092
:209A4000E12818BF1D280CD17889DFF86C92000B80F003813846002104F05EFF002840F0E7
:209A6000BF8010976B788DF84430A87B8DF845008F4C387C002840F085808B4802685AB103
:209A8000384619469047012804D179894FF6FE70084078819DF84430787B02282BD17989FA
:209AA000890826D3E92B24D0CD2B22D0F02B20D0788A7E4B000A08D3B87E30B1B87338688D
:209AC00000881BF009F8194603E01946887A401CB873B87B401EC0B2B876B87304267E7351
:209AE000C88D38812078202118F05CF89DF84430787B022801D0062839D1608F398B884277
:209B000015D0607898B138680088ADF80A00388BADF80800387B8DF80E308DF80C000126CA
:209B20008DF80D6002A81FF005FD9DF84430788940081CD37E6946B1707810F0030F04D18A
:209B4000B078317BB2881BF0D1FF79894FF6FE7008407881386800881AF0BEFF002600B160
:209B600001269DF84430301C01D10BB10FE073B940463E68036830881AF0AEFF28B923B105
:209B8000984702E010A809F01BFC9DF84430E92B18BF002B07D1396801200090EA7B0888FE
:209BA00049890BF00FFE94F8320080086ED3787B022802D17889C00806D26878E92865D18C
:209BC00038461AF01FFE61E03B6818881AF084FF20B94FF6FF70188005205BE0032059E0EE
:209BE00048460078800826D33968086A18B3C97F02AA0BF061FD6B78E92B07D13968012022
:209C00000090EA7B088849890BF0DCFDBDF81200396808809DF80D0000280CBF0022402210
:209C2000BDF81200BDF814100EF026FC18B1788940F0200078816E783889E13E18BFB6F10D
:209C4000100608D1798911F0300F04D020F019FA00F00700801C388101E0052078736878BF
:209C6000E92813D04046006800B18047134C206A60B148460078800808D339680888498924
:209C80001CF0C6FC10B1226A69789047787B022801D106207873A87814F0A4FB07F0DEFE5B
:209CA00013B0BDE8F083C046C4000120ACFE0020E4FA002008FC002016FB0020ECFB0020BA
:209CC0002DE9F04F044665692888ADF1440D0027ADF8380016E010FB04F2BB189B780B701C
:209CE000BB185B88BA181B124B701279401CC0B28A70C91C11E1BDF838007F1CFFB2401C35
:209D0000ADF83800A878B8420CDD21680BA800906268087D89880EABC2F3C00217F0C0FA46
:209D20000028E8D1E07A0C2800F09680152840F01081022000EB870080B220F0ADFAB84635
:209D4000061C00F00681002F4FF0010939D028880025ADF83A00216808A800906268087D1D
:209D600089880DF13A03C2F3C00217F099FAC8B1BDF82410A800321851809DF8262033183B
:209D80001A719DF82710BDF83A207F1E05F1010506EB000301F00700587102F10100ADF876
:209DA0003A00D8D1216808A800906268087D89880DF13A03C2F3C00217F072FA08B14FF07A
:209DC000000986F8009086F80180216804236768087DA57AB1F804A0109001F1060BF8085A
:209DE00080F0010000F0010918FB03F0401C044620F052FA071C1BD00146307801F8010BEE
:209E000000207278824215DC00200090CDF804900121029103900495524605941623069792
:209E200010980791594606F043FA384620F074F937468BE08200B3189B780B70B3185B88A4
:209E40001B124B70B3181B79B2188B705279401CC0B2CA70091DD4E73E4606EB4600801CEB
:209E600080B220F019FA071C73D0002E4FF0010933D02888B0460025ADF83C00216808A8C8
:209E800000906268087D89880FABC2F3C00217F007FAA0B1BDF8241005EB45003A183B1885
:209EA000B8F10108518005F101059DF82620BDF83C101A7101F10100ADF83C00DED12168B0
:209EC00008A800906268087D89880FABC2F3C00217F0E6F908B14FF0000987F800907E70CD
:209EE000216894F80A806568087D0324B1F804A0109001F1060BE80880F0010016FB04F5EF
:209F000000F001096D1C284620F0C6F9061C1DD00146387801F8010B00207A7882423FF76A
:209F2000DAAE00200090CDF80490012102910390CDF81080524605950D23069610980791B5
:209F4000594606F0B5F9304620F0E6F8384620F0E3F811B00120BDE8F08F70472DE9F04FDF
:209F6000DFF84C9204460D460020ADF1440D01461F460D9016460E9183460F91D9F808A05A
:209F8000CDF840B014F0AEF8262803D014F0AAF8252825D1308843F6070181420ED040F688
:209FA0000201814206D0B0F5C15F19D1F07B022816DD43E0F07B022812DD3FE096F8240056
:209FC00002280DDD307C0F2838D13169C1F31421B1F5803F04D00F2830D1B1F5A02F2DD11A
:209FE000002D2BD056B328784FF0010808FA00F01AEA000F22D03046594620F0F5F865607A
:20A000006C4DA660A86980B110A800900DA90EAA0FAB30460BF0F2FF0E980B214FF6FF72E5
:20A0200050231DF0A5FDFF2808D020F0CFF882462878022804DB504620F052FA5C46B3E090
:20A0400000286DD107F088F95B495C4E086840F00200086009A8C9F800601FF00BFE584E3A
:20A060005849707809AA0B9005F1E00018F012FE554905F58E7009AA18F00CFE09A81FF000
:20A08000C1FD192109AB3078504A0A9005F160001BF080F84E4A05F17C001A2109AB1BF05B
:20A0A00079F84C495A4605F5AC7013461AF0B4FC49495A4605F5CE7013461AF0ADFC4748CC
:20A0C0000068C0F3814030B1454A05F1340004215B461DF089FDB078012802D10E200FF060
:20A0E000F3FC05F1A0001FF087FB05F198001FF083FB594685F8241085F83010072085F87E
:20A100004002A960E962374B1970E960052685F83110354A2E610420AA621EF02FF8287859
:20A1200005EB8001401CC1F8B840C0B22870504620F0D6F91FB901A81FF086FB01AF3868C1
:20A140004FF4FA76E6602060B8694146A062388A61766083F8692063786800280CBF40F673
:20A16000C410594620616061204E266266622176E661F86800B12062786900B16062B86887
:20A1800000B1E061C82204F13800594614F0DEFB04F1500059461DF0CDF815495A4604F191
:20A1A000B80013461AF038FC204611B0BDE8F08FCC21084030F5002000200940110000E031
:20A1C00050C302000D9302007D880100011C020015090200E9860200FD8C0200B44F005034
:20A1E000E5360200FD130120B967010077F500005DA102002DE9F04715469F4A13680F4623
:20A20000ADF1A00D23A90B6053684B6012890A8101A91DF0D9F98046B8F10A0F00F0278187
:20A22000B8F10D0F00F0238112A801A902221FF035FA814601A9022268461FF02FFABDF8CF
:20A24000000010F0070F13D0BDF8000000F00700022818BF022413D10DF106014846082291
:20A260001FF01CFA0B240DF10E010122814603E00DF10A010422062448461FF00FFA8146EA
:20A280009DF80500800908D30DF10F01484602221FF004FAA41CE4B281469DF805008011AB
:20A2A00041080DD30DF11101484601221FF0F6F981469DF80500641CE4B28011410803D290
:20A2C0009DF8041089090BD30DF11201484604221FF0E4F981469DF80500241DE4B28011EB
:20A2E000400808D30DF11601484610221FF0D6F91034E4B281469DF80400C0093AD3002058
:20A300000DF1260A8DF898000A22514623A81EF021FC2646641CE4B278B901220DEB060065
:20A3200026A98DF8982048301FF0B8F951460A221FF0B4F90A34E4B281460DF1300A23A8BC
:20A340000A2251461EF006FCA0B99DF898000DEB060326A90122401C8DF8980003F14800FC
:20A360001FF09CF9484651460A221FF097F90A34E4B281469DF80500400836D39DF83A30C4
:20A3800026460020641C8DF89900E4B2580811D301220DEB06000DF199018DF8992048304A
:20A3A0001FF07CF90DF13B0104221FF077F9241DE4B281469DF83A00800816D39DF899002E
:20A3C0000DEB06030DF199010122401C8DF8990003F148001FF062F90DF13F0148460422AF
:20A3E0001FF05CF9241DE4B281460DF14301484601221FF053F981469DF80400641CE4B297
:20A40000000903D39DF80400400906D211A9484601221FF043F9641CE4B217B9287818BB94
:20A4200020E02878264608B1A41EE4B20DF1020102222018ADF8020038461FF02FF92878A6
:20A4400000B9BF1C422E0744A8BF012010DA3246384612A91FF022F92878002818BF9DF82C
:20A46000020003D1A41CE4B2287800192870404628B0BDE8F087C04648C002002DE9F04F80
:20A480008246ADF1240D12980D460890287A984617464FF0000B012818BF032808D1BAF1BA
:20A4A000000F05D0BAF1FF0F02D0032802D10FB95C4612E104A80A221EF0ECFE894C207895
:20A4C0008DF81A7020BB0420874E8DF800003088ADF802001EF0AEFE01AE014630461FF080
:20A4E0006FFC68460BF078FA1FF0CEFCBDF8021081420BD04FF6FE71814207D0ADF80200A3
:20A5000030461FF0EDFD68460BF066FA01202070287A4FF004095C468DF80090022815D05E
:20A5200003280AD001281CBF4FF6FE71ADF80C1017D12888ADF80C0012E001A829461FF03B
:20A540003FFC684616F0E2F838B109E02888ADF80200684614F034FA10B968460BF03CFA81
:20A56000287ABDF80C10012819BF3A1C271C0127221C4FF6FE70884200F09B805B484B46AC
:20A5800026460E3810F80E5FDFF864C1554508D14578BD4205D145888D4202D105799542CF
:20A5A0004DD05B1E06F10106ECD1002C48D14F484B4626460E3810F80EEFBEF1FF0F04D095
:20A5C0005B1E06F10106F6D173E080F800A0477004464180B8F1040F0271C8BFC8466046A6
:20A5E0008168B8F1000F17D0089D4746E146AD1E35F8022FADF81C2011B104A888472A8881
:20A600001146504601235A461DF08EFBD9F808107F1EEDD14FF0010B089984F80580A01D05
:20A620004FEA48021EF036FE3048330131460E22A3EB46031B1802201CF004F839E004466B
:20A64000B8F1000F35D0089D4746E046AD1E35F8029F204649461DF0EBFD40BB34B36079A7
:20A66000042823DA04EB4000A0F806906079401C60711E48330131460E22A3EB46031B1803
:20A6800002201BF0DFFF08F108002A880168ADF81C2011B104A888472A88114650460123B2
:20A6A00000221DF041FB4FF0010B00E000247F1ECDD1BBF1010F10D10E48007880211AF08F
:20A6C0004BFA40B11CF0EAFA05461FF0F3FA0121284619F0F3FB1CF0F9FA204609B0BDE8C3
:20A6E000F08FC046FC0201201EFB00206C010020DC0201204DFF00202DE9F04F07460020C3
:20A70000ADF1340D002106900C22079003A814F01DF907F1240414F8011B01F00300C1F329
:20A720008018089000208DF80C00CE110A901AD020460078022500F00701641CC0F3C103E1
:20A74000C0F380198DF80C10C0F340120993B9F1000F0B9218BFB8F1000F40F00281184675
:20A76000012805D1FDE081460B9001254B4609930898012824D09DF80C0050B1022812D1DC
:20A7800014F8010B6D1C07F1080108220A90032004E02146022004222D1D241D387404A8BA
:20A7A0001EF078FDEDB268460021082214F0CEF804A8694608221DF067FF002840F0D18013
:20A7C0000998022810DAA3469BF80000E02803DBB8F1010F00F0C58097F8223097F82300E1
:20A7E0000793401BC4B212E007A8214604221EF051FD97F823002D1D211DEAB28B46801A23
:20A80000001F0422C4B206A809191EF043FD089801281AD1002E40F0A4809BF80000F0287E
:20A8200080F29F800998002840F09B80B8F1000F0BD1002001464C4A8DF800001226019193
:20A8400001231660684600F079FD04F1440080B21DF043FE061C00F0848004203070012195
:20A8600031750025757097F92000707597F82100B07597F82200F075387CB9F1000F2A46CB
:20A8800086F8200018BF0A1CAA46B8F1000F914618BF8A46022808D0032808D106F11800E2
:20A8A00004A908221EF0F6FC01E038893083B88B7084089D86F824509DF80C0086F825005A
:20A8C000099D86F82650DDF82C8086F8278086F828A086F829900498F062DDF8289086F8C2
:20A8E0003090079B7363069AF2639BF8000086F8380000201BF0BEF930710020B060FF230D
:20A90000F3607868306120201DF0E7FD0746174890F800A01FB930461DF0C6FE21E01449F1
:20A9200030461EF007FC0720387000237B70307959462246387706F141001EF0ABFC86F8E9
:20A94000404087F81090079887F8158003A93D750C22B861381D1EF09DFC5046394618F0E7
:20A960009BFE0DB0BDE8F08F480501209C0301205C190020F0B5064600240A20ADF15C0D54
:20A980004FF6FF7502228DF85B0021468DF85A403768ADF80E500DF1560013F0D7FF9DF810
:20A9A000560007F0070100F0F800014341F018018DF85610BDF85600203D21460540F808CD
:20A9C00000F020002843C7F34115ADF85600012D08BF01212246032D08BF01229DF856006D
:20A9E00062F39F1040EAC11022468DF8560005B901222046022D08BF01209DF857103B0977
:20AA0000022D01F0E00140EA010003F0080141EA000141EA02118DF8571009D09DF85700F3
:20AA2000F90A01F0200100F0DF0001438DF85710C7F34120012899BF9DF8570000F0BF00CB
:20AA40009DF8570040F040008DF857009DF85710022201F07F019DF856008DF8571040EA2C
:20AA60000120ADF80C0003A90DF112001EF016FE306810F0070F13D000F00700022818D18B
:20AA800005A806F1080108221EF008FE022006F1080108228DF8000001A81EF0FFFD08E05F
:20AAA00006A8311D04221EF0F9FD8DF800407068019007A806F1100101221EF0EFFD3068D6
:20AAC000400C34BF0DF10E0106F134010DF11D0002221EF0E3FD30689DF85A700122400A6D
:20AAE00000F01C0100F00300084347EA00018DF85A100DF11F000DF15A011EF0CFFD08A8EA
:20AB000006F1200104221EF0C9FD09A806F1240110221EF0C3FD0DA806F1110108221EF060
:20AB2000BDFD0FA806F11A0102221EF0B7FD0DF13E00FF2110221FF0B1FB3068C0F34110C7
:20AB4000022820D1BDF80C1012A80122C1F300211FF0A4FB0DF1490006F11C0102221EF01C
:20AB60009DFD3068400C0BD2684614F09DFD04A9ADF810000DF14B0002221EF08FFD0DE0D8
:20AB800006F13401F6E712A8214601221FF086FB0DF14B00FF2102221FF080FB0DF14D0076
:20ABA000FF2104221FF07AFB0DF1510006F1360101221EF073FD9DF8120000090BD29DF88B
:20ABC0001200400907D20DF152000DF15B0101221EF064FD05E00DF15200FF2101221FF07E
:20ABE0005DFB31680DF11200FCF792FB17B0F0BD2DE9F04F994E96F83D0096F83F10F37811
:20AC000096F83C800027ADF12C0D0918491E91FBF3F296F83D4077705A43891AC9B20891AD
:20AC2000810001EBC0018919B1F84C0096F83C10ADF81C00880000EBC1008019B0F84C50A3
:20AC4000CDF8248006A81AF0F7FB70780A97A04500F0A180B946CB46BBF1010F00F0908096
:20AC6000BDF81C10162966DD002840F09580BDF81C0001AAC01F81B2ADF81C10204610F03F
:20AC800061FDBDF81210BDF81C30884608F1070008F1100287B29A4246D89DF80E00962811
:20ACA00042D19DF80F00420839D2800837D3BDF81C0000230093A0EB08001FFA80FA9DF8B4
:20ACC0000D20BDF81C002346401A80B21BF07EFAF8B9E819B0F5005F15DCF068C5F188526F
:20ACE0000AEB443A3B46D21B514602F500521FF0C3F9ED1909F10109ADB2B5F5005F08BF8F
:20AD00004FF0010B0BE0BDF81C004FF0010BC01D2EE0BDF81C00401EADF81C0004E0BDF86D
:20AD20001C00A0EB080023E0204607A916F0C4F801281FD030E0F278B9F1000F07D0484BD4
:20AD4000BDF81C70A10001EBC401C9188F830899A14220D04249641C94FBF2F05043241AAC
:20AD6000E4B2A00000EBC4004018808B4FF00009ADF81C0009997078A1427FF46DAF0AE09C
:20AD8000B9F1000F07D0364ABDF81C70A10001EBC40189188F8320B106981EF063FA102053
:20ADA00059E0DDF824804FF6F0704FF40051C5EA0040C5EA0141E1FA40F01FFAA0F283B2DD
:20ADC000102102F18852404618F058FF71780843707006981EF046FAA0450FD1F278204FF2
:20ADE0001019401E90FBF2F15143401AC4B2A00000EBC400C019808BADF81C00184FBDF8EA
:20AE00001C00A6F840504FEA8801A6F8440001EBC80186F83E40C9198D83B6F9422096F802
:20AE20003D10012340461CF0CBFE96F83E10B6F94420022340461CF0C3FEBDF81C001628D0
:20AE4000DCBF01200A90B5F5005F03DB0A9840F002000A900A980BB0BDE8F08F5CFC00204E
:20AE60008CFC00202DE9F0410546A88CADF1380D0328C0F22881954F0024069507F1180048
:20AE80000B94AE6A09940822ADF828402146056007A81FF003FA079816F8012B20F00700B0
:20AEA00002F00301C2F380030143104641EA830102092CBF41F0080121F00801000960F375
:20AEC0000411079133B171783078B61C00EB0120ADF8200016F8010B8DF82200AB6A16F8C9
:20AEE000010B0996AA8C8DF82300F61A901BADF82800287D1EF0D6FEB846002800F0E18043
:20AF00008068002800F0DD80408800909DF82330079AA988287D02F003021AF0DFFF002816
:20AF200000F0CF801EF02EFF0246D8F80810A888012741B18B88834202DCCB88834203DA72
:20AF400009680029F6D121460798002900F00306C0F3800034D050EA060303D19DF8233032
:20AF60000B2B2DD0D2092BD36B7E4BBB0699487D002840F0A6804888002840F0A280224642
:20AF80001EF07CF8079E9DF82300069A8DF83000F00880F0010000F001000090BDF820506E
:20AFA00001959DF82200911D0290107D92888DF831700CAB1AF098FC3A461EF05FF880E09D
:20AFC000002E4BD1002847D19DF82300172841DA3F4E56F8301000293CD0287D8DF810004B
:20AFE000BDF82870ADF81270099D059504A888470B9048B906994F7D002F62D14F88002FB3
:20B000005FD10798802743E09DF8231006EBC106716819B106A888470B9808B11FF07CF818
:20B020009DF8231031F002004BD0032949D0052947D0062945D0082943D00C2941D0112978
:20B040003FD013293DD015293BD00B2939D02746069915E08227FBE78427F9E749B1896810
:20B0600039B106A888470746FF2F2AD00798C0F380000699012F03D1002814BF8327812732
:20B080004E7DF6B94E88E6B90798420900D3C7B1C0089DF823208DF8317080F001008DF8D0
:20B0A000302000F001000090BDF8206001969DF822000290087D8A888B1D19460CAB1AF04B
:20B0C00013FCC8F818400EB0BDE8F081800301204CB502002DE9F043054697484278ADF103
:20B0E000B40D8DF8012000218DF8B21088468DF8008082788DF80220C2788DF803200830F3
:20B1000058C802AA58C209C8C1464746464682E809002979CDF80490C1F3C1008DF80810D8
:20B1200040BB11F0070F13D001F0070102291DD14FF0FF30039005F10801082204A813F02F
:20B140004AFF06A805F10801012213F044FF0DE003A805F10801042213F03DFF04A8FF21C8
:20B1600008221FF09BF8FF208DF81800FF208DF8190013E0012811D14FF0FF300390FF216B
:20B18000082204A81FF08AF8FF2005F1080101228DF818000DF1190013F01DFF4446204644
:20B1A0000DF12A011CF010FA30B99DF80100401CC3B28DF8010001E09DF80130641C052C22
:20B1C000EDDB9DF80800C0F3C100012842D1002B00F0A2809DF819409C4200F39D80062C0F
:20B1E00012DA9DF8B260204641460DF1B202FFF701F848B99DF8B2004A2803DC641C062CE3
:20B20000EFDB01E08DF8B2609DF8B20010B39DF8B2001FF041F8071C1CD041468DF80380B5
:20B220009DF819408DF8B210062C13DA204639460DF1B202FEF7DEFF60B99DF8B2309DF82C
:20B2400003009E4200F101008DF8030002DD641C062CEBDB9DF80810C1F3C10000284ED1D1
:20B2600011F0070F0CD001F00701022947D102208DF81C0004A9082208A81EF00FFA03E05B
:20B280008DF81C8003980890FF208DF802000DF16E010AAA07A814F059FDA0B99DF8B240AA
:20B2A000BDF8280041460DF1B202FEF7A3FF30B99DF8B2004A28C8BF8DF8B24006E04146D4
:20B2C0008DF8B2101BE08B208DF800009DF8B200A8B19DF8B2001EF0DFFF071C0FD04146A0
:20B2E0008DF8B210BDF828008DF803800DF1B2023946FEF77FFF10B901208DF803009DF877
:20B3000019008DF8020028680197694610F03CFC38461EF001FF0BE09DF819008DF80200D2
:20B320008DF8008028688DF80380694610F02CFC2DB0BDE8F083C046E8C002002DE9F04F9F
:20B3400005460020ADF1340D8DF81A0028789A46894658B1022840F01A81291D04A808229B
:20B360001DF098FF4FF00808032006E04FF6FF704FF00408ADF810000220DFF818B28DF8D5
:20B380001800002701E07F1CFFB2D7B95BF82740002CF8D02E7820798642F4D104F108003A
:20B3A000291D42461DF070F90028ECD0022E02D0002EE8D105E0B9F1FF0F02D0207C4845E4
:20B3C000E1D1012F00F0E380B90001EB0B0000245BF801700790BAF1010FFC7009D12046A2
:20B3E0000090012122460190234602908A46039108E02246009201920292012003902B78E3
:20B400000DF11A0051461AF0FFFF8346079800685FEAEB1600F1170500F10407017C90F84D
:20B4200016900995437C08919DF81AA00A930BD09DF81A00C0F3C100022803D0032818BF87
:20B44000032602D10B2600E002261BF0030F07D13D78022D02D01DB9361D00E0761CF6B2C9
:20B460004E44F6B2304611F0F5FB00280B9046D005465FEAEB1805F801BB18BF05F801AB82
:20B480001BF0030F11D13B78022B0BD06BB9387905F8010B787905F8010BB87905F8010BE0
:20B4A000F8790890089805F8010BB8F1000F0DD0CAF3C100022818BF032807D105F8014B7A
:20B4C00005F8014B05F8014B05F8014B0A984A46099905F8010B28461DF0DCFE4D44B8F125
:20B4E000000F0CD0CAF3C100022818BF032806D105F8014B05F8014B05F8014B2C70DDF894
:20B500002C80B8F1000F42D0B1460798224E00687768C57890F812A027B170681DF0C4F878
:20B52000204670602C201CF0D8FF074677605FB3680829D2384621462C2213F007FA4FF689
:20B54000FF7BA80803D3F88A40F00100F882F88A052540F4807004A9F8820A22FC7607F131
:20B560000800BD761DF096FEA7F812B0C7F828803C7587F82790094887F815A032680078A9
:20B5800001211EF0E8FD02E0404619F005FB0DB0BDE8F08F58190020480501209C03012085
:20B5A0002DE9F04F0546ADF1140D02911EF00EFE8A4C012D039000F0D280A346DBF80000EA
:20B5C000D0F838038047002800F0C58016F0DCFF002800F0C080DBF80410864C8969606898
:20B5E0000F783C30002F40F0B6807D4E0068357880477168F268AB00401AB0FBF3F7B06837
:20B600004FF00008C2469146534611464F4573EB0A0301DA884206D84146524687428A41DF
:20B6200043DA024600E041461046EB172A46C01B71EB08011DF08AFF07466F480068884666
:20B64000418B00694018643081464FF00001B7EB090778EB0A08784271EB080125DA1EF06F
:20B6600007FC024653464146384614F04CFC884607464FF00001784271EB080115DA1CF020
:20B6800059FD054630691EF09DFA10B130691EF095FD28461EF031F8306939461EF08AFD7F
:20B6A00030691EF089FD002000E001204D490870884698F8000000284DD1DBF80000D0F8EF
:20B6C000940000780027394615F05AFC00B101274FF0000A381C3CD1DBF8040080690078A2
:20B6E000002836D16068404D436C286902216A4698479DF8000060B302984FF00109012820
:20B700001ED03A4F6268286997F9001011F1020F05D0926B97F90010904762682869344E7E
:20B7200096F9001011F1020F05D0926B96F900109047626828696FF001013170397001E028
:20B7400062682869DBF80410896981F80090D169884788F800A003981EF0C2FE3AE0206878
:20B76000D0F894000078012115F00AFC03981EF0B7FE606880690078012811D11DF0C4F86D
:20B7800060B1606880690178012909D10021029F0170012F04D01DF085FE01E00FF096FE2F
:20B7A0001DF0B2F8B0B960680C30C1680978022909D101680F7837B12068D0F84C05804776
:20B7C000241D20680C3001680F781FB9C16808780228FCD005B0BDE8F08FC04614010020E9
:20B7E000D800002008140120700001200C0501200D050120DCFF0020800001202DE9F04F2D
:20B80000002124220823ADF12C0D68461EF058FE7C4E002421466A4606F138058DF8184097
:20B8200028461EF049FE06F10C0000F1040B05601EF03EFEF16806F1100215F037F830705D
:20B8400086F8244086F82540B48316F011FD4FF0080806F1280080F800806B49316310F02A
:20B8600051FE6A4D287830B9694A204614211AF06DFB012028700C201EF00EFD6F68B146AD
:20B8800088B1046009F1540180F80480816037B9686008E011467FE0114654E00F46396808
:20B8A0000029FBD138601EF05DFA5A4D40460A212A1D1AF02FFB584E776840461CF0EAFDC5
:20B8C000F0B1DFF858A12546BD4208D03879082814D03B6803B93D461F46002BF6D10C208B
:20B8E0001EF0DAFC60B10460514680F8048077688160002F0CBF7060286001E05146B960B9
:20B90000474DF22705F13C00077005F16001696410F0F8FD434E307830B9434A2120014681
:20B920001AF014FB012030700C201EF0B5FC716868B1046005F12C02077173688260002B68
:20B9400008BF706003D00A68002AA5D10860374A38460C211AF0DEFA38461DF073FB10B13B
:20B9600033498160C460204614F0B8F916F0CCFB1CF062F90C201EF08FFC2E4AD16880B150
:20B980000460012380F80480224E4371D768002F866008BFD06004D00A68002A7FF47AAFA8
:20B9A000086099F80000D9F80C70C5F824B04FF480764FF40073E8701F49AF623222AE806E
:20B9C0004FF48067EB8005F174002F8118F00AFA1A49A8614FF4FA6205F1980018F002FA0F
:20B9E0001749E86141F2883205F1BC0018F0FAF928628DF8244009A81DF094FF0BB0BDE8E0
:20BA0000F08FC0467CFB0020F4030120081800209927020060B90200F8FD002065E5010075
:20BA2000481900207004012065420200FCB302006D5E020080030120559602006D96020033
:20BA4000859602002DE9FE4F824C00906068C06801910121017080484FF0000A80F800A0CA
:20BA60007E4880F800A02068403001680D681E46174615B9D0F80C0580477949DFF8E481E5
:20BA8000DFF8E491886E4FF0E2450AEA0702354008BF002A40F089800D46B5F89E1008228A
:20BAA00053463A4013EA060708BF002A0BD118B14246508B401C50834A4692F90000401EC8
:20BAC00010701D20ABE04A4692F90030DFF89CB142F201468E42A3F10103137002D0321D28
:20BAE0008A4216D118B14246508B401C5083584600680199826C0098904750B1424602F1BF
:20BB000016010088B5F89E30098842F60147874233D15748411C0A78B5F86610B1F5105F77
:20BB200012D0AF6E42F60600884206D0002FC8D04246508B401C5083C3E7002F71D042462D
:20BB4000508B401C50836CE0A96F5B460C3319604189062A0CD1427A022902F101024272B6
:20BB600006DB491E89B24181062003F089FF58E018F026FE0FF06CFF53E0491C361D88B2EC
:20BB80009E42D08214BFE1201C2011F04DFA99F9000020B199F90000002854DC48E020681E
:20BBA000D0F85824514650464CE04A4692F900102768491E117007F1400118B14346588BD8
:20BBC000401C58830868006840680078800925D2284A1078832824D125484378032B1BD1DA
:20BBE00004234779D1F8945013707B1CDBB2437195F8241099420DDB817895F831304D1C82
:20BC0000AB42C4BF491CCBB28370832010701DF0E5FC06E0E12002E0852051E7E92011F01E
:20BC200003FA99F9000040B199F9000000280ADC2068D0F84C05804705E02068D0F85824CB
:20BC40005046014690476068C06880F800A0BDE8FE8FC04614010020100501200F05012050
:20BC6000501800208C11012012050120E0FF00204C0201200A1401202DE9F047884E05462B
:20BC800096F84A00ADF1200D08280CD004280AD0287800F00300012840F0FA802869007880
:20BCA000062840F0F58068884FF6FE74844200F0EF80718F814206D1287F20B9284613F05A
:20BCC0003BFA0446E5E01CF027FF002840F0DE80287F4FF000092746E8B1724800780421EC
:20BCE00040EAC00010FB01F05FFA80F8698885F81C80FF201BF0E4FB8A4648B1E88A48F007
:20BD000001034FF00109671C2B7740F00400E8824FF0400802E0B5F802A0C846504618F0AF
:20BD2000DBFE08B100206876A87E08B90F20A876287830F07F0008D1E87E50B996F8240006
:20BD4000411C86F82410E87603E0287800F003002870287E012806D196F82F0018B9287894
:20BD600008B90020287696F8320080081CD3B9F1000F0AD1688818F0AFFEA8B1287820B10A
:20BD8000286900781DF096FE70B1E88AC00902D3A87E012804D028461BF0CCFD20B975E035
:20BDA000E98AE01E0840E8822878012807D128690078022803D1E88A40F04000E882E88AFA
:20BDC000C00937D2B9F1000F34D196F83200800830D3687E6988AA1D434613F043FB28B147
:20BDE0000020EB8A687643F02000E882A87978B1698805F1080018F04FFE07466888B8424E
:20BE000004BF0021A971E98A41F04001E98200E068882978012904D0A98842460FF050FF5E
:20BE20006888A98842460CF027FB18B1E88A40F02000E882284606A907F000FC8046BC4272
:20BE400008BF6F88B8F1000F1DD0059528788DF810006C8DADF812406B7D0093E88A019042
:20BE600095F82C00029004AA0392728F9DF81830394640460DF0B0FC0446102C04D14046C7
:20BE800018F08AFE00E0102420461AE7112400E0C224284618F080FE204608B0BDE8F0876E
:20BEA000E4FA0020B7FE00202DE9F04F7F4E7068416EADF1340D02A88847DFF8F4B19BF99E
:20BEC000000038B17B4890F90000002818BF002040F0E9801EF07AF9DFF8DC910A9099F885
:20BEE0000000800806D27D2000210DF08FFD0025079001E00025079502958DF80C5005952B
:20BF000003228DF818206D4CA4F8BE50C4F8C45094F8C800012705F00F013B4620F00F00EB
:20BF2000014384F8C810DFF898A10B9394F8C81063F3C71194F8D73084F8C81023F001002E
:20BF400007F0010343EA000184F8D71094F8D70067F3410084F8D70094F8D70065F38200C7
:20BF600084F8D70094F8D70065F3C30084F8D70094F8D70065F3041084F8D70094F8D70018
:20BF800062F3461084F8D700DAF80000D0F8282404F1D801F4209047DFF8288198F80030C4
:20BFA000A3B94946706809788446890910D3C06B8047C4F8C40094F8C81021F00F0141F0D6
:20BFC000020184F8C8108DF80C700290D6F804C03E4A3D484FF080738DE80C00DCF8507091
:20BFE0003B4B006804F1BC01894602AAB8470028708006D5022041F2883115F057F80B9532
:20C000004DE02C49334F91F90000401C087097F90000401C38709BF90000C6F808902946B1
:20C02000401C8BF80000022015F040F8DAF8001001F1AC021068077888F8005007B180251C
:20C04000308F17684FF67F7303401D432843308794F8D420387860F3C71284F8D420D1F811
:20C06000D400C28CA6F84620428D00F14403A6F844201A6806F13B052A6058686860D1F8FD
:20C08000D400C18CA4F8EE10418D00F14407A4F8EC10396804F1E4063160786870600A98E0
:20C0A0001EF01EFA0B980DB0BDE8F08FDCFF002014050120130501200614012050180020A5
:20C0C00014010020110501208000012020004300F9470000120501202DE9F04F0746861C34
:20C0E000ADF11C0D30461EF027F882490446182268460FF0FBFC7D780DF10B0031461EF060
:20C100004BF84FF6FE794FF0010802208DF8160000208DF80800B87AADF81490810805D392
:20C12000B87A000934BF0326042603E000092CBF0226464670480078002808BF002D00F0B7
:20C140008E80704890F84A10082940F08B801DF021FD10B1012D00F08280002C27D0207903
:20C16000864218BF022D72D1042818BF032803D1042E10D0032E0ED0022818BF012812D17E
:20C18000022E08D0012E06D0022818BF01280AD11EF02EF807E0208882461BF03DFE08B9FB
:20C1A000ADF814A003E0B81C16F024FC0024BDF81430DFF848B1994514D11BF089FC70B9E0
:20C1C0005846008882462DB11BF026FE002808BF504601D01DF03EFDADF814000346484636
:20C1E000984231D018462B4612F078FA07F1020A002839D15846001D016811B1BDF814003C
:20C200008847BDF81400514632460AF069F904463C4800784FF4803141F288321DF09BFF4D
:20C2200038494046087164B1022D05D0012D11D1607940F0100002E0607940F00800607178
:20C2400008E0ADF814900FE04FF0C7080CE02088ADF8140000208DF81600804604E04FF0BF
:20C26000C30801E04FF0C208CDB125480078A0B9012D12D144B902208DF8160031460122E8
:20C28000684610F0A1FC31E0002001228DF816006846314610F098FC04E02A46F8E76846CA
:20C2A00017F0B8FA06469CB145B16079022D40F04000607104BF40F020006071B87AC0090E
:20C2C00003D3607940F080006071A079401CA07156EA08000AD014B1B81C16F08BFBBDF8AC
:20C2E00014104846884201D01DF082FF07B0BDE8F08FC046E8B8020034040120F0FB00207C
:20C30000ADFE0020E4FA00202DE9F04F09AF8846ADF13C0D0026079098F80350B8F806102C
:20C320000993B868089204240B903879DFF8F0910A9019F80E0F854205D148461BF078FF66
:20C3400008B1761CB6B2641EF3D1002EB34600F0CD8098F81440F1B2182000EBC10085B2DE
:20C36000601900B210F076FC041C06D02A46002112F0ECFA26746019E060002C00F0B18011
:20C3800098F80350B8F806100022284619F09EF906466571B8F80600E08098F81600608105
:20C3A0000021217298F81420D8F81010E0681CF071FF00250C95B8896082387C0D95A94623
:20C3C000207551E04FEAC900002104EB000A0019817570780AF11605012810D0B0788AF8BB
:20C3E0001D007088ADF8180004218DF80C1003A816F074FDBDF80E00AAF8180005E0012000
:20C40000287001230C93708868803079287198F80000C00903D3A87940F00200A8710C9860
:20C42000B0B9404869880088884211D1287988F802000A9E00960B9B01930D9B0293089A6C
:20C44000079940460DF064FDA87940F00500A87109F101005FFA80F9B8F8061098F80300C3
:20C460004A4619F033F906460EB1CB45AADC2E4D281D06680D98314604E00E4620E0096863
:20C48000401CC0B20029FAD1052813DB96B1334600E01B6813B99E4202D00BE09E42F8D18A
:20C4A000306801216860304614F05EFF304618F073FB6E68687820716878401C6870204676
:20C4C00016B131680029D8D10D99002E01600CBF686030600A9B009409993A78404600F0CF
:20C4E0004BFBBBF1000F18BF002C15D198F8030098F816708DF80F00B8F806608DF81070FA
:20C50000BBF1000FADF812600CBFB92010208DF8140003A81DF04DFC0FB0BDE8F08FC046F2
:20C520005E0100201EFB0020400501202DE9F041844FB81C00780D46290C1FD2E80B38BF14
:20C540000020C0F0FB801BF0F5FD7D4C804604F10C00006858B107463E6938461DF0A4FF70
:20C56000384618F019FB371CF6D10020E06040461DF0C3F885F48040BDE8F08115F0E4FA27
:20C58000061C00F0D9803078F9780024D2280EDCD22800F0C7801A3860D01738052840F2AE
:20C5A000C1809F3800F0BE80401E48D0B2E0D33800F0B580401E022840F2B480293823D0BB
:20C5C000401E40F0A78016201BF087FF071C00F0A9802146162212F0B9F9932038707C7009
:20C5E00070783871B07838743079012814BF02200120B871F0883881F0783875B0781CF04B
:20C600006BFC00287DD080E00A201BF066FF071C00F0888021460A2212F098F991203870AA
:20C620007C70B078787170783871F078B871B0883881B0781CF050FC002862D065E07078E3
:20C6400088426FD0404BF870FA1C21464FF000701AF05CFC78783D49087063E030201BF0C4
:20C660003CFF071C5ED02146302212F06FF9922038707C70B07B032838711CBFF088F880FB
:20C6800004D1B81DB11D08221CF004FEF07BB873308A388270887882B088B882708AF88208
:20C6A000307D3876737D204603B101207876707E214600B10121B976B07DF876F07D3877F8
:20C6C00096F918007877F069386296F8200087F82400B08DF88496F82E0087F82800B08C28
:20C6E0007885B08C10F0B6FAF862D8B1B16AB28C1CF0D0FD307D1CF0EFFB30B9F86A18F046
:20C700004BFA38461BF0D0FF0CE00079394616F0C3FF07E03046F3F793FC044602E0304658
:20C7200002F0D0FA012C03D030461BF0BDFF03E0B078314616F0B0FF85F40040BDE8F081FA
:20C7400080040120281A0020E17E020070FB00202DE9F04F8246DAF8185069782878EA78AC
:20C7600000EB0120A978ADF1240D044601EB0221069118F0B1F9012800F0D9804FF0000862
:20C78000CDF810802046CDF8148018F0A5F92D1D60B970480088A04208D06F48007830F033
:20C7A000010040F0D48040468123C2E015F8014B5CB1600010F04EFA049030B1049A2046A1
:20C7C00029461CF05EF9054600E0444615F8017B5FEA07090AD0780010F03CFA059028B1FA
:20C7E000059A384629461CF04CF900E0C1465B480568002D76D046460796089668680178E2
:20C8000000296CD0AA7B520869D3AA68002A04BF8668DDF820B004D0012090474FF0010B4F
:20C820000646002E5BD070880699814204D006984FF6FF7181424CD1F279B3680499204669
:20C8400019F0CDFF38B9327B33690599484619F0C6FF00283DD009EB0400022110FB01F083
:20C860001430C0B21BF039FE071C2AD0D2203870BAF80200788087F80C90002C3C7104BFA6
:20C880000798B86008D007F114000499B860620007F114001CF0FEFCB9F1000F04BF0898B8
:20C8A000386108D0059907EB44004FEA4902143038611CF0EFFC686840680078394616F066
:20C8C000EBFE3078264908F1010701F808005FFA87F8BBF1000F02D0304618F05DF92D6888
:20C8E000002D8BD1B8F1000F05D19AF80C00A8B90023984600E00023164800880090CDF8E3
:20C900000480174F02979AF8100003909AF811100AF1020248F2060014F064F8049808B1B8
:20C9200018F03AF9059890B118F036F90FE0002080230094019002909AF8100003909AF877
:20C9400011100AF1020248F2060014F04BF809B0BDE8F08F50FD0020ADFE002024050120D1
:20C96000A8FF00202DE9F041064606F11600ADF1380D18F0F1F97A48007806F11607012804
:20C9800018BF02282FD100200DF1320501A905AC8DF8320001220095601A83B201A907A86F
:20C9A00017F0B4F898B16F4800680DF1330101AA11F04EFFADF81C00BDF81C40032C12DA44
:20C9C00003A8394608221CF065FC214606E003A8394608221CF05EFCBDF81C100420142254
:20C9E00001AB19F02FFE3846FF211CF07CFB10B15D4901200870002402A839468DF804401E
:20CA00001DF0CAFB1DF0C6F848B901A813F07EFE012804D02046394608AA1AF00FFD3079FD
:20CA2000534D012861D006285FD0691C0B7804282AD0032840F0918038460DF11E011AF060
:20CA4000A3FF58B14FF6FE7039460DF11E021AF0F5FC214638460A4614F06CFEBDF81E006A
:20CA600006A91AF001FD069838B906A81AF0E6F818B9BDF81E0006990880B11D38460FF0C4
:20CA80001DFE13F095FC68E0002B66D038460DA901AA11F0DDFE01469DF8340000285CD01F
:20CAA0008DF8154020460290019001278DF81640142201AB8DF81470042019F0C3FDB21D69
:20CAC0004FF4817010211DF099FA06F1060828B94FF48170102142461DF096FA6D1F3846D7
:20CAE0000321AC7119F072F837E0721D1021204612F8017F1FB9491E00F10100F8D11B4F57
:20CB000010280CD07179B01D1AF04CFB387808B12878D0B170790EF049FB2C7015E0387803
:20CB200098B9204662210DF1220212F049FD0DF1220021461AF036FB20460EF037FB0DF1FB
:20CB400022002146102211F001FF0A480178052903D1C079802115F025F80EB0BDE8F0817C
:20CB6000ADFE0020B800012056FE002049FB002051FF002034FD00202DE9F04F0646ADF139
:20CB80003C0D032700200A91189D0C93297C0B920CE005EBC002127F530805D3D30803D2BF
:20CBA00012093CBF7F1EFFB2401CC0B2814201DD002FEED1B9460124002010E005EBC002CE
:20CBC000177FFB1109D07A0807D307F0040207F00807174304BF641EE4B2401CC0B28142B5
:20CBE00001DD002CEAD1A346B9F1000F08BF002000F0C5804FF00008B7E04FEAC8002A1891
:20CC00004019007F02F11604400880F0AA80002723780D9793B9108B1DF05EFA70B1007901
:20CC2000012818BF032809D1A079BBF1000F40F08000A07100F0948001200D900C9800B143
:20CC4000202700210C22684611F080FE237813BB0A9800280EBF4FF0080A47F040074FF003
:20CC60000A0A60884FF6FE71814228D104208DF81800E379ADF8243006A816F02FF94FF611
:20CC8000FE7000210346B0800A46ADF8003007A814F050FD15E03B480078012808D060888E
:20CCA00047F00C074FF00C0AB0804FF6FF7006E06088FF2147F00807217141F2080AADF841
:20CCC00000008DF80270307D8DF8040001238DF80530684608F0E0FB9DF8141061BB039858
:20CCE000417D6171A0F816A00B9F4776277817B124490978017769890185698A4185297D4B
:20CD000080F82C10697980F83A10217980F83B10F188C1873189A0F84010717D80F849103C
:20CD2000B1888187406C327D31691CF0B3FA684617F032FE9DF81410A07940F00100A0710B
:20CD400051B90D9818B1ABF101075FFA87FBA9F101075FFA87F903E0A07940F00800A0711C
:20CD6000297C08F101005FFA80F8414503DDB9F1000F7FF442AF2846002114F0F5FA0FB07F
:20CD8000BDE8F08F70FB00202DE9FE4F9B461546894682461DF01AFA7B49019008680CAF0D
:20CDA000504508BF48687B4C6FF0010828B1B8301CF008FF002840F0D6801BF0CDF9061CC3
:20CDC00000F0DB8004F5CE701DF0F8F90023B4F9B400C6F80C90401C86F832306FF31F3008
:20CDE000A4F8B400C6F808B0B4F8B40030866748C6F810A097E80C0020210027B8461940F0
:20CE0000104006F1180383E80300424686F8332006F1200383E88001E8683064287C86F8DD
:20CE2000440028687063287986F83800A868F0636869B064A869F064287F86F85000687FEB
:20CE400086F851002F7C27B9EF6817B1012086F844002F795FB999F80C0000F00F000228F0
:20CE600005D1012086F83800D9F808007063484608274568002D18BF002F70D100886FF391
:20CE80000900B0F5305F18BF022506D196F83300082540F0100086F8330006F1180090E81A
:20CEA0000C00414606F1180745EA0200194387E80300D4F8D800824507D194F8DC004108D6
:20CEC00024BF00F0FE0084F8DC0031480768002F39D004F1A0000090D4F8A810D4F8AC20C8
:20CEE00004F198052B463046B84710F1030F10D0B6F93010B4F9B420914207D0B4F9B4103C
:20CF000001F6FF716FF31F31A4F8B41010F1020F1BD010F1030F18D096F83300B6F9308080
:20CF200040F0800086F8330000278AF8FC702868864205D0F068007B00F00F0002281CD165
:20CF400013F094F919E06FF00200B4F9B410804601F6FF716FF31F31A4F8B41005E07F1EB5
:20CF60002846FFB285E76FF0020894F8DC0040F0040084F8DC00C4F8D8A001981DF0B0FA45
:20CF80004046BDE8FE8FC046E8F50020FFEFFF9F5805012030F50020FEB50E461DF016F964
:20CFA00000257F4A7F4C517855708A080ED2C9081AD31DF095FAA4F1080000F108048068DC
:20CFC000D0F858242846014690470FE01DF088FA6068C068007828B92068D0F8582429467F
:20CFE000012090471DF0F2F81DF07AFAB00941D337E02168D1F8982050600098D1F840136F
:20D0000088472168D1F89800D1F85413001D884732E01DF0DBF82168CA6B117B491E117314
:20D020001DF05EFA216800983C31CB6D0278586000988DF8042047782FB1162A0AD1D1F8CF
:20D040001813684601E0D1F80413884721689DF804203C31162A06D0C86DD1F81813001D5C
:20D06000884721683C310868001D1AF056F800280090CED1300C08D32068D0F8940000783C
:20D0800014F062FD00280090B3D1700907D327682E20D7F840138DF8040001A88847700826
:20D0A00007D327682520D7F840138DF8040001A88847B00807D327682620D7F840138DF891
:20D0C000040001A88847F00807D327682720D7F840138DF8040001A88847300907D3276867
:20D0E0002920D7F840138DF8040001A88847F00909D32D2027688DF80400D7F840138DF8E3
:20D10000055001A88847300A09D3302027688DF80400D7F840138DF8055001A88847700AD6
:20D1200009D3352027688DF80400D7F840138DF8055001A88847300B07D38DF805503720EC
:20D140008DF8040001A81DF0ABF9700B07D38DF8055038208DF8040001A81DF0A1F9206804
:20D16000D0F898000068C8B11DF030F82168D1F898100A6800920D601DF0B2F921680098F5
:20D18000D1F8982050600098D1F8401388472168D1F89800D1F85413001D88472846FEBDAC
:20D1A000D8000020140100207E492DE9F04F0A680746ADF11C0D0DF10E00026049684160E0
:20D1C000F88900280CBF08210221BC69DFF8DCB1754A14F801A0A0B9104621461BF008FF72
:20D1E00060B920461CF0A8FF4FF6FE7650B30179012918BF022925D106881CE059460E88E6
:20D2000020E0617820785E4600EB012031880646B14216D01CF060FF002498B10179012993
:20D2200010D18DF800404088ADF80C00684615F055FE00B101ACBAF1000F18BF4FF0FF0A92
:20D2400000E014464FF6FE71B14218BF002C03D13D7B002D40F0A38056484568B1424FF061
:20D260000B080DD064B13AF0010006D0387B012800F095804FF080090AE04FF0000907E0E6
:20D28000FB894FF08109002B0CBF4E1C0DF10E0405F8019B002C14BF211C0DF10E01284681
:20D2A0001CF07AFF0546BAF1010F05F8016B4FEA2620287064D158460088B04260D1B9F13B
:20D2C000000F5DD1DFF8E8903320002649460C791CB1032CBCBF761CF6B2401E01F124010F
:20D2E000F5D136B1022016FB00F000B20FF0B2FC00E0002003466D1C002B08BF00260DD038
:20D30000844633214846047924B1032CBCBF02882CF8022B491E00F12400F4D163B3FC89AE
:20D32000002C0CBF08210221B8694018417803EB4100B142A8BF002605DA761AF6B208EBBF
:20D3400046085FFA88F805F8016B297066B16D1E017805F8021F30F8021B761EF6B2002EBC
:20D360004FEA21216970F3D1184617F015FC08F102005FFA80F803E000204FF00C08287065
:20D380000C49FA8910204346C87042F4004207F11100B91C13F0C2FB06490020C87007B050
:20D3A000BDE8F08F44B7020020FC002050FD0020E40D002098FD00202DE9F04F074678695A
:20D3C000824600780321ADF12C0D10FB01F0401C80B21CF061FF5FEA000808BF002400F0F0
:20D3E000EC80002635464FF00709099512E0049931B93968087D228889881AF085FD01E06C
:20D4000019F06EF9ADF82000BDF820006D1CEDB23618B6B29AF80000A84223DD396815FBF7
:20D4200009A4641C087D2288898802AB16F094FB80B19DF80E00A178884209D19DF80F10F8
:20D440008A0803D38909D2D37E2004E0882002E08D2000E0862088F801002088A8F8020023
:20D46000012509950998002888F8000040F09180CB4610FB0BF0C4B2A01980B21CF00CFFCF
:20D480000A90002808BF002400F0948081460026A14404E0BDF82000761C8144F6B29AF8BF
:20D4A0000000B04268DD3968087D16FB0BF50AEB0504641C2288898802AB16F04DFB0028A2
:20D4C0005AD00A982388049A2D18C5F803902B808AB9396808A800902288087D89884B4602
:20D4E00019F0ECFD3968D4F80330087D02AA891D18F0D8FC0BE0484602A908AA1AF0DAF934
:20D500003968087D02AA2346891D19F0FEF90028C0D0099B032113FB01F108EB010208EBC1
:20D520000105507021885A1C6980D0B209901EB30A9C3968087D2288898805AB16F00CFBED
:20D54000D0B1079840B93968D4F80330087D05AA891D18F0A7FC0BE09DF81A00D4F8031014
:20D5600019F0BEF80246D4F8031007981CF096F8761E04F10704DCD1099888F8000028B949
:20D58000002088F80100012688F800600A981CF0C3FD78683A68C00880F0010000F00100C9
:20D5A0000090B87A911D0190107D928843460FF081FD012440461CF0AFFD20460BB0BDE894
:20D5C000F08F70472DE9F0470646F08917468946ADF1280DC01D80B205460EF0B5FE7A4C33
:20D5E000FF280BD12846FBF7EFFD854204DD641C207800B90520E3E0012000E00020617881
:20D60000D9B917B1022F18D1B8B1307A8DF80C00F788ADF80A70B588ADF808500023009364
:20D62000E18E94F8330001AA032305F0F1F89DF814003074BDF81070B78194F83310E58E11
:20D64000E06806AA0423884649031CF015FD069800F0FF0100F0FF007E2806D140467C2156
:20D6600019F0CCF9069901F0FF017C2940F0A580F08942F20102C11D8FB2E9198A4240F382
:20D680009A80F188327AC1F301238DF81D10B18843EA82038DF81C308A1006468DF81E205C
:20D6A0000423C0F3851201F0030142EA81128DF81F2010FB03F1F21D01F0FC01731990B2B7
:20D6C0008DF820101FFA83FA0D282BDB4846314600221CF003FC0246052107A81CF0FEFB70
:20D6E0009DF82010334600F03F064A4641EAA011B0008DF8201040F0020096268DF8210052
:20D7000029468DF82260404616F0B8FA0646514607AA07234046667016F0B0FA3043607048
:20D720004DD135E004F12400494632460EF0DEF907A90A68301900F12409484609790260C6
:20D74000731D0171002204F1240099B21CF0C6FB9DF82010962300F03F068DF8223041EABF
:20D76000A011B0008DF820103B4640F0020007AE49468DF821003268B0790A60B288887196
:20D7800040468A8004F12402294616F077FA6070E18EED194FEA8806AAB2C919E18606EB56
:20D7A000C8010919A1F84C2048B14046514615F04DFF607803E0052000E001206070C0B2EF
:20D7C0000AB0BDE8F087C0465CFC00202DE9F04705467B4895F80B900078ADF1180D00280F
:20D7E00008BFBA2000F0E980684600210C2211F0ADF801264FF0000A298B8DF80560C808AE
:20D800000AD39DF80220C8100B0942F040028DF8022038BF032602E09DF80220C8104B0988
:20D8200028BF46F0400640080FD342F0C00288098DF8022039BF9DF8030040F002009DF8D8
:20D84000030040F001008DF8030001EA6100000A28BF46F00806287A5A4F002830D00F28E1
:20D8600028D0022822D0032818D0012832D1387848B94FF6FD70ADF80000288842F00C025D
:20D8800046F0040608E0288842F0080246F480564FF0FF09ADF80000824619E0284669469A
:20D8A00019F064F89DF80220298B13E02888ADF800000FE0288842F0080246F0040605E050
:20D8C0001CF0F4FA9DF8022042F00402ADF800008DF8022048081AD312F00C0F0DD128882B
:20D8E00014F0DCFF002808BFBB2066D09DF80220298B42F020028DF80220480807D302F0C7
:20D900000C00042804BF42F020028DF80220A87C8DF80400684607F0BFFD9DF81400002832
:20D920004BD1039CE682E87E6076287FA076287A012804BF38782077A87E2085288B608593
:20D94000E87F84F82C00288B00EA6000000A15D395F82000667D804618F08EFE071C0DD0DF
:20D960003A7C002008E007EBC001CB7E984504BFCE763A7C401CC0B28242F4DCA87A84F853
:20D980003A0084F83B90A4F83CA0E889E087288AA4F84000A87E84F84A00A87F84F84B004E
:20D9A000687F84F84900606C69696A8A1BF072FC684616F0F1FF9DF8140006B0BDE8F08791
:20D9C000AF00012070FB00202DE9FE4F07462C200FF040F90028386100F0E68000212C2232
:20D9E00010F0B4FF38694FF6FF7585823C6938880DF1020112F0CEFBDFF8B4B168B30DF18D
:20DA0000020069461BF048FBBDF80000854224D0002006262074BDF80010BDF80030668225
:20DA2000674E8A0002EBC100A38206F1240143181A68A2611A68521C1A600E584FF47A74D7
:20DA4000B6FBF4F06043361A07D101205E46187230784FF4006114F0A5F83969388808318F
:20DA600012F098FB5348846880461CF093F868B13869002141823869682686823869022392
:20DA8000037438698461621CC8F808204A48D0F800903869DFF824A10446A18A2E468E4243
:20DAA00054D104F1080049461BF0A2FA48B91BF0C1FB014648461BF09BFA10B91CF06AF89A
:20DAC00060B13888396904F04BFD002400B1012400200CB139698D82396908743869044606
:20DAE000A18A8E4232D15146303991F82F303BBB91F86510012923D101200DF10A013A22A8
:20DB00001CF073F9C8B901209DF80A50207400233A22A5755D466382D8F80410A28228789F
:20DB2000A161D8F80410491C0129C8F8041005D14FF4007114F036F800E0A5823C692046CE
:20DB4000828A3146914204BFA1213975818A8E4224D0017C01290ED0BE6856B91CF01AF895
:20DB600020B9B878400838BF052100D30D21204602E00D2100E00E210177B87800F0030016
:20DB800001281ABF514608780520396948703C6960781BF0C7FB6077BDE8FE8F16F0FCFF99
:20DBA00000203861BDE8FE8F10203875BDE8FE8F3BFD002048040120B800012014FB00209E
:20DBC00064FE00207A492DE9F04FFF28ADF13C0D0AD148780A78824240F3E680850005EBAE
:20DBE00000156D18183503E01422183110FB0215E8884FF6FF74844200F0D680287B0028BB
:20DC000000F0D28068788DF8310000268DF83060684FADF8286038882B7BADF83200C3EB22
:20DC2000C300401C0FF016F80746287B80000FF011F80D90002F00F0B380002800F0AD800C
:20DC40002B7B0E904FF0FF0A4FF00709A3463B7050E016FB09F039183C180023A1F801B009
:20DC6000804684F803A007EB08004360287BB0423EDD2C69711C1846002C39D08642C8BF6E
:20DC80006468401C491EC0B2F6D18CB32068008807EB0801A1F801002268698868781288E3
:20DCA00008AB0EF0D7F9012822D19DF8220007EB080107EB08030422C8700E9809995860BA
:20DCC0001BF0E8FA0E909DF822001BF076FA78B1206800210422801C10F038FE9DF8220006
:20DCE0000FF02EFA024609992068801C1BF0D2FA761CF6B2287BB042ABDC95F801B0B5F8D7
:20DD000002A01CF09FF900242346804624E015FB09F0391838184078491C02F8010B088809
:20DD2000001202F8010B887802F8010B8878D1F8031009F09DFE6D1CEDB2024616E013FBE1
:20DD40000971491C8878D1F8031018F0C9FC5B1CDBB20019C01C84B238789842EFDC204651
:20DD60001CF09AFA061C18D0024600253878A842CDDC002100910120019002910391CDF8F9
:20DD80001080524605940A230696584607910AA902F08EFA30461CF0BFF9384616F0FCFEDE
:20DDA0000D9808B116F0F8FE0FB0BDE8F08FC046F00C01202CFB00202DE9F04785682A68F0
:20DDC000D16944681162490832D3D4F8C01049BB2968486820F0020048602968486A20F0A6
:20DDE00003004862D4F8CC002A6941686F69096847EA0200C862D4F8CC006E6941682A6951
:20DE0000096846EA0200C1F804052968486920F001004861286801210162284619F0D4FF42
:20DE2000BDE8F08703220A7403F026F9BDE8F087D4F8CC0041682A696F6909684FF0000990
:20DE40000226CA4647EA0200C1F80405D4F8C070002F00F0A880D4F8CC00D5F814E0406851
:20DE6000D4F8E0C0D0F80080BCF1000F04D1EA69A86904F1D80103E004F1DC016A6A286A10
:20DE8000D8F8043513EA0E0F11D0806810F0070F0DD13868D4F8D030984208D17F6937B9AB
:20DEA0002B68586A20F002005862C8F804E5906810F0070F74D10F68002F71D0D4F8D400BE
:20DEC000BCF1000F3844C4F8D40014BF48462020C4F8E000C1F80090D4F8C010D4F8D0209C
:20DEE000086890424BD8D4F8D420904247D881F81090D4F8C80004F1300730B9D4F8C010AE
:20DF0000C4F8C810D4F8C80008E04369002B34D1D4F8C0104161D4F8C01040694969C4F824
:20DF2000C010C0F814A0D4F8E00000280CBFD4F8D800D4F8DC00C4F8D000D4F8C000C4F8E6
:20DF4000D49088B12046294606F08EF994F8FE0078B1D4F8CC00406801686869D1F80425B3
:20DF6000024218BF886204E02968486A20F00300486238461CF04AF912E01846C5E7204689
:20DF8000294606F071F994F8FE0048B1D4F8CC00406801686869D1F80425024218BF8862BE
:20DFA000761E7FF453AFBDE8F08770472DE9F84F0746714D714C28684030D0F89410267856
:20DFC00091F883B026B1D0F80C0580472868403001680E6816B9D0F80C058047A046694928
:20DFE000674C0120012F88F80000D1F8009067702AD9DFF894A1654EBF1E59D07F1E52D0E6
:20E000007F1E3DD07F1E73D07F1E34D12968096C096891F86D20628191F86E70002F06BF09
:20E02000E070071CE770686840683178007811FB00F0784381005046C16690F8701021F06F
:20E040000F0141F0030151E000202E686071306C0068D6F8D410C08AC00934BF91F8250059
:20E0600091F84E00A070B7B9CF78A7B10228C4BF0220A0700FE02868D0F84C05804737E055
:20E080002868006C006890F86910617190F86A00A0700027A77109F09DFE2868006C006810
:20E0A00030BBBDE8F88F0020607117F087FB1FE030788700D9F83C00804771683C22401A3C
:20E0C000B0FBF7F0B0FBF2F15143401AC0F1780086B2D9F83C00804707FB06015046C16637
:20E0E00090F8701021F00F0141F0020180F870102748007898B92868403001680F682FB9CB
:20E10000D0F80C0580472868006C07687A686178107800F0200020719078E07100E06178FE
:20E12000032903D0022918BF062923D11CF04EF805466078022815D01648077817B916492B
:20E140000F787FB10221BBF1010F88F8001004D10078832801D113F095FE28461CF0C0F906
:20E16000BDE8F88F832088F8000028461CF0B8F91AF06CF9BDE8F88F140100200A14012016
:20E180004C020120E0FF002050180020D8000020FC13012005140120071401202DE9F041A4
:20E1A0000D4677490A680646ADF1600D14A802604A6842600A8902810A310C2268460DF0E7
:20E1C00095FC0024204603A919F0FEF98046B8F10A0F1DD0B8F10D0F17D09DF80C0031780D
:20E1E00000F0070001F0070188420ED1371D0DF11201042238461AF0ADFC48B90DF10E01BC
:20E20000384608221AF0A6FC10B9641C052CD9DBB8F10D0F02D1042C00F3AF80F220594CDB
:20E220008DF80900B4F848009DF80C70ADF80A00F80937D34FF002080DF12E0114A80A2233
:20E240008DF808801AF086FC98B90DF13601684642461BF023FA284614F070FD071C08D067
:20E26000608F69460C22B88138460DF03FFC2878B8730EA914A80A221AF06CFC90B910A905
:20E28000684642461BF00AFA284614F057FD071C08D0608F69460C22B88138460DF026FCD6
:20E2A0002878B8739DF80C00C01123D001208DF80800304611F0F8F9ADF80000284614F001
:20E2C0003DFD071C16D09DF80D00800904D2304611F0EAF9B88106E007F10C000DF1170167
:20E2E00002221BF0DBF9694638460C220DF0FEFB2878B8739DF80D0040083ED301209DF84E
:20E3000042708DF80800780819D30DF14301684602221BF0C3F9284614F010FD071C0ED0F7
:20E3200007F10C000DF1450102221BF0B7F9694638460C220DF0DAFB28780938B8739DF8E8
:20E340004200800819D30DF14701684602221BF0A5F9284614F0F2FC071C0ED007F10C00E1
:20E360000DF1490102221BF099F9694638460C220DF0BCFB28780938B87318B0BDE8F0819B
:20E3800058C10200E4FA00202DE9F04F724C002704F19800ADF1140DB946B84605680297DB
:20E3A0008246CDF80C903DB3D4F8AC00B84203D1D4F8A800B8421DD0D4F8A8600EB3D4F842
:20E3C000A8102869096988421BD195F83300400917D3D4F8AC60A6B90127D4F8A800C068DE
:20E3E00040880028F9D0D4F8A800C06840880128F3D006E0012704E004F1E00002211BF01F
:20E4000003FF002D43D087F0010B03A802AA59460CF02CFE5FEA000809D0012F07D003994E
:20E4200029B104F5AC701BF073F94D462FE0002D2DD04A48066856B3B8F1000F27D0039857
:20E4400028BBCDF800B002980190D4F8A800D4F8AC100AF108035246B047401E02D0401E1A
:20E4600008D014E0029800B9284601214B460091014605E001230093D4F8A800D4F8A810F0
:20E480000069B1F930104A4605F04EFB60E0002F5ED0002D5CD060682969884252D1B8F175
:20E4A000000F0BD0039848B1D4F8A80030B9D4F8AC0018B9082017F0BDFE49E008201AF0F3
:20E4C00047FC95F8330004F1E006C0F3001028B9504619F0F1FFC4F8A80004E0504619F044
:20E4E000EBFFC4F8AC00A8691D49C0430860A8694A6810434860E869C04341F8080CE86938
:20E5000051F8042C104341F8040CEC680820294619F034FE204619F0FBFD2088A0F6020019
:20E5200040B141F21E01401A04D041F6E671401A012803D80120214619F020FE4FF08041CF
:20E54000304603E004F1E0004FF480611BF05CFE05B0BDE8F08FC04630F500205C0501205E
:20E56000101004402DE9F047ADF1200D109C1D4682460E469046E811002110221FFA80F940
:20E58000204610F0E3F9C5F3C307D6B104A8214610221AF07FFE2046514610221AF07AFEB3
:20E5A00004A8214617F02AFC1026224613781AF8011B761E81EA030102F8011BF6D180352F
:20E5C000ADB24846411E00281FFA81F940F09980002F72D00E2F28DA04A8214610221AF0EC
:20E5E00059FE204600210E2210F0B0F93A46204641461AF04FFE2E128020E05521461022F2
:20E60000E5736846A6731AF045FE04A8214617F0F5FB10206B46227813F8011B401E81EA19
:20E62000020104F8011BF6D187E004A8214610221AF030FE20460021102210F087F93A465B
:20E64000204641461AF026FE802021461022E05568461AF01FFE04A8214617F0CFFB102741
:20E6600021466B460A7813F8010B7F1E80EA020001F8010BF6D104A8214610221AF00AFEBD
:20E68000204600210E2210F061F92812E57321461022A07368461AF0FDFD04A8214617F05F
:20E6A000ADFB10206B46227813F8011B401E81EA020104F8011BF6D13FE004A82146102201
:20E6C0001AF0E8FD204600210E2210F03FF92F128020E573214620701022A77368461AF028
:20E6E000D9FD04A8214617F089FB10206B46227813F8011B401E81EA020104F8011BF6D159
:20E700001BE004A8214610221AF0C4FD2046414610221AF0BFFD04A8214617F06FFB22461D
:20E720000021137818F8010B491C102980EA030002F8010BBFF645AFF3E708B0BDE8F087A9
:20E740002DE9F04F09AF3D7AD7F804800E1C9A4693460446ADF12C0D26D0207A29098DF857
:20E76000260010D302281FD121881BF09FFB884209D008460322012111F05EFF002818BF93
:20E78000CD2040F0C180237A022B07D00F2B05D0032B0DD0012B0BD033B909E0208816F0D6
:20E7A0009BF918B90F2B03D10220ADE00F2323728DF80830032B1CBF2088ADF8000003D189
:20E7C000684621461BF0E8FCA8081DD250484FF000090368ADF8109043B15868864203D0B7
:20E7E0001B68002BF9D101E09A681AB9B3688BB158880DE031780220904758B10188ADF8EE
:20E80000101016F0C9F905E04FF6FF704FF00009ADF810006809ADF818900BD39DF8080041
:20E820000F2807D0012805D0BDF8180040F00400ADF8180035F07F0005D0BDF8180040F098
:20E840001000ADF81800E80938BF484606D3BDF8180040F00100ADF8180001208DF8250016
:20E86000E80805D3BDF8180040F04000ADF818008DF82490A80934BF012004208DF81B0014
:20E88000617A8DF80B10ADF80EB0ADF812A03D68059598F800008DF81A00397B8DF81C1070
:20E8A00030788DF80A001AF0C3FA18B1016909B16846884709A815F0DDFA504508DA15488F
:20E8C0000168002908BF022706D06846884702E06846FEF77BFF07469DF8080002280CD173
:20E8E0001BF0E4FABDF80010884206D1307898F800105A463B4617F0F9F827B998F80000F8
:20E90000401C88F8000038460BB0BDE8F08FC04624050120B40001202DE9F8430646307B51
:20E92000894603461AF02CFB0125041C5DD1D6F8008077891C461C200EF08CF950B1002189
:20E9400041730473478101818173C173C0F8008041614160041C00F0C08000270781307CF4
:20E960002074708A6082337C23BB716911B30F460E200EF06FF9E0B1394691F838200270B0
:20E9800091F83920427091F83A20827091F83B20C270CA8F8280B1F84020C28091F8422067
:20E9A000027291F84A2002734A88428191F849104173074638466061308B20836189B07E4E
:20E9C0004FF67F472E46A07607EA0100C108608107D244490A78802707EBC2110843608186
:20E9E00004E0608940F08000F9E700266089DFF8F880B9F1000FC0F3C21224D10AB38109E0
:20EA000011D2410909D2C00838BF281C10D31BF038FB00F02000801C0AE01BF032FB00F00C
:20EA20000F000A3004E01BF02CFB00F07F005F3020810420474660733878202113F0B2F8B6
:20EA400017E0002515E0022060732068C089C00803D3404634300088208152B160894FF6FD
:20EA60007F414FF680770140618107EBC21001436181012E32D1667B27893CB3012E0AD0D2
:20EA8000042E02D0022E0BD020E0042019F060FC062805DB1AE0012019F05AFC082815DC35
:20EAA000667300202781114960600868002808BF0C6003D00146486830B94C604046007873
:20EAC000202113F06FF809E00146F4E7606908B116F062F8204616F05FF800252846BDE8A3
:20EAE000F883C046C1FE0020E4FA0020380501202DE9F04F0C4606460D220021ADF1640D08
:20EB000014A80FF023FF10220DA821461BF066F94FF0010A002840F0CE8096F82600032891
:20EB20000DD196F840000EF095F8051C00F0C38096F8402006F141011AF0ACFB00E000256D
:20EB400096F825004FF000088DF8440040B1022808D112A806F1180108221AF09BFB01E089
:20EB6000F06A1290726B404611A914AB13F0C1FE96F82500002808BF062403D002280CBF67
:20EB80000324022496F82610009196F82710019196F829100291C146CDF80C9096F82820E4
:20EBA000034618A8414617F02FFC834696F82600241DE4B2032805D0022833D196F8400043
:20EBC0002418E4B220460EF045F85FEA00082CD0074607F801BB9DF8600007F8010B96F8DF
:20EBE000250038B102280CD1384606F1300152467F1C04E0384606F12C0104223F1D1AF015
:20EC000049FB06F13401384604221AF043FB96F82600022806D196F84020381D06F1410167
:20EC20001AF038FBB8F1000F03D1002D43D0A8463EE004A81BF048FA14AF0D230A940DA880
:20EC4000089706F13C028DF8303096F82610CDF814801B4C049004270992032904F13403C5
:20EC600018688DF8317016D10695079596F840100B9104A91BF054FA38B996F8402006F17A
:20EC8000410029461AF006FBCA46284615F084FF606B96F8261002290AD1CDF81890CDF8EC
:20ECA0001C90CDF82C9004A91BF03AFA00B9CA46404615F071FF504619B0BDE8F08FC046EE
:20ECC000D4DB002090B50446E08948F20601ADF1240D814211DB81421CD0133800F0AB8099
:20ECE0001939401A5CD0401E51D0401E00F09780801E21D0401E16D0ADE01A31401A00F063
:20ED00008480401E78D0401E6CD0123860D0801E55D0A0E0204617F07BFD011C00F09B80E5
:20ED20004E4B40203AE0204617F072FD011C00F092804B4B202031E06846002118220FF0D6
:20ED400005FEA06910F8011B8DF800109DF800704278017801EB0221ADF802101FB9C01C3C
:20ED600001A90DF019FC61883E4B10206A4618F0CDF8039818B115F00FFF002003900598F1
:20ED8000002868D015F008FF0020059063E0204611F0D8FA011C5ED0334B02200F4606E0B0
:20EDA000204611F0CFFA071C55D001202F4B61883A4618F0ABF8384615F0EEFE4BE0A06989
:20EDC0002B4B007807AA8DF81C004FF480003FE0A069284B00780DF11B028DF81B004FF41F
:20EDE000801035E0A069244B00780DF11A028DF81A004FF400402BE0A069204B007806AA9B
:20EE00008DF818004FF4005022E0A0691C4B00780DF119028DF819004FF4804018E0684678
:20EE2000002112220FF092FD204669460BF08EFD144B04200BE0684600210C220FF086FD67
:20EE40002046694619F05AFB0F4B4FF080706A46618818F05BF809B090BDC0465120020043
:20EE6000F51F02005BBD01002D1402008F140200DD6E0200AD6E02003D6F02004D6E0200A6
:20EE80007D6E0200E18A01008D4102002DE9F04F07467E6931780120ADF13C0D00EBC10063
:20EEA00080B21BF0F9F95FEA000808BF002000F0CB80307800254FF08F0B4FF0860A88F8BB
:20EEC000000041E06A00B018B0F8010008EBC504641CB21820803968B2F80120087D89888E
:20EEE00008AB14F039FE01282AD19DF82710C80909D2002031F07F0318BF01207A68C2F336
:20EF0000C00282421CD1480817D33868490900F1060909D3007D1AF02DFF031C04D0484642
:20EF200008A90122984700E00020A0709DF8261040B9E1700A98606004E084F802B001E0A4
:20EF400084F802A06D1CEDB23078A842BADC3968087D7B688D888E1D00240D9697F80AA07A
:20EF60000C90464631780E95D808254680F0010000F0010B19E0EA00B018B218D778E41CA1
:20EF8000A4B2401C7FB94168641CA4B229B902880E990C9818F0B8FF02E0C07817F0A0FBD6
:20EFA0003178001984B26D1CEDB2A942E3DC20461BF072F95FEA000942D00746002527E0CE
:20EFC000E900701871184978401C07F8011B0188091207F8011B817807F8011B8378ABB9CD
:20EFE000C17807F8011B416859B90BA9009102880E990C983B4618F061F8BDF82C003F18CE
:20F0000004E0C0783A4608F033FD07466D1CEDB23078A842D4DC00200090CDF804B0012328
:20F0200002930390CDF810A00594CDF8189007930E9A0D990C9801F03BF948461BF06CF87F
:20F0400030461BF069F801200FB0BDE8F08F70472DE9F0410D4680460E220021ADF1200D97
:20F0600003A80FF073FCA86A417811F01F0F18BF002040F0BD80880924BF01208DF81800E7
:20F0800031F07F001CBF01208DF81700C80924BF01208DF816009DF816200024012A03D0DB
:20F0A000287A00B1AC6902E0E87900B16C6934B10DF10E0021461BF06FF89DF81620A98958
:20F0C000012AADF80C1020D14B4A5778167F27F00100064300F08B80002F00F08880022FA6
:20F0E00004D11AF0D1FE884240F08180688915F0F3FC00287BD144B11AF09CF801460DF136
:20F100000E0019F075FF002871D03C4E96F83200800815D39DF81600012811D0BDF80C10BB
:20F120001AF0B2FE88420BD09DF81700012807D008461AF05BF818B1BDF80C0016F05CFB32
:20F140009DF81600012821D0BDF80C101AF09CFE884211D19DF81700012808D02848007834
:20F1600000F00700022807D101208DF818009DF818000AF07DFF35E09DF817209DF81830F7
:20F1800008460DF10E0107F051FE2BE000249DF818008DF81A40E0B99DF8175007461AF027
:20F1A000BFFC96F84A00082818BF042811D14FF6FD70ADF800001AF03DF801908DF80940B2
:20F1C0008DF808708DF80A508DF80B4068460DF005FB9DF818000AF04BFF52200DF11A015C
:20F1E00016F01AFA0748016809B103A88847404608B0BDE8F081C046ACFE0020E4FA0020E7
:20F20000E41201208CFD0020F0B50C460546A9792068ADF1440D40EA01406979206040EA5C
:20F22000012029792060084310F0070F206015D000F00701022920D14FF0FF30606005F18D
:20F240000801082204F108000FF0C5FE04F1100005F1080101220FF0BEFE0DE0201D05F1BA
:20F26000080104220FF0B7FE04F10800FF2108221BF014F8FF202074206841097AD2410932
:20F2800011F0030F18D001F00301032914D0012918BF022922D104F11100FF2108221AF0F5
:20F2A000FDFF4FF6FF7005F108010222608304F11C000FF090FE10E004F1110005F1080105
:20F2C00008220FF088FE04F11A0005F1080102220FF081FE4FF6FF70A083206800093ED356
:20F2E00004F11E0005F1080101220FF074FE206805F10806C10B3CBF4FF0FF31216206D34A
:20F3000004F12000314604220FF065FE2068000C06D204F12400FF2110221AF0BFFF05E055
:20F3200004F12400314610220FF055FE2068410C3CBF4FF6FF71A18606D304F13400314694
:20F3400002220FF048FE2068800C38BFFF200ED304F13600314601220FF03DFE2EE04FF0ED
:20F36000FF312162FF20A0774FF6FF77A78684F8360023E000252846694618F025F90A286D
:20F380001CD00D2817D0276817F0070706D10DF10600211D042219F0DDFB48B9022F0AD194
:20F3A0000DF1020004F11101082219F0D3FB10B1684619F084FB6D1C052DDCDB11B0F0BD6E
:20F3C0002DE9FC4F83F0004301E02DE9FC4F1F03FF0847EAD2574FEA42284FEA43095FEAE0
:20F3E000595906D147EA080A1CBF00210020BDE8FC8F57F000575FF4E06E1EF1FF0EF14564
:20F4000005D14FF00000190D0905BDE8FC8F002B05D55FF0000AD8F100086AEB07070C03D2
:20F42000E40844EAD0544FEA40254FEA4106760D08D144EA050A19BF00210020191C101C5D
:20F44000BDE8FC8F44F00054764504D10020090D0905BDE8FC8F002904D55FF0000A6D42E6
:20F460006AEB0404B6EB090E08D5A2463C465746AA464546D046CEF1000E4E46BEF1360FAD
:20F480005CBF4FF0000B23E0BEF1000F04BF4FF0000B1AE0CEF1390ABAF120092EBF08FA7A
:20F4A00009FB07FA0AFB4BEA080BDEF1200A07FA0AFA38BFBA4647FA0EF72DBF28FA0EF8AB
:20F4C000AEF1200E4AFA0EF8D04415EB08057C4154EA050A02BF00210020BDE8FC8F002C8C
:20F4E00058BF4FF0000A06D55FF0010A5FF0000E6D426EEB0404A6F101066D006441FAD58B
:20F5000015F4806E11D005F480794BEA090B15F5806554F1000428BF761C0BD205F40079D8
:20F520005BEA090B08BF25F4006525F4E0656D0044EB0404B61CDEBF00210020BDE8FC8F4B
:20F540005FF4E06E1EF1FF0E76450AD34FF0000013F00043FF21C900C91D09051943BDE8F3
:20F56000FC8F270547EA1530210B41EA065141EACA71BDE8FC8F704767492DE9F04705461B
:20F580000878ADF1580D002800F0C280A878884610F007008DF844000FD0022840F0B8805F
:20F5A000A96812A808221AF079F8A96801F10800A86090F800A009310EE0A968CA780878A5
:20F5C0008F784E784FF0000A00EB0260091D00EB074000EB062012900846491CA9604C1C99
:20F5E0000F460678AC603C78E32E18BFF32E05D19DF844101298084340F08A8004F1180074
:20F6000080B218F06AFF071C00F08280FF2C08BF002487F810A04FF0010987F80390A96881
:20F6200007F1170022461AF039F8BC75381D11A90C227E741AF032F8484616F01BFBB874AE
:20F640000520387000267E70A878000903D3F87840F02000F870314CAA8804F13A01D8F8F3
:20F6600010000988914215D011A869460DF1520210F06CFB60B99DF80000800808D3694650
:20F68000087800F0FD000870BDF8520013F0CEFEBE7038E010B18047002839D088F801909F
:20F6A00011A8694614AA10F051FB60B99DF80000800808D26946087840F002000870BDF83A
:20F6C000500013F0B3FE87F8029094F83C1088F80410A8790B30814215D0114E306A1AF0A2
:20F6E000A0FB40B9306A41F288311AF005FD06F1BC001AF08DFDA87904F13C010B30087097
:20F70000E12015F089FF07480078394613F0C4FF16B0BDE8F087C04620040120E4FA002024
:20F72000481900209C0301202DE9F043002407460C22ADF1340D214668468DF814400FF0D4
:20F7400005F9624DDFF88881B87804281DD001280BD0062809D0022805D003281CBFB320F0
:20F760008DF8140014D11B2010E0687858B91AF055FD40B9B9684646082206F11C0019F0A7
:20F7800089FD38883080232000E022208DF804009DF81400002840F086803888BE7BADF8E0
:20F7A00000003B698DF805607A7B0293012A14BF012021208DF80200684605F06DFE9DF8A7
:20F7C000140000286FD10398466C05233370B8787070796829B9B01C214610220FF0B6F8B0
:20F7E00003E0B01C102219F055FDB8781236012812BF0628F87806F8010BB96830461AF012
:20F80000DFFAB8780836042806D0012804D006281CBF387B307004D1AB202146324613F0C4
:20F82000A3FE388815F058F910B103980421C1829DF81400002836D1B878042809D038699F
:20F8400018B9684615F0A8F82DE068460CF032FD29E0B8680BA906AA0EF0FAFF06469DF839
:20F860002C0018B94FF6FF70B0421CD038694FF0010918B9684615F08FF802E068460CF078
:20F8800019FDB96808A8082219F004FD8DF8289020468DF8294031461422079006AB069031
:20F8A000042016F0CFFE687850B91AF0B7FC38B946462146082206F11C000FF047F8348098
:20F8C0009DF814000DB0BDE8F083C046ACFE002070020120F8B5694C21680546143108685C
:20F8E000407F002800F0C880D1F8C000B5F84220C08C904240F0C080D1F8581305F1280071
:20F900008847002800F0B880206840690026467721687031486E90F8290028B16068816A97
:20F920000220884721687031086890F82B0018B16068816A01208847287C400908D360688D
:20F94000816A102088472068D0F82813802088476068C16B202088472168C868D1F8FC142E
:20F96000103088476868226841785269007800EB0120C0F30321517622685269C0F3003759
:20F9800097762268526900F00F03C0F3031793772068D0F8D40080F82C7022680C32D2F872
:20F9A000C81091F84F000F2806D093689B7F984202DD6B68DF780FB19068807F48731068A8
:20F9C00080F83060D2F8C800417B0F290BD19068C07E022850D1D2F8580180472068D0F802
:20F9E0006C018047F8BDD2F800252846904723680C339868C07E022815D1D3F8F014186883
:20FA000088472268D2F8D4001169467BD06831F81630D2F8F0244FF4707707FA06F1C91A2A
:20FA2000904723680C33D3F8C8002A89D3F8A83190F82C1002209847206800F11401D1F81F
:20FA4000C020D0F8D400527B90F82C0082420FD00868D1F8E81488472268D2F87C01516977
:20FA6000886050694169D2F8F024904721681431D1F8141310208847F8BDC04614010020D9
:20FA80002DE9F047634F8046381D0068416EADF1280D02A888475B4D2A684032106800685D
:20FAA00020B9D2F80C0580472A68403256484FF001096E6880F80090F068007830B9D2F87F
:20FAC00018244846002190472A684032106801684C68088921788246C1F3401109F096FF46
:20FAE000079011F0B7F8494E746786F873A00024A6F866401AF06AFB059482463146B8F164
:20FB0000010FA6F8664004BF4148C1F8B80038F001083E4654D1A1F89E4001F16400C1F874
:20FB2000A00091F8A90002231A4602F00F0220F00F00024381F8A92091F8A80004F00F078A
:20FB400020F00F0047EA000291F8B3708C6627F00F0081F8A82040F0040009F00F0291F887
:20FB6000717081F8B30027F00F00024381F8712028684030006800684268127801F16407A2
:20FB800092090FD301F120028A66406891F87150807803F00F0381F82E0025F00F000343E4
:20FBA00081F8713001F1100001F19C0242604A7F04F00F0322F00F0213434B77014601E0C5
:20FBC00064310F467068174A056D08238DE81800114B106802AAA84710490028088006D486
:20FBE0000F4991F90000B760401C087004E0484641F2883111F05AFA50461AF071FC0AB0BE
:20FC0000BDE8F087140100200F05012050180020801A0600DCFF002045BA000028050120EE
:20FC200012050120800001202DE9F8430D4606466868002800F0C580007819F04DF90028DF
:20FC400040F0BD8019F0DAFB052880F2B6804FF00008304685F8018019F030F9041C01D0A6
:20FC6000207B60B11C200CF0F5FF041C00F0AB8041461C220EF06AFE2671012600E046461C
:20FC80006868007820736868007A504F2076142027610CF0DFFF0028606141D041461422BD
:20FCA0000EF054FE6968626949689079897900F0F00001F00F010143917168684068616933
:20FCC000808888806868406861690078087068684068616940884880686840686169C07995
:20FCE000C871686840686169007B08736069C07940000CF0AFFF616988606769B86818B13C
:20FD00004046F97981424EDC387B40000CF0A2FF3861606907691FB14146027B8A4238DCE8
:20FD200004F10C00814608F00FFE0746022F18BFB82F06D1207B13F0B9FD484608F004FE07
:20FD4000074637B9012E1FD1204615F05BFFC0B11AE0012E15D0606968B1816819B1084620
:20FD600014F01AFF6069016919B1084614F014FF606914F011FF4846414610220EF0E6FDFF
:20FD800002E020461AF0C0F9022F18D0B82F16D019E06B685B684A001B690069D35A13521A
:20FDA0006069491CB9E76A68526841009268BB688A5ACA526769401CA3E7D12002E0D02012
:20FDC00000E0022068700120BDE8F8832A1A00202DE9F04FDFF898910646A9F1080000F170
:20FDE00008078068D0F80001807AADF12C0DC0000CF030FF0028089008BF1A2500F0B4809D
:20FE00001AF0E4F900244FF0FF0B25460A9027E0ADF800608DF80240D2F88823D0206946A2
:20FE20009047D8B99DF80C00012802D19DF80B1019B998B99DF8071081B1002814BF0823E6
:20FE400004230DF103005B1E00F801BBFBD105703868D0F894246946D0209047641CE4B260
:20FE60003A6802F580721068C07AA042D0DC4C462068D0F80001C0884FF6FF78AA461DE0E3
:20FE8000089901EBC0018A8896421CBF401CC0B261D1C1F800A0A1F804803A68D42004A996
:20FEA000904702E07F1CBFB225E020682268D0F800016D1CEDB202F58072C088A842D8BFC3
:20FEC00055464BDDADF80060ADF80250D2F88823D120694690470028E7D1BDF80400804519
:20FEE000E3D0ADF810002068D0F8882404A9D420904790BB5746226802F580721068C0880B
:20FF0000B84210DDADF80060ADF80270D2F88823D120694690470028C4D1BDF81000BDF8BB
:20FF200004108842BED12068D0F80001C088B842BBD1ADF81480ADF8168006A8594608224A
:20FF40000EF004FD2068D9F8003000F29447D3F80001837A5046834292DC19250A981AF0D0
:20FF6000BFFA089814F018FE28460BB0BDE8F08F140100202DE9F04F654CE768ADF1140D78
:20FF8000002F00F0C2804FF0000A5046039094F8028004903DE094F8028035E00A200CF086
:20FFA00059FED4F80C80071C00F0AF8019F0BBFB0BEB0800808805EB080104220E31388075
:20FFC000B81D19F067F9049D3A88029948466B460CF040F8012808BF0125284604F11805DC
:20FFE00020B10199B81C042219F054F9B000394600EB061040190C3015F02CFB012800F03C
:020000040001F9
:200000008480204690F80280E7680AF101005FFA80FAD04579DD16201AFB00F5E919785DCC
:2000200049888146029116F087F9AB460646FF2EB4D12278002F8C46E7D004984FF6FF7678
:20004000B646014615E0162310FB03F5EB197D5DA9450CD15D88AC4509D1DD88AE42C8BFF7
:200060002E1C1B89491CC9B29E45C8BF9E46401CC0B28045E7DC0029C7D0042A45DC90006F
:2000800004F11805634600EB0210291881F80190DDF80CC04B8007198E80521CA1F806E0D6
:2000A00007F11803A1F808C066461E6131461973D7B229540A2027700CF0CCFDE668071CA1
:2000C00023D019F030FB06EB0B018888042238800E31B81D19F0DEF83A88029948466B467F
:2000E0000BF0B8FF012804D10199B81C042219F0D1F82178880000EB0110401939460838B5
:2001000015F0A8FA01287FF446AF05B0BDE8F08FF00C01202DE9F04160485F4E614C604DBB
:2001200070601030B06004F14400B0E88C1005F17C01A1E88C108DC881E88D00182204F120
:20014000140705F1340039460BF0D0FC1822394605F14C000BF0CAFC05F16407182238463F
:2001600004F12C010BF0C2FC95F870003C2204F1840140F0800085F8700005F1BC000BF085
:20018000B5FC95F8CB100120024602F0010221F001010A4385F8CB2095F8CB1060F38201E2
:2001A00085F8CB1095F8CB1021F0200185F8CB1095F8CB1060F3C71185F8CB1004F16401B0
:2001C000B1E8085105F19C02A2E8085191E80A5082E80A50C5F8A07095F8A81060F3C711E2
:2001E00085F8A81095F8A91021F00F0141F0020185F8A910042385F8AD30052185F8AC1019
:2002000095F8AE1000F01F0221F01F010A4385F8AE20032185F8B01095F8B31000F00F0207
:2002200021F00F010A4385F8B320B4E8841005F12001A1E8841014CC81E8140095F82C1076
:2002400060F3C71185F82C1095F82F1003F00F0321F00F010B4385F82F3095F82F1060F37F
:20026000C71185F82F1095F82D1000F00F0021F00F01084385F82D004FF4586028630A4833
:20028000F0600A4800684069007808B10CF056FC0AF0A4FDBDE8F0817000012038FA002098
:2002A000501800208CB4020068050120180100202DE9F04F09AF9A4690468146ADF1240D54
:2002C000B7F814B0BE89069119F0ECFC0028079008BF022000F0B38019F054FD0446E00984
:2002E00008D259481830056825B1687E012808BF44F0400404A80021082219F0CFFF3D7827
:2003000035B904A90868002220F00300086006E00498012220F0030040F001000490079819
:2003200085683DB16888534641460090484615F0D5FD08B9012082E0002E04BF0498C0F359
:20034000800607D004A90868ADF81460012640F0040008603D7925B904A8016821F0080184
:2003600003E004A8016841F008013D7A016025B904A8016821F0100103E004A8016841F0F5
:2003800010010160387C8DF817A0002E8DF8160014BF05200320584480B2814619F07CFFFE
:2003A000061C4AD0049901F003010170049AC2F3800241EA8201C9B20170049A02F00802F5
:2003C00011430170049A02F01002114300F8011B0499C90808D39DF8141000F8011BBDF883
:2003E0001410091200F8011B9DF8161000F8011B9DF8171000F8011BB9695A4619F04EF9F9
:20040000387F68B90F480096811C01910294007803900799069842464B46FEF791F907E08A
:20042000009601940698079942464B4608F072FE0446304619F070FE00E01024204609B068
:20044000BDE8F08F800301208003012001282DE9F84F40F0B080DFF88491D9F8340101282F
:2004600040F0A6800220C9F8340118F01DFC012015F070FC5FEA000805D00120C9F834011E
:2004800018F020FC99E0112019F052FD00280CBF00250125102019F04BFD08B145F0020582
:2004A0000F2019F045FD08B145F00405444CA06A0068014601208847012805D099F83801CA
:2004C000012818BF002703D1002004F021FD012719F028FDDFF8ECA040080AD20026206A62
:2004E00080680146504688478346BBF1040FF6D000E00126304600214FF0FF3202F0DCF846
:20050000012E0ED0BBF1010F05D1206A4068012102465046904732496C39086840F0030070
:200520000860206840690146284688470B2019F0FFFC254E30B12068C06A3146091D024684
:20054000088890470A2019F0F3FC28B12068C06A31460246088890471C4903200124C9F8F3
:2005600034011B4E0C6000233360284613F048F80128FAD1174D2868042015F0EBFB0646C7
:20058000154804602868012F02D1204604F0C0FC19F09EFC082015F0DDFB0746C9F83441C6
:2005A00018F090FB57EA060018BF4FF0FF3804E06FF0040801E06FF001084046BDE8F88FCA
:2005C000B8010010004003401ABD0200282008600C2008402C2009400C4009401015002063
:2005E00090220840F8B5074661485F4C001DC26A0168B7F5C067C2F30722C4F81071C1F35F
:200600008441C4F81421C069C4F81811C0F38120C4F8280100F0A38094F830616EB9C4F8CA
:200620002C71D4F81801C4F82001D4F81461C4F81C61D4F82851C4F82451D4F82C01D4F8A6
:200640001451002854BF02236FF0010304F59072116800EB4000C018431000EB937001EBCE
:20066000A0011160D4F82011C4F81C5100291CDD1E293DDDD4F8240130B93429B4BF1539C7
:200680001E21C4F8201125E02A29BABFD4F820010B381E20C4F82001D4F81C013E28D4BF30
:2006A000401C3F20C4F81C011FE0D4F82401032812D011F10A0FA6BFD4F820010B300120E0
:2006C000C4F82001D4F81C010028CCBF401E0020C4F81C01032009E011F1140FA6BFD4F8E8
:2006E000200115300120C4F820010020C4F824014FF08057D7F8A401B4F81C111B4D406822
:200700004FF47F4208230646009128463021B047D7F8A40101214FF400321123406800919F
:20072000064604212846B047D7F8A401B4F8201140684FF4F8021223064600910421284608
:20074000B047D7F8A401B4F8241140684FF440620A230446009120212846A047F8BD00204D
:2007600084F83001F8BDC0461015002000A00C4000A00C402DE9F8435F4CDFF868815B4D90
:20078000D4F83C0100286ED0574E401E0AD0401E60D0401E1CD0401E53D0401E1AD0401E0E
:2007A00033D02FE04E4801250221006884F83A517022042340680091002107464046B847F4
:2007C000356004F1500019F0F7FC2846BDE8F883022100E003214FF08059D9F8A40184F884
:2007E0003A1140680025702204232946074600954046B847D9F8A401C0687022294613465A
:200800000125DAE70320BDE8F88300262E606E6028688008FCD268688008FCD23748344924
:200820000127001D06600E200F6008F057FE022016F044F9C4F83C6184F83B610220BDE886
:20084000F8830520C4F83C010027376030688008FCD242E00320C4F83C01002737603068BF
:200860008008FCD239E0234F01260F202E6042F62A21C7F80B004FF08059C7F80F10D9F89F
:20088000A40140684FF4C072072302218446404600910021E047D9F8A401C06800214FF41E
:2008A000C072072384464046E0472E6028688008FCD394F83901C7F81B6018B903210020DB
:2008C0000E4602E0002028630321C4F83C6147F8011C686068688008FCD20020BDE8F88330
:2008E000A401001000A00C4058600C4054600C4004800C4001400C401015002038500C40DD
:200900002DE9F0410D46044602220021ADF1480D11A80EF01BF800263046694616F054FE4E
:2009200007460A2F00F0AD800D2F32D094F825809DF8000008F0070100F00700884227D157
:20094000B8F1000F0BD104F12C000DF10601042218F000F918B1E06A6860002015E0B8F11D
:20096000020F16D104F118000DF10201082218F0F1F870B105F1080004F11801082218F0F7
:200980008DFE94F83000287402208DF8440005E00227761C052EBFDB002F72D19DF8000015
:2009A0009DF844709DF801609DF80D30C11007F007009DF845209DF80D7001F018010143FD
:2009C00006F0010094F8296041EA401103F00300002E41EA80118DF8441002F0F800C7F332
:2009E000820141EA00018DF8451007BF9DF8450000F0F7009DF8450040F008008DF845000B
:200A00009DF84510676B94F838602A8841F050016F619DF844002E7601F0DF0110432880A9
:200A200040EA0120288094F840008DF8451050B1687619F031FCE86128B194F8402004F105
:200A4000410118F02BFE104894F9151000880829288405DC11F16D0FB8BF6FF06C0100E032
:200A60000821A77D6E3148B2002F4FEA60010CBF00220222C8B285F8220040EA821085F864
:200A8000220012B0BDE8F0811EFB00202DE9FE4F5B4C5C4994F83C80B4F848500A688346AD
:200AA00001A8026049684160DFF85CA101A80AF11409494618F09CFA00280CBF01260026D7
:200AC000A76887B11EB93888854206D008E007F10C00494618F08CFA10B1B878804502D00A
:200AE000BF69002FEED1002F08BFCA2000F0858039894FF6FE70884208BFC3207DD019F0CC
:200B0000D5F9884208BFC22077D03888A84218BFA4F8480017F094F9F87A4946401C84F87B
:200B20005C0004F15D0019F037FB02208DF80100684617F069FD04F12405061C58D0306908
:200B4000062100F8011B94F8321001704FF0010986F81E9018F06EFB706286F81A904020DB
:200B6000F0823889708086F818B03046FBF784F8061C3ED1092084F84A003B89E38794F84E
:200B80003C00804518BF84F83C8005F11A014B2014F042FD05F12401502014F03DFD05F1C7
:200BA0001801E12014F038FD05F11601532014F033FD082049460AF063F94FF4005000216D
:200BC0000AF05EF920784FF4806111F0A9FB0F480078022804D008200FF0C2FC820001E04E
:200BE0004FF4DC6220784FF4806119F0B4FA00E0102600208AF805003046BDE8FE8FC04696
:200C0000E4FA0020E0B8020034FD0020ADFE00202DE9F043054603200C46ADF1340D8DF8B3
:200C20001E000DF1160019F0B7FA18F003FB01460DF1160018F0DCF9002800F08980207DCC
:200C4000032818BF012840F08380277A002F7DD0FE2F7BDC032804D1A07D002876D0FE28E4
:200C600074DC45490A6809A8026049684160DFF80C81082209A908F10C09484617F004FDDB
:200C800028BBAE1C3E483188008888421FD040460178FF2909D0B94207D040884FF6FF71D8
:200CA000814202D06189814211D100208DF808004946082203A818F0EDFA02A80FF026FD44
:200CC0003088BDF80A10884218BF8D2042D12D48EB890768AE1C212B11D02B48076867B1E3
:200CE000207A6189A37D04F10C02B84728B900208DF82C0016F0B4FF2EE088202AE08C2077
:200D000063898DF82C00ADF822302FB30DF122000090A27D207A04F10C010123B847D8B146
:200D200000278DF82C7016F09BFF207D032813D104F10C0008A915F019FE04F10C0858B937
:200D4000394640460A4610F0F5FC05E0822000E08420AE1C8DF82C000BA80090287C01904F
:200D6000EA893146012305F1110042F4004213F07DFC0DB0BDE8F083B8C3020094FF002065
:200D80001EFB002000030120BC0001202DE9F04F0446E078ADF11C0D400810D304F1130028
:200DA000FF2103220DF0D2FD012001904FF0000903902079CDF8089030B1022801D00120A2
:200DC00099E00820009005E00427E078009700F0DF00E0704F464A48039E0497C8460597B7
:200DE00000F1100B069660E04FEA88005BF8007000EB0B0A002F52D025793E79B5424ED1CB
:200E0000009A07F1080004F1080117F03DFC002845D0A3785BB9022D06D1E078800903D3D1
:200E2000387C217C88423CD1069F02970FE0DDF818903EB1E078800906D3387C217C88421C
:200E400002D02EE04F460297B9F1000F24D0042017F043FB071C1FD00498787006263E70FE
:200E6000DAF80000807CF870DAF8000017F01CFC0598B9F1010FCAF800001CBF0420B8700B
:200E800005D10698B870059E0396CAF800401B480078394612F000FC029810B12AE0CDF8F6
:200EA000048008F101005FFA80F8B8F1000F9BD0029D45EA0905012D1CD0042017F00DFB97
:200EC000011C17D0059806224870019F0A70A27CCA7057B9A078012818BF042005D138467F
:200EE0004BF82040059A0392022088700348007812F0D2FB039807B0BDE8F08F9C03012039
:200F0000481900202DE9F84F534D2968D1F8D40090F883A040310868006820B9D1F80C057E
:200F2000804729684031886F4C4EDFF83491DFF834810078E8B919F049F9377883464FB94B
:200F400049460F7837B9832041460870584619F0C7FA60E002214046BAF1010F017004D197
:200F60003078832801D110F08DFF584619F0B8FA65E014F023FC3C4800683C4F016C38687B
:200F80008847044619F022F9824630460778002F44D149460F78002F40D12868D0F8B800AD
:200FA000C16C002088472868D0F828246946F42090479DF90000A0421EDC2D4CA079D8B942
:200FC000504619F08DFA6078042803D02868D0F84C05804704204146A7792E680870781C37
:200FE000A071D6F8B800C16C09B103208847032060810FF0C7FD22E08320414608700020F6
:2010000015F09EFA504619F06BFA1A486968C01D09690078087017F019FA10E00222414608
:201020000A700078832801D110F02CFF504619F057FA2868D0F8B800C16C04208847686826
:20104000C068007828B92868D0F85824002001469047BDE8F88FC04614010020051401205C
:20106000071401200A140120E0FF0020800001204C0201204D0201202DE9F0410646746807
:20108000B56819F0A3F8D4F8C0108046002900F0A18094F8F80028B9087C032818BF0428DC
:2010A00040F09D80287919F093F8D4F8CC0041686F690968CF6294F8F90018B92968C868DC
:2010C0004009FCD22968486820F002004860D4F8CC0041682F690968CF622968486A20F030
:2010E00003004862D4F8CC002A6941686B69096843EA0200C1F804052968486920F00100E6
:201100004861286801270762D4F8D400D4F8C0100860D4F8D87067B1E8698068C0F3091030
:20112000401C874205D3D4F8C0201168C919091A1160D4F8DC7067B1686A8068C0F3091061
:20114000401C874205D3D4F8C0201168C919091A1160304610F00CFE287919F033F8287901
:2011600019F038F8D4F8C070386857B100230222397C03291CBF04293A743B607F69002F02
:20118000F6D1D4F8C0100860D4F8C8100022002904BFD4F8C000C4F8C80004D04869B8B9CC
:2011A000D4F8C0004861C4F8D020C4F8D420C4F8D820C4F8DC20C4F8C020C4F8C420404670
:2011C00019F08EF904F1300019F020F8BDE8F0810146E3E72968486820F002004860404691
:2011E00019F07EF9BDE8F0812DE9F0418046D8F80460D8F80050307817F0CAFC7178002773
:20120000814249D02879401E28D0801E1FD0801E012803D9001F14D0801E35D1287C10F080
:20122000120F08BF02240AD00324AA69E96928682C71891A18F0BEFF286818F0BDFF2C71B4
:2012400022E0287C800928BF20270A201DE00421287C2971800828BF022717E019F044F9D2
:20126000297CA860480828BF012711F0120F0BD00322AB69E96928682A71C91A18F09AFF2B
:20128000286818F099FF01E0022028717078002850D0012851D055E02879401F26D0401E7F
:2012A00017D0801E08D0C01E3ED10721287C2971C00828BF042739E0A86818F0BFFB297C14
:2012C000E860C80828BF0427080928BF47F008072AE0A86818F0B2FB297CE860480928BFB2
:2012E0001027C80828BF47F004071DE0287C80090ED2A86818F0A2FB07212971297CE86050
:20130000C80828BF0427080928BF47F008070DE00822AB69296A28682A71C91A18F04AFF90
:20132000286818F049FF01E007202871707820B1012807D14FF4A02101E04FF4C0213078C1
:2013400015F074FF2FB1686918B10246394640469047BDE8F08170472DE9F043584C94F831
:201360004201ADF1140D002840F091804A484B4E4FF00108027B3368416884F842818146C8
:2013800084F84121C3F38147C4F86C11BFB9D9F81000A0B156F8085C18F06AFD6421024620
:2013A000C5F306604143B1FBF2F23D49002304F1940013F031FB3B494FF00040086001A886
:2013C00018F04BFE00252F4604F10C00029501AB8DF80470344903953A4613F01DFB01A88C
:2013E00018F03BFE04F150000822029501AB8DF804702E49039513F00FFB2D4A04F1D800A1
:2014000032213B4613F0C6FE2B4A2A4F04F1F4002C212B463D6013F0BDFE306899F80D30DB
:20142000C0F381501BB1032803D184F8398103281FD002281DD001281BD14FF08059D9F8F8
:20144000A4011E4C406803214FF040521C230746009129462046B847D9F8A4014068294662
:201460004FF4007209230746CDF800802046B84706E0386840F040003860022015F036FBAE
:2014800056F8040CC00802D2284615F02FFB05B00020BDE8F083C046FCC10200B44F0050B0
:2014A0006595020000A10C404F510100553D0200917E02009022084095F2010000A00C408F
:2014C000101500202DE9F04F044608469A46ADF1240D214605908E680692129B04914C68AB
:2014E000756807935044854238BF6FF00304C0F093804B4D28684FF0FF3118F008FB4948C7
:20150000328C079F48496368026083460B60780819D23846800813D3F768002F3AD03569E8
:20152000002D37D000970195012002900599069A049853460DF0ACFB5FEA000813D114E057
:201540004FF0000811E0A0683AEA00070AEA00021CBFB1680A4405990140049808F010FB6A
:201560005FEA000801D0044652E034680598DDF818905746241805E0BBF80010049818F0F2
:20158000ABFAA944AFB90798C00840D3F16809B1306910B96FF007043AE000910190002795
:2015A0000297069A0599049853460DF071FB80462DE0049810F0BCFF38BB049814F00AFFF0
:2015C00018BB04F0FF05C5F58075BD4288BF3D1C210C8DF80D1002208DF80F40230A8DF87B
:2015E0000C00BBF8001004988DF80E3018F06BFA03A8042111F0DAFD7F1B641928B9484622
:20160000294611F0D3FD0028B6D04FF0FF3844460348006818F0F0FD204609B0BDE8F08FF1
:20162000A8130120A4130120A0130120F0B50446207CADF13C0D0F28C0F2A680656860690B
:201640000DF1260210F07AFC9DF82600002840F09B80207C0B28C0F29780287A022840F02C
:201660009380A88900F00F010F2940F08D80C0F303100F2840F088809DF82860002E18BF5A
:20168000022E40F08180424C404894F84A20022A3BD00068062A39D010B18179012935D01B
:2016A000082A18BF042A6FD16D8910B18079022827D0B4F84800854266D1012E07D004F1F5
:2016C0005D000DF12D0117F093FC00285CD120784FF4007113F040FA002855D1E06C0290E1
:2016E00001268DF80D6002238DF80E3094F852708DF80C7002A80FF08DFF10B114F0FEFCA6
:2017000042E0284615F0B8FF3EE0006840B900230093288869896A7C04F054F89DF8286063
:201720002888ADF810006889ADF81200A87B8DF81400AF8900206FF30E0707B101208DF8B3
:2017400018608DF815009DF827408DF819409DF82C708DF817709DF82A009DF82B308DF82C
:201760001600687C0DF12D018DF81A009DF838608DF81B3008228DF81C600DF11D0017F05A
:2017800089FD04A804F036FD0FB0F0BD38040120E4FA00202DE9F04380460E20ADF1340D0D
:2017A00015464FF001098DF80100B8F1000F8DF8023050488DF8005000F1010000788DF834
:2017C00004900F468DF8030047D1112004A93A2218F00BFB00283CD1444E0DF111007B19CE
:2017E0009DF80320716803901C4642F02802481C7060581C227017F041FD054617F01AFD1F
:201800000146284618F0C8FC48460DF131013A2218F0EBFA083500280CBF9DF8310000202A
:20182000287017F007FD01460DF1210018F0B4FC7088401C80B27080B0F57A7F02D8706821
:2018400001282FD12A4800784FF4007110F0AAF928E000207C19039024E07C19ED19687B4C
:2018600011F054FC3A2808D03B280FD1112004A93B2218F0BAFA30B108E0112004A93A22A0
:2018800018F0B3FA10B90DF1110000E0002003909DF80300217808432070611D0DF121007F
:2018A00018F07AFC0DF12900611C042217F0F2FC039E2078002E8DF82D0008BFA12012D068
:2018C000404669460DF121023B4604F009F9054620780021102200F0F80020700DF111007E
:2018E0000DF034F828460DB0BDE8F083480401203BFD002013FB00202DE9F047564CA4F105
:20190000080000F108058068D0F80001807AADF1280DC0000BF09EF90028089008BF1A242C
:2019200000F0958018F052FC8246286800F59162D0F8000100894FF6FF780026C14608E0E9
:2019400020682268D0F80001761CB6B202F591620089B042D8BF002473DD2068D0F80001F1
:20196000C07A0127002548E0ADF81480ADF8168006A8FF2108220CF0E9FF2068D0F8942460
:2019800004A9D42090472068ADF80480D0F894246946D12090472068D0F800012268C08804
:2019A0006D1CEDB202F5916230E0ADF800608DF802501268D02069469047A8B99DF80C0037
:2019C000012810D19DF80B0068B90DF102020820002112F8013FFF2B03D1401E01F1010157
:2019E000F7D10829ACD0002720682268D0F800016D1CEDB202F59162C07AA842D5DC002F5A
:201A00009ED12068D0F80001C0880025A84297DDADF80060ADF802501268D120694690474E
:201A20000028B8D1BDF804008145B4D0ADF810002068D0F8882404A9D4209047002893D03E
:201A40001924504618F04CFD089813F0A5F820460AB0BDE8F087C04614010020574B2DE9F3
:201A6000F0475879002840F0A5800020012116F07BFF002800F09E800668002E00F09A8043
:201A800007464089C1096CD2984698F83210890872D3326A51791479400B04EB01242CBF65
:201AA000402500253868B7F818900088824613F013F8002846D15046032112F0E7FE00283F
:201AC0003ED15046002113F02FFD29460DF090FC061C31D07079012806D0032824D00428C3
:201AE0001FD14FF6FE702FE0B179708811F0180F10D0FF21A042317105D0484503D04FF6EC
:201B0000FE71814209D1204649464FF6FE7205F041FF02E098F8381031714FF6FE71814207
:201B200008D17079022807D05046072112F0AEFE10B105E0824603E0504616F025FE03E083
:201B4000504601E04FF6FF70844202D0398B81420ED1386801880222002320460DF000FA8F
:201B60000AE038680088034612F0B6FF30B918464FF6FE71814203D1CD2111E04FF6FF702E
:201B80003968088012F0A8FF00280CBF012000203968C8810849386809F0A8FB011C04D0D7
:201BA0003868407B12F0CEFA20B91FB138460121FCF7B2FEBDE8F0878D5D0200E4FA00200E
:201BC0002DE9F04F0446656928780026ADF12C0DB0468DF824000DE03918C978401CC0B20F
:201BE00002F8011B74E09DF82400761CF6B2401C8DF824006878B0420EDD216809A80090FC
:201C000008AF01976368E27A087D8988C3F3C0030CF026FA0028E6D1F01C80B218F03CFBC7
:201C2000071C7BD006B3287845468DF82400216809A8009008AB01936368E27A087D8988DB
:201C4000C3F3C0030CF00CFA68B19DF822009DF824307919761E05F10105C87003F1010001
:201C60008DF82400E3D1A846216809A8009008AE01966368E27A087D8988C3F3C0030CF0D0
:201C8000EFF900280CBF012000203870E07A87F8028078702168666808F1010501F1060BE4
:201CA000087DB1F804A0A47A0A90F00880F0010000F00109E8B2804618F0EEFA051C08BFFF
:201CC000102624D002463878002602F8010B3046B978814280DC7878112803D0132813D1D5
:201CE000142300E012230096CDF804900120029003960494CDF81480069507900A985946F9
:201D00005246FEF7D5FA0646284618F005FA384618F002FA002E08BF012000D000200BB063
:201D2000BDE8F08F29282DE9F0410EDC29285FD0203800F09A80401E00F08C80401E7ED015
:201D4000401E71D0401F61D007E02A3845D0401E38D00E3820D0401E02D00020BDE8F081F4
:201D600093E8600091E880010CCA284631460BF091FC4FF0000403D828461E46154601E01F
:201D80001946104633462A46FDF71AFB43463A460BF080FC74D872E093ED000A92ED001A5B
:201DA000D1ED000A0024B4EEC10AF1EE10FAACBF30EE410A31EE400AB4EEE00AF1EE10FA2F
:201DC0005EDB5CE018680B68116800248142D4BF411A091A8B4253DC51E018680B68116891
:201DE00000248142D4BF411A091A8B4248DC46E0B3F90000B1F90030B2F9001000248142AC
:201E0000D4BF411A091A8B423ADC38E093F9000091F9003092F9001000248142D4BF411A00
:201E2000091A8B422CDC2AE018680B6811680024814294BF411A091A8B4221D81FE01B6834
:201E4000106809680024984294BF181AC01A814216D814E01B881088098800249842D4BF3A
:201E6000181AC01A81420BDC09E01B781078097800249842D4BF181AC01A814200DC0124C6
:201E80002046BDE8F0817047F0B504462C20ADF16C0D18F001FA071C00F0A28008223A70B1
:201EA00000257D70207FF870207C04F11401387407F1140017F0F2FB381D211D0C2217F0EF
:201EC000EDFB4848237D217FC01E466984462846B04206D000E0B6683279914218BF002E3C
:201EE000F9D1F6B1DCF80C00D8B173B9C17DF27D914212D190F8251096F8252091420CD139
:201F0000C16AF26A914204D007E0416B726B914203D101793279914203D180680028E4D1EB
:201F200001E000283AD120461AA916AA01F0C2FC0246BA7098B1401E02D0C01E0FD010E05D
:201F4000607D9DF8681016AB09F054FF38B107F11C0016A9102217F0A1FBBA7801E0BD70B9
:201F60002A468DF80020F8783E1D8DF8010096E80D0001A981E80D00387C07F114058DF806
:201F8000100095E8050005AC07F11C0184E8050007A8102217F082FB68461CE0BD708DF8B7
:201FA0002C50F8783E1D8DF82D0096E80D000CA981E80D00387C07F114048DF83C0094E871
:201FC000050010AD07F11C0185E8050012A8102217F064FB0BA817F0B9FC384618F09CF8DD
:201FE0001BB0F0BD4B1900202DE9F0470546A87A022840F09B804E4CAF7B5248DFF840A1A0
:20200000666A002F7CD1E168F9B12769EFB16769DFB1A768CFB114300078012815D16888A7
:202020008847AE1C88B943490A6830889101A1EB820122699047012878D16169308888474A
:20204000A16830888847BDE8F0873B486D88006878B101680A88954208D1096A4A7809786A
:2020600001EB0221490A01D220B136E040680028EFD10020314933230027012401F6C4427B
:202080001679FF2E02D01688B54206D05B1E02F124024FEA4404F3D100E0274601F59A781B
:2020A00001F12E09002319F803208AB19E0058F8064027420CD0104616F062FF38B1417B8A
:2020C000052904D1BC431E2348F8064000E000205B1CDBB21E2BE6DB68B1417B05290AD14B
:2020E000016801270D8056464773307820210FF059FDBDE8F087284611F0B2FBBDE8F087DA
:20210000A6B1017D012911D1807F40080ED3042016F0E3F9011C09D06420087001274F70D7
:20212000688856464880307811F0B6FABDE8F087ECFB00206CBC0200380501202001002006
:20214000E4FA0020ACFE002070B5534C054694F84A00ADF1300D082818BF042840F099807B
:2021600028460DF10E0116F0C9F94FF6FF7012F033FFBDF80E0004AE314600F0EFFD012843
:2021800000F087800DF11A0017F0AAFF0DF11A00314616F02DFF58B1BDF80E2017F074FE5A
:2021A000904205D004F13E014B200A8013F034FA17F07CFEA98A3B4D884216D004A817F07F
:2021C000BBFF38B10079012818BF022802D104A810F010FC3148016839B105F113000078E1
:2021E000012802D1BDF80E008847BDF80E00002115F0D6FFBDF80E0015F036FE00248DF8EE
:202200000040BDF80E00ADF8020068460CF0D8FB98B10DF11A00214608220CF097FB01AC6A
:202220000DF11A00214616F0E3FE30B104A9204617F0C6FD684603F0CFFB01A804A917F0B2
:20224000BFFD68460EF062FA50B1BDF80E00BDF80210884204D0ADF80200684603F0BCFB92
:202260000F482E78046836F0010012D10DF12200FF2108220CF06AFB5CB104AD0DF1220141
:202280000822284616F000FA18B9BDF80E102846A0470CB070BDC046E4FA0020F4FB0020B1
:2022A000B0030120ADFE00202DE9F041524D2968F4310A68064692F84400ADF1180D8228EA
:2022C0001ABF92F84400401C002082F84400086890F8441000EBE10090F82C104A1080F86F
:2022E0002C2048080AD22968F4310A6892F84400401C82F84400C0B28128E8DB2A68F432C0
:202300001168DFF8F88091F84400812824DB8878E8B944462168D1B10868C0B10F4615F00F
:2023200009FF8046386817F0A9FF10B1386818F0B3F8384618F0B8F8384612F02DFC083C49
:202340000020A060404617F0D8F92A68F4322A203070D2F84C1249E0D2F83C234431E1206D
:2023600090472C684FF6FF730220ADF80830F43422688DF810009778BFB917F079FD4FF4AE
:202380007A71B1FBF0F01E49434600220AF0A8FC00282DD02868D0F8F4001A2141702A2768
:2023A00037702868D0F8401320E0022F1CD0012F19BF0720832108208021002700974932D9
:2023C0000192D4F8844202AAA047DB2807D0E52805D0F32803D0DF2818BFE82808D1296843
:2023E000D1F8F4104870DAE7D4F874133046884706B0BDE8F081C04614010020D8040120FB
:20240000FD7C01002DE9F041064670680F46ADF1300D000944D2F07A002837D0012841D1B4
:202420000024B968ADF8284021B13068801D089008A8884731680094087D898822460AAB4C
:2024400013F0C7FABDF82800002800F083803168012500959DF828008DF82A00BDF82870B3
:20246000019538128DF82B0002950394B27A0492022305930DF12A0706970795087D03220D
:202480002346891DFDF714FFFF2064E0F06841783768007800EB0120397D10F025FC59E07F
:2024A000F07A08B1012056E02C4D346868784FF480410FF035FF6869A846A41D40B91820C5
:2024C0000AF0C8FBC8F8140008B10021416121E070B1637A417A8B4207D161894289914208
:2024E00003D121880288914220D040690028F1D1D8F814501435286820B100F11405286807
:202500000028FAD118200AF0A5FB286070B100214161286850B1217A017221880180617AE6
:2025200041726189418100250573056198F801004FF480410FF036FBF96859B13068F76812
:20254000801D08907A78387800EB0220ADF8240008A8884700200CB0BDE8F0814CFF0020F2
:202560002DE9F0430E460024ADF1240DADF8160006F108078DF81440384616F055FA50B955
:2025800005A80CF01DFAA124012840F08A8005A814F004FA85E038460DF122016A460CF0F4
:2025A00057F905464FF6FF70A84276D09DF82200DFF8FC8000282BD03C4801789DF81000CD
:2025C000F8B1401E11D0401E04D0FB3814D0801E12D048E001290CD002290AD006F11E0002
:2025E00002A9082216F056FE3DE0012918BF022902D14FF4817001E040F20310B08274820E
:2026000031E005219DF81300718200F07F0029E002A83946082216F03DFE4FF001098DF80E
:202620001190FF208DF8100017F02BFD274600F00F0000942946142201976B468DF8120091
:20264000042013F0FFFFAF0007EBC507404621460C223F1838460CF079F9748287F809907C
:2026600040F20310B082A8003474414600EBC5000A58B2610F580A237F1CB7FBF3F20F50C2
:202680005A43BF1A0DD1401801210A4F017238784FF480610FF086FA03E0748240F203102F
:2026A000B082204609B0BDE8F083C046ADFE002064FE00203BFD00202DE9F0478246484E5B
:2026C0004E4C56F80C0C9046894680082AD245480068810D28D2051704F13400006800683F
:2026E00080476D1CC0F13E0110F1020F4FEAE101D8BF07218D42B8BF0D1C3B480068C0F3A1
:202700000320401B102803DA0028D8BF012000E00F20364900F00F0040F0F00081F84D00D3
:20272000087801E03248306000203249324F256808603868A96927208847324D304805F168
:20274000300211682B460840106003F17800006820F48070A8672068016B4FF480608847D8
:202760002068016B4FF4816088472068016B4FF4C0608847244901200860C5F88091286000
:2027800056F80C0C800806D2B8F1FF3F14BF40464FF0404030603868E8698008FCD3072075
:2027A00010F07CF90228FAD1BAF1010F13D0206A164E8168304688470428F8D0012804D103
:2027C000206A4268032130469047D5F8180220F00300C5F818022068806B8047BDE8F0872D
:2027E0001C000940B44F00500C1300500D620840FD0000400C4009402C200940B8010010CB
:20280000FFFFFEFE0C20084028200860004003402DE9F04F15460646287A0C4600F03F01F7
:20282000E8886FF39F2040EA0130A988ADF1140D6FF39F2141EA003B49490E9FC8789A46D5
:202840004FF0000988462EE09DF80B10C8080CD3BDF80E00844204DD241AA4B2162C13D9C9
:2028600031E02146304610F0F1FE0020F6F7ACFC98F8330098F803204FF00009401C90FB21
:20288000F2F15143401AC6B298F803008119491E91FBF0F24243891ACEB2B10001EBC601E1
:2028A0004144B1F84C40484503DC0020A8810A2052E098F8323009F10101B3421FFA81F9D7
:2028C000E4D0172CE2D3E41F30466A46A4B2214608F038FF9DF80B108808B7D34808B5D296
:2028E0002A7AEB881AF00F0018D0401E12D0401E07D0401E18BF04202ED100985845A5D148
:202900000CE09DF808009042A0D1BDF8060098429CD103E09DF80800904297D1AFB10AF0D5
:20292000F000102811D1BA89BB68684600210FF0DDF8002888D1F988B868BA884018396827
:2029400015F0F4FC00287FF47FAF68460EC80EC503C885E80300002005B0BDE8F08FC04628
:202960005CFC00202DE9F84F504CD4F8A000D4F8A060002800F095800546E86840F60301AC
:2029800008274A1C02E040687F1EFFB260B15FB10388994218BF9A42F5D129692CC83831DB
:2029A0002CC189C881E8890006F1280090E800034FF0000A06F12807D34687E8000CB16831
:2029C00021B357464FF0E24A07EA08001AEA090508BF002813D036A090E80C0002EA0802EE
:2029E00013EA090308BF002A04D0B5683069B6F93010A847504607EA080800EA0909B568C5
:202A00003069B6F930104B464246A84717F0DEFB0546B4F9B600401C6FF31F30A4F8B60039
:202A2000214886F833B06FF00207378615F044FD284617F055FDB4F9B400B4F9B6108842FC
:202A40002FD16068D4F8B860D4F8BC7090F8FC1000290CBF052007200AF068FF58462EB120
:202A600096F8FC5005B9306886F8FCB05E462FB197F8FC5005B93E6887F8FCB0864238BF4F
:202A8000061C66B1B6F1FF3F0BD017F0F1F9B6FBF0F104F5CE7016F03BFEBDE8F88F16F012
:202AA0002DF9BDE8F88FC046D0F5002030F50020F0FFFFFFFFFFFF8EFEB5524C6069258954
:202AC000A689E169806D2A468919083109F00EF86269916D49199165E2697619B0B21218BF
:202AE0000832127801A90A70444EE169401C80B20918097A721C401C117081B2E269A181D5
:202B000052180832126868460260091DA181042115F099FF63690090054616F035FFD86361
:202B2000284616F0F5F9A3F84000EA2013F0BAFC02213548324D017068684069007830B133
:202B4000307810B97078FF2801D00420E0706769E078397C084338749DF9040017F07AFBC6
:202B600087F8460007F17406BE6539899DF904007B6887F84800B7F85C000026401AC01892
:202B80007860B88987F84760800A0AD32868D0F80813384688476769786E10B1B7F8680041
:202BA00010B397F8600050B12868D0F80C13384688476769F86C10B1B7F85000A0B12968C8
:202BC000B8310A68107838B1936C2BB119463846884767692968B831D1F8A0113846884791
:202BE000666116F0F7F9FEBD2868D0F8541204F11400884766610DF0F9FFFEBD240001200B
:202C00001401002068110120051401202DE9F04F0546E97A6869ADF11C0D0229814609D144
:202C20000078032410FB04F0401C80B217F034FB061C01D100208DE00027A346A246B846BB
:202C400047E017FB0BF0862332E09DF80E00A178884230D10498F8B129688888032814D108
:202C6000238893B9D4F8031005A8022216F012FB2868007D10F040FE11F068F92968BDF8A7
:202C80001400097D10F030F81FE0087D02AA2346891D13F03AFE07E02968D4F80330087DFC
:202CA00002AA891D13F0FEF8031C0ED017FB0AF031184B7004E017FB0AF08D2231184A701A
:202CC00021887F1C3018FFB2418008F101005FFA80F899F80000404522DD2968072018FB4B
:202CE0000094641C087D2288898802AB10F034FF0028A6D09DF80F30002033F07F0318BF92
:202D000001206968C1F3C00181429ED017FB0AF1862072187318507021887F1CFFB25980C5
:202D200037701FB9002070700127377068682A68C00880F0010000F001000090A87A911D59
:202D40000190107D928833460AF0B4F9304617F0E3F9012007B0BDE8F08F70472DE9F047C2
:202D60008A46071CADF1200D08BF002000F0918049480088B8420AD116F05CFA0146504686
:202D800016F036F900280CBF0125002500E012254FF00009ADF8027068468DF800900BF08C
:202DA0000FFE20B101A815F03FFE012843D0122D4AD1504617F0C0F928B101888F4202D059
:202DC0000679052E03DBB9F1000F3CD13CE00780E6B132490D78032E18DA31493DB901EBE4
:202DE0008502126B01EB8501C261096B0AE001EB85010B6B9A01A2EB8302C2610A6B91011D
:202E0000A1EB8201816180F8209003E06FF00101C16181614E46C6600125ADF810705146B5
:202E20008DF80E500DF1120016F0CAFF0DF10E0002F0D2FD07E001A9504616F0D9F80028DD
:202E400008BF012500D04D463846514610F04EFA0A2818D0A02813D1124C322604F102084A
:202E60004046514616F0C4F830B9761E04F11C0408F11C08F4D100E02780384612F0ACF854
:202E8000012D01D004E001253846494616F01EF9284608B0BDE8F0871EFB0020CBFE00209B
:202EA00018BC02006C0800202DE9F84F8146D9F80040D9F8047094F82360B4F814A0D4F8F3
:202EC00010B090460D465EB1A168434816F01FFE002818BF6FF001007BD1012084F82600D5
:202EE00084F82180002625604A463C483C49E66115F06AFB3978272017F070F95146584623
:202F0000062204F06BFC002857D13749091F086820F00200086094F82000042806D1334822
:202F20004C38006840690146272088472D4F4FF0020B4FF0805AC7F8FCB2DAF8FC014068DA
:202F40000146062088470AF5FE7A38BB584613F0CDFDB8F1020F4FF0010005D0B8F1040FD5
:202F600018BFB8F1060F01D1314600E00421C7F84C11E968C7F85011C7F8546184F82400CD
:202F8000DAF80000AA68E968036968681C460B46A04748460DF086FBBDE8F88F40203860F6
:202FA00080253D6094F8260020B10B4817F024F984F82660C7F8FC6207E094F8260020B14C
:202FC000054817F019F984F826604FF0FF30E061E069BDE8F88FC046B80E01204012012005
:202FE000510002000444024088470240FC0100102DE9F04F80464E489346ADF1240D07690D
:203000000691002F00F090807D6801248246494F07940320B8F1000F8DF8140003D0069800
:2030200003A914F098FF4FF000094E4601E0761CF6B2A968087BB04217DD03A80090CDF8D8
:203040000480079802900969FA7C7B69287831F816100AF039FE0446B22C06D0002CE6D1EE
:20306000DDF81C90B8F1000FE1D1B22C26D0B9F1000F02D0B8F1000F20D0A968002602E045
:20308000A968761CF6B2C879B04217DD03A80090CDF804800024029489683A7EFB692878D3
:2030A00031F816100AF010FE0446B22C06D0002CE6D1DDF81C90B8F1000FE1D1B9F1010F33
:2030C00004D1B8F1000F08BF802100D0FF21DBF80000B22C017314D03878FF2824D1DAF864
:2030E00010000668CAF81060F6B175682B7823B1F12B02DA002E8CD116E03668CAF81060DC
:20310000F2E700208AF800009AF8010040210FF007F915F07BF89AF801004FF480410FF033
:20312000FFF80C2016F0CEFD09B0BDE8F08FC0464CFF0020DC0201202DE9F0470646880F1E
:20314000C0F08E8000200EF095FA464816F072FD454C40F60A09A4F8009000256580207B56
:2031600005F00F0120F00F00014321736560607B4FF0010808F00F0720F00F0047EA00010C
:203180003046617306F086FBD6F808A04A462146D01F574600F1010C00E027467C6834B161
:2031A00023889A4203D0984218BF9C45F5D179607A7B2E4C05F00F0322F00F0213437B73A7
:2031C000D4F8983033B1DA681288904223D06046904220D0338FF3B1F56306F138025580AA
:2031E00096F8440005F00F0320F00F00034386F8443096F8450008F00F0320F00F0003435D
:2032000086F845304A60487B05F00F0620F00F0046EA00054D7316F02BFB1548A06294F819
:20322000310080B91348006801684046884701280FD0787B08F00F0120F00F000143797351
:203240000D4EA66205E011F0C7FC0028FBD010F0A5FD504616F0EEFC5146404614F08EFF99
:20326000BDE8F08701010E04F412012030F50020F95E0000E0010010992B02002DE9F0435B
:203280004E49DFF830910A68ADF1140D1AB94C464A34267800E00226444BD9689F68761FD9
:2032A0007ED0761E7AD0002A67D09179012964D03F4CE76A022903D0A169002973D071E078
:2032C00038460027002854D1780009F0C3FC5FEA00084BD0E06A40B10021028828F8112029
:2032E00040684E1CF1B20028F7D14C46B4F89200618F814233D081460A2000EB47008DF8FB
:203300000D0003A815F080F9061C2CD035690920287004F15D016F70A81C16F03DFF5FB1B2
:2033200008354046017805F8021F30F8021B7F1E4FEA21216970F5D10124B47715F07AFF69
:20334000706201A9484614F006FE10B1747701A83062A6F802903046F8F78EFC03E0CDF8AD
:203360000080FAF72EF9404611F016FC12F0C6FE19E040687F1CFFB2A4E740780E498DF84A
:203380001000086838B900208DF8050001A9012013F03CFC07E0096804A803E019B101E07A
:2033A0000FB13946884705B0BDE8F08334040120ECFB0020E4FA00207CFD002038040120DE
:2033C000F0B5064631684889ADF1440D4008C0F092804A894FF6FE70104048810868036A1D
:2033E000C57F5978187800EB0120694611F010FFD878997801EB0021ADF80A105A791879CC
:2034000000EB0220ADF80C0098799DF807708DF81200D879002F8DF8130008BF082403D05C
:2034200003F10800102405909DF808701FB1181908340690E4B28DF801409DF8057037B199
:20344000185D641C8DF80500E4B28DF801409DF806C02A480027BCF1000F06D190F82F2033
:2034600052B1428F8A4206D106E090F82F201AB99DF8022002B90127A7B9BCF1000F05D1B9
:203480001B190A932D1B8DF81C500CE090F830001B190E330A9315F045FF2D1B281A0E3853
:2034A0008DF81C000A9B37BB1878042823D10DA800210E220BF04AFABDF80A000A9FADF8D2
:2034C00034007978880924BF01208DF83F0031F07F001CBF01208DF83E00C80934BF0699AC
:2034E00005990DF1360016F057FE30798DF840000DA812F037F811B0F0BDC046E4FA0020D9
:203500002DE9F84F80460D462868DFF824A1D8F80040D8F804700689D0F804B0E16891468A
:20352000504616F0F4FA0028CDF8009018BF6FF0010074D148464FF0000960723A49656117
:2035400042464B46C4F804903648A37015F03CF83978272016F042FE31465846062204F0C9
:203560003DF9A8B9334E4C3E306840690146272088472E4F4FF0020BC7F8FCB2F06C4068D1
:2035800001460620884750B14020386080263E60504616F031FE4FF0FF30BDE8F88F5846AF
:2035A00013F0A4FAF06C95F82010C26928699047F26CDDF800C095F8200095F821101368E5
:2035C000BCF1010F4A4608BF01229847E869C7F85001C7F85491A869C7F85801A96959B18B
:2035E000F06C076968684A461346B847F06C806901461148401E8847207A042804D0306803
:203600000069014627208847F06C0369E969EA68A8681C460B46A04740460DF0B7FBBDE8F4
:20362000F88FC046401201205515020004440240B80E0120FC01001003000080F8B5054625
:20364000687F0F4600280CBF08201020AE7F0EB10830C0B22E7F0EB1401CC0B2AE7926B115
:20366000297A00EB4100801CC0B22E7E6870002E0CBF00260E260024297D2B7E85F8344032
:2036800009188919397033B13A48007815F04AFE3978081838703878742867DC09F0DAFABE
:2036A000071C64D016F0FCFB95F83420A97F2B7F41EA42016A7F42EA4102A97941EA4201AD
:2036C0002A7E42EA410203B1012429786B7E44EA420441EA800103F0030041EA801141EA73
:2036E000042188B2397000127870A878B87068880012F87028793871A88800127871A87E7B
:20370000B871E87EF871687F002808BF082405D0296A07F1080016F03FFD1024A87F28B1D1
:20372000696A381916F038FD0834E4B2A87988B1287A3855697A631CD8B239542A7AE96861
:20374000431CDCB2E019520015F0A4FD287A04EB4004E4B2287F00B13855687829692A7D22
:203760008019C0B2C01915F095FD00E027463846F8BDC04614FB0020F8B50546A869837815
:20378000002427461BB3FE2B21DC41780078474E00EB01203188814206D015F01BFD00283B
:2037A0000CBF8126892613E0184615F041FB264650B18268002A04BF4068846804D0012089
:2037C000194690470127044604B9832600E08226374801685EB954B1227BE079022380189C
:2037E00010FB03F00C30C3B2502B01DD58E0042301F8016BA869007801F8010BA8694078A6
:20380000042B01F8010B42DD181F01F8010B207801F8010BA07801F8010B6088001201F86C
:20382000010B207901F8010BA088001201F8010BA07900F00F0001F8010BE07901F8010B24
:20384000E67916B10020864214DC207B0870267BFEB1491C002086421BDD26694200965DFE
:203860000E702669925B12124A70267B401CC0B2891CF0E7A6684200965D0E70A668925BC9
:2038800012124A70E679401CC0B2891CDBE70020087005F11100A91C48F204020DF03EF9DE
:2038A0001FB114B1204611F077F9F8BD50FD00209CFD00202DE9F04100250E1CADF1580D28
:2038C000904603950746ADF8105004D0B8F1000F18BF002F01D1042083E0104635702946D3
:2038E000102216F0DBFC38798DF80000002804BFB868019005D001A807F10801082215F039
:20390000CDFE68460DF1120104AA0CF01FFA36490C7802284ED001284DD09DF8000002280A
:2039200008D1387C9DF81C10814203D0002818BFFF2840D19DF81F00397D00F00300884245
:2039400004D19DF81F0010F0030F49D008A903A8042215F0A3FEB8690399884228D99DF86E
:203960001F00397D00F00300884221D19DF81F00801000F00401042902DA797D012917D07A
:2039800000F00701072918BF042901D1787D78B105290DD006290BD009A94046102215F087
:2039A0007DFE9DF81F00C0F382003070012018E00CB115E00CB9284613E0387D0228A8BFCC
:2039C00003200EDA787D58B9084C40461022214615F0C0F820B921464046102215F05EFE4D
:2039E000022016B0BDE8F08120040120CCB302002DE9F04F05468846ADF1140D1C46D5F8A7
:203A000008B00E990092DBF80400019108EB0401884238BF6FF003047BD3404E30684FF07A
:203A2000FF3116F074F83E48019F01684FF0000978081CD23846CDF80C90800827D334B357
:203A40003046DBF800200099066823464244491E521E11F8010F12F8015F054085421CBFC6
:203A60006FF00604301C52D15B1EF2D10FE034EA010701EA040202D02A480068121801EA6B
:203A8000080128460EF046F9002803903CD1DBF8005010F0A3FA27464544DDF800A00290ED
:203AA00002E0BF1BB244AD1997B1082F8CBF08263E1C16F08BFB049029463246504615F09A
:203AC00083F88146049816F00BFDB9F1000FE8D0029814F0F1F9B9F1000F12D10198C00804
:203AE00012D38CB1DBF8000000994044491E401E10F8012F11F8013F9A4202D1641EF7D175
:203B000002E04FF0FF3003900448039C006816F073FB204605B0BDE8F08FC04694130120EE
:203B20009C130120981301202DE9FE4F0CAF1D468B465FEA02083E78009014BF4FF0804A22
:203B40004FF0005A16F042FB0324DFF804910190BBF1FF3F14D1D9F8A810009816F072F805
:203B600058B9D9F8AC10009816F06CF800280CBFD9F89870D9F8AC7008E0D9F8A87005E036
:203B800000985946002211F093FC0746002F59D097F8330030F07F0053D04C46D4F8A8000D
:203BA000B84219D0D4F8AC00B84215D000982A463346394608F05AFE002842D094F8240091
:203BC00001283CD094F82400042838D0214904F1E00016F019FB32E0D4F8A8005346002232
:203BE00011F084FCD4F8AC005346002211F07EFCB8F1000F14BF1848184814F089FAB6B15D
:203C0000D4F8A80000224FF0807311F06FFCD4F8AC0000224FF0807311F068FC3869C4F8E2
:203C2000D80094F8DC0040F0010084F8DC0035B1D4F8981000982A46334608F017FE83242C
:203C400000E00424019816F04BFC2046BDE8FE8F30F500200200004001000204010001044A
:203C60002DE9F04FADF1140D02921D460191DDF83CB00E9C009016F0A9FA464A6FF001080B
:203C80004FF00109002392F840A2039009FA03F616EA0A0F6FD0B5F1FF3F18BFAB426AD182
:203CA000D8B215F003FE002865D0877A002F62D192F84012B14382F840124F468772009DED
:203CC000437292F842120560491C82F84212019E06722E4F4760017A074601291ED0022973
:203CE00024D140F20361018290F90930C17C5B1D21F00F0103F00F030B43C3746379817CBB
:203D000063F3C7018174C17CA37963F34611C174C17CE37963F30411C17407E00A20388251
:203D200097F90900401DB874A0687861BBF1000F08BF002012D09BF801009BF8001097F935
:203D40000960134C4FF6FC75800040EA4110711D40EA012005EA000144EA0100B86102983F
:203D600000B17860506808B9386850600CF07EFA97F9098002E05B1C032B87D3039816F0E2
:203D8000AFFB404605B0BDE8F08FC04677F500000100040630F500202DE9F84306464FF676
:203DA000FC751C4617468846B54200F08480002111F0BAFBDFF804910646B9F83A00B042AE
:203DC00001D1E00977D3214630460BF011FBC0B9A81C00210BF00CFB98B914F0180F0DD041
:203DE000374B0020997911F0180F03D1962805DA184606E0401C08339628F3DB0220BDE848
:203E0000F883AD1C0680454518BFA0F802808471610824BF44F004048471012F0CD0417925
:203E2000012913D0817911F0180F0CBF99F83710FF210171477109E001214171817911F0AE
:203E4000180F0CBF99F83810FF210171012F32D1B9F84810404612F0DBFB60BB194C1A4F82
:203E600000204101A1EB8001C919B1F84C6707F52772002396215588AE4205D0491E02F12A
:203E8000080203F10103F6D1962B04D0401C1C343228E6DB0FE0204600211C220AF056FDFC
:203EA000A4F80080B9F848006081AA27A77401266674062525740020BDE8F883E4FA00201D
:203EC000BC0300206C080020200100202DE9F0479646464A88461E2300240146012520466F
:203EE00097782FB15B1E02F1080204F10104F7D11E2C79D03E4C3F4F814633264FF6FF7C10
:203F000082F8069037F824AFD04510D0638F53450DD03B7933F0040A06D0012B07D14B89A0
:203F20009C4508BF284302E093795B1C9371761E4FEA4505E6D1304D3226ACF1010C35F88B
:203F40001C3F98450DD09C450BD0B4F848306F89BB4206D16F7C27B1AF7C17B193795B1C67
:203F60009371761EEBD19779082F01DC17B909E0082393718B7C012B04D094F826305B1C81
:203F8000137101E082F8049094F82B30937094F82570D7708E891680CD7C82F805E0D571C1
:203FA000B8B116491E2201F12D030D46494613F8017F37B1BE4504D0521E01F10101F6D180
:203FC00007E01E2905DA83F800E005EB8105C5F834012078402110F0BFFD20B9207840218A
:203FE000642216F0B5F80120BDE8F087CC020020E4FA0020C00D00205008002020010020B9
:204000002DE9F84F8346DBF81800057800216A46A3200FF0A9FABDF800004FF00009854218
:2040200024DABDF80000401B84B2042C01DA0CB91DE00324E00000EB041008F00BFE5FEA1F
:2040400000090FD007464FF000088CB146467119A2203A460FF088FA761C1837F6B2B4424F
:20406000F5DC05E04FF0B508002401E04C46C8469BF81100E1B215278DF8020011FB07F0EC
:20408000001DC0B2401C08F0E5FD4E460BF1020B071C45D0781C82468AF800809DF8001083
:2040A000E3B2B970FD7004253C7143B3001DE4B2314616F071F8317A00F8011BB17A00F88E
:2040C000011B7189091200F8011B317D00F8011B317D032906D0317B00F8011BB1890E35EC
:2040E000091205E006F10C0116F056F8B17D1535641EEDB200F8011B06F11806D8D10C4EA3
:204100002B460DF10200594648F23302341DC4F800A00CF003FD384610F03EFD09347460AD
:20412000B9F1000F02D0484610F036FDBDE8F88F98FD00202DE9F84F8046D8F80430B8F87B
:204140000240002739463A461D191EE013F8036B7F1CD21CFFB292B2A6B913F8056B30467C
:2041600015F02BF8521D92B278B1304608F0E8FF8618B442B8BF002073DB09181B181218EF
:2041800089B201E09B1C921C92B29D42DED80E2017FB00F0401CC5B2681880B216F07CF896
:2041A0005FEA000A5CD0D8F80440002F0AEB05068AF8007054D04FF000084FF0010B0AEBA0
:2041C000080500210E226D1C284616F067F814F8010B28702B7861782078A41C00EB012095
:2041E000A5F8010093BB14F8010BE87061782078A31C00EB0120A8801878597800EB012092
:20420000E880E878014614F0D8FF9C1C20B30846314612F065FAADF800B09DF80030A14602
:20422000002B07BF411E4FF0FF335B46002128B119F8012B401E72541944F9D1E878C5F87D
:204240000A6008F07DFF2418361805E061782078A41C00EB012028817F1E08F10E08AED100
:204260005046BDE8F88F70472DE9F84FD0F8E8200023083A002AC8BF0123D0F8C0C0D0F84E
:20428000D020E346DBF8004094420CD8DBF81470002FBC4678D001228CF81020D0F8C0B059
:2042A0004FF0000E00E09646DCF80020A2EB0E02B2F5806F88BF4FF48062D0F8D8702FB96A
:2042C000C0F8D820D1F81C808E6904E0C0F8DC20D1F824800E6ADCF804402CB92B4C9F0042
:2042E000E55900F1F6040AE0294D9F00ED5903F1010A02FA03F90EFB0A444C44641EB560DB
:2043000034600C6804F10809C6F80490B56843F6F07A1401103C0AEA04042543B560DCF8CF
:20432000086026B9194BDD5900F1F40308E0194DED595F1C02FA03F30EFB07669B195B1E10
:20434000C8F80850C8F80430C8F80090D8F80830E34544EA0304C8F8084004D1D0F8D030F7
:204360009B18C0F8D03090F8FE706FB90B685A6A42F003025A62D0F8CC004F6943680A6920
:20438000196847EA02008862BDE8F88FE8C30200F8C30200F0C30200F8B5374D0024287047
:2043A000364E85F84A40382030804FF4287008F051FC706028B1706821464FF428720AF08B
:2043C000C5FA2F482F49304F304E81613049C7610A7D0662012A15D12E4A2F4F4262897F0D
:2043E000C760490802D2006B58B90BE02B4F07632B4981622B4E06612B4B83602B4A42617E
:2044000038468047AC602A48046012F007FD15F0D1FB294996274FF6FE7201F1E80020F8C8
:20442000082F4280047144717F1E8471F7D121480C2700F150035A805C705C607F1E03F825
:20444000084BF8D10827428004727F1E00F10A00F9D128781E277F1E21F8082BFBD1174A7C
:204460000121117010214FF47A7215F071FE02F02BF913480460F8BDE4FA002030050120E7
:20448000ECFB00208D6A02008D8C020045080200ACFE0020CDD101005D8002006986020079
:2044A00021F20100B1EA01006D300200758C010038050120A4010020CC020020D513012091
:2044C000380401202DE9F04306467568B7680C46ADF1140D15F07AFE95F8FD1021B9616922
:2044E000102901D8042903D215F0FAFF00206FE04FF0010985F8FD9015F0F2FF2069C5F8AC
:20450000E4006069C5F8E800207B85F8F900207885F8F8000020616885F8FC008046C5F846
:20452000C080C5F8C480C5F8C8802B4AC5F8EC10217E12F8211085F8FA10F989A5F8F61081
:20454000237B002B0CBF1021494685F8FE00C5F8F010387B05F0B8FA30460DF009FC97F86E
:204560003B0085F8FB00304609F0F0FB684615F049FB787900966B463979184A01902846EC
:2045800010F008FE684615F075FBB96802911449009605F130006A460EF07CFB0FF014F9F4
:2045A000014633460F4AC5F8CC1005F11C00042113F01AFB95F8F80030B905F16C004146A3
:2045C00012F0B8FE084800E0A068C5F8BC00304605B0BDE8F083C046A0C10200B9DD000030
:2045E0001549020015A0020001A102002DE9F0410221ADF1280D8DF81210C188ADF80A1014
:20460000417D8DF814108188ADF81610417E8DF81810818C491E8DF81A10816A4A1C0892E5
:2046200009788DF81910418A808DADF82400374800250768ADF81C10002F31D04FF0D3087C
:204640004FF6FF74BDF81600F988884206D08C4223D1C10BCE0301D113281ED19DF81A00AC
:20466000203080B213F039FF061C16D002A9202214F010FE9DF81A1041B106F120000A465E
:20468000B061089906F1200014F004FE86F80080387931460FF000F801253F68002FD1D190
:2046A0001B4908310A884FF6FF732F4693420CD0BDF816500C460020954220D0401CC0B2CC
:2046C000C2001119A25A9342F6D1DFB9BDF81610C80BC00316D19DF8140098B9132911D04F
:2046E00041F4004100919DF8180001909DF81900842200230DF10A0112F08AFE02E04968D8
:2047000002A888470AB0BDE8F081C046A0FD002044B702002DE9F04FADF1140D02A914F0CD
:2047200083F85FEA000940F08380434F029CFE68218856B1B61F0322002036F8063F9942CB
:2047400005D0521E00F10100F7D1C82601E080460026182008F07EFA051C0ED0002118229D
:204760000AF0F4F8608818212A4615F04DFC4FF6FF706080284610F00FFA4FF6FE7A4FF06D
:20478000000BA4F800A0002E84F804B050D1F868444668B3142008F05DFA5FEA000827D083
:2047A0004C205946022203AB15F016F902255E46F868B44207D0A9B24C2006226B4615F06B
:2047C0000BF9694603E0610001EB84010918A8B20622404414F05EFD761CAD1D032EE7DB9C
:2047E0004C201421424615F00FFC404610F0D4F94C205946022203AB15F0EEF8C0B9FF6885
:204800005FB1610001EB8401BDF80C007A5A5646964204D138B1401E03E0BDF80C00401C91
:2048200080B2ADF80C004C20022103AA15F0ECFB484605B0BDE8F08F54FE0020F0B5ADF151
:204840003C0D12F009FD454E96F84A00082807D0332086F8290086F8270001277765B765D6
:204860006846002124220AF071F83D4D2878012804D0012000278DF80A0002E000278DF834
:204880000A700F2446208DF837400DF13701B47010F0C2FE6D1E8DF82470A87B8DF825007E
:2048A00015F0FEFA8DF826008DF827708DF8287096F85C008DF82A700F28A8BF201C06F13D
:2048C0005D018DF829000DF12B0015F065FC0DF13300FF2103220AF039F896F896008DF8F3
